:100000000C9460180C9499180C9499180C949918E5
:100010000C94758B0C94758B0C94758B0C94758B60
:100020000C9499180C9499180C9499180C9499188C
:100030000C9499180C94F3720C9499180C949918C8
:100040000C9499180C9424710C9448CF0C94991822
:100050000C94C4400C94BA400C9499180C949918C0
:100060000C9499180C9499180C9499180C9499184C
:100070000C9499180C9499180C9499180C9499183C
:100080000C947E330C9499180C94991805A84CCDB7
:10009000B2D44EB93836A9020C50B9918688083CC2
:1000A000A6AAAA2ABE000000803F4E414E494E49F2
:1000B0005459494E46CDCCCC3D0AD7233C17B7D135
:1000C0003877CC2B329595E6241FB14F0A000020DB
:1000D000410000C84200401C4620BCBE4CCA1B0E5A
:1000E0005AAEC59D7400407A10F35A00A0724E18A3
:1000F000090010A5D4E80000E87648170000E40BDA
:1001000054020000CA9A3B000000E1F5050000809F
:10011000969800000040420F000000A086010000F9
:1001200000102700000000E8030000000064000049
:100130000000000A00000000000100000000002C88
:1001400076D888DC674F0823DFC1DFAE59E1B1B74D
:1001500096E5E3E453C63AE651997696E8E6C2841A
:1001600026EB898C9B62ED407C6FFCEFBC9C9F4032
:10017000F2BAA56FA5F490055A2AF75C936B6CF957
:10018000676DC11BFCE0E40D47FEF520E6B500D02D
:10019000ED902E0300943577050080841E08000042
:1001A000204E0A000000C80C333333330F986E1210
:1001B000831141EF8D2114893BE65516CFFEE6DB16
:1001C00018D1844B381BF77C1D901DA4BBE4242060
:1001D0003284725E228100C9F124ECA1E53D2743FF
:1001E0004F4D4D554E49434154494F4E004452598D
:1001F00052554E004552524F525300494E464F0001
:100200004543484F0053544F505045442E20005012
:1002100072696E7465722073746F707065642064A7
:10022000756520746F206572726F72732E20466937
:100230007820746865206572726F7220616E642028
:10024000757365204D39393920746F207265737468
:100250006172742E202854656D70657261747572B8
:10026000652069732072657365742E205365742050
:10027000697420616674657220726573746172744A
:10028000696E67290A004E6F20436865636B73755A
:100290006D2077697468206C696E65206E756D627B
:1002A00065722C204C617374204C696E653A200095
:1002B0004E6F20436865636B73756D207769746852
:1002C000206C696E65206E756D6265722C204C61C4
:1002D0007374204C696E653A2000636865636B73C4
:1002E000756D206D69736D617463682C204C61734A
:1002F00074204C696E653A20004C696E65204E751D
:100300006D626572206973206E6F74204C61737426
:10031000204C696E65204E756D6265722B312C2004
:100320004C617374204C696E653A20004D31313058
:100330000053657269616C20737461747573206D0C
:1003400069736D617463680A005344207265616467
:10035000206572726F720A002121204B494C4C209B
:1003600063617573656420627920746F6F206D75A9
:10037000636820696E6163746976652074696D6570
:10038000202D2063757272656E7420636F6D6D61D0
:100390006E643A20004D3235004D65646961204934
:1003A0006E73657274656400627573793A2070616A
:1003B0007573656420666F7220696E7075740A00CB
:1003C000627573793A2070617573656420666F7227
:1003D00020757365720A00627573793A2070726FC6
:1003E00063657373696E670A00506C65617365209D
:1003F0005265736574005052494E5445522048412D
:100400004C5445440025533A202553004B494C4C4D
:1004100045442E20005072696E7465722068616CCC
:100420007465642E206B696C6C28292063616C6C88
:100430006564210A0053544F505045442E2000500B
:1004400072696E7465722073746F70706564206475
:10045000756520746F206572726F72732E20466905
:100460007820746865206572726F7220616E6420F6
:10047000757365204D39393920746F207265737436
:100480006172742E202854656D7065726174757286
:10049000652069732072657365742E20536574201E
:1004A0006974206166746572207265737461727418
:1004B000696E67290A006563686F3A004572726F5A
:1004C000723A0042696C696E656172204C657665AE
:1004D0006C696E6720477269643A0A0021212053D3
:1004E000544F502063616C6C656420626563617574
:1004F0007365206F6620424C546F75636820657287
:10050000726F72202D207265737461727420776926
:100510007468204D3939390A0021212053544F5035
:100520002063616C6C65642062656361757365202E
:100530006F6620424C546F756368206572726F72EB
:10054000202D20726573746172742077697468203D
:100550004D3939390A0050726F62696E6720506FE9
:10056000696E740025532025692F2569002E0A0025
:100570002F0050726F62696E67206D65736820701E
:100580006F696E742000202844525952554E29003C
:10059000473239204175746F20426564204C65767E
:1005A000656C696E67003F20284C2C522C462C420B
:1005B00029206F7574206F6620626F756E64732ECC
:1005C0000A003F2856296572626F7365206C657654
:1005D000656C20696D706C61757369626C6520284B
:1005E000302D34292E0A00426164205A2076616C35
:1005F00075650A004E6F2062696C696E65617220D4
:10060000677269640A004732384C30004465766985
:100610006174696F6E0025533A2025730046696E38
:100620006973686564210A003A207A3A2000206FD5
:10063000662000476F696E6720746F3A2058004348
:10064000570A00206469723A0020616E676C653A4F
:10065000005374617274207261646975733A004D5D
:10066000343820506F696E740025533A2025642F6A
:10067000256400506F736974696F6E696E672074CA
:1006800068652070726F62652E2E2E0A003F4C65E1
:100690006773206F66206D6F76656D656E74206977
:1006A0006D706C61757369626C652028302D313511
:1006B000292E0A003F2028582C5929206F757420B4
:1006C0006F6620626F756E64732E0A0050726F62DF
:1006D00065206F7574206F6620626F756E6473009D
:1006E0003F53616D706C652073697A65206E6F741D
:1006F00020706C61757369626C652028342D35300B
:10070000292E0A004D3438205A2D50726F62652010
:100710005265706561746162696C697479205465B1
:1007200073740A003F2856296572626F7365206CE6
:100730006576656C20696D706C61757369626C6556
:100740002028302D34292E0A005374616E646172A2
:100750006420446576696174696F6E3A20002052A6
:10076000616E67653A2000204D61783A2000204D87
:10077000696E3A2000205369676D613A20004D652B
:10078000616E3A200020204D3230312058004D61FA
:100790007820416363656C65726174696F6E2028AF
:1007A000756E6974732F7332290020204D323033F7
:1007B0002058004D617820666565647261746573C8
:1007C0002028756E6974732F732900205200202031
:1007D0004D323034205000416363656C6572617442
:1007E000696F6E2028756E6974732F733229202803
:1007F000503C7072696E742D616363656C3E20526B
:100800003C726574726163742D616363656C3E2034
:10081000543C74726176656C2D616363656C3E292E
:1008200000204A0020540020530020204D32303553
:10083000204200416476616E6365642028423C6D0D
:10084000696E5F7365676D656E745F74696D655F12
:1008500075733E20533C6D696E5F666565647261B9
:1008600074653E20543C6D696E5F74726176656C90
:100870005F66656564726174653E204A3C6A756EA8
:10088000635F6465763E29002044002049002020F3
:100890004D333031205000486F74656E64205049EC
:1008A00044002E0A00206E6F742064697361626CCC
:1008B00065642E20536861726564207769746800EE
:1008C000203B204C6576656C696E67200020204DCA
:1008D0003432302053004175746F20426564204CDF
:1008E0006576656C696E6700204600204800202010
:1008F0004D3134352053004D6174657269616C204F
:1009000068656174757020706172616D657465727F
:100910007300203B2053656E736F722000204400EB
:1009200020204D34313220530046696C616D656E74
:10093000742072756E6F75742073656E736F7200BC
:10094000204A002020473239205720490020204DDE
:100950003134392043203B20556E69747320696E11
:100960002043656C736975730A0054656D70657218
:10097000617475726520556E69747300202047326A
:1009800031203B004C696E65617220556E6974734D
:100990000020496E76616C696420657874727564B4
:1009A00065722000536C6565702E2E2E005A205003
:1009B000726F62652050617374204265640A005A48
:1009C0002050726F6265205061737420426564002C
:1009D000205A3A200020593A200042656420583AB3
:1009E00020004D65736820706F696E74206F757498
:1009F000206F662072616E67650A00436C69636BE5
:100A000020746F20526573756D652E2E2E00616CFB
:100A1000736F20656E61626C6564290A004E6F20F9
:100A20004D6F76652E004E6F206D656469610A001A
:100A3000456E642066696C65206C6973740A0042B7
:100A40006567696E2066696C65206C6973740A005D
:100A5000286E6F2066696C6529004E6F74205344C0
:100A6000207072696E74696E670A00534420707258
:100A7000696E74696E6720627974652000437572CF
:100A800072656E742066696C653A20002E0A004417
:100A9000656C6574696F6E206661696C65642C2095
:100AA00046696C653A200046696C652064656C6532
:100AB0007465643A002569730025696D20256973A2
:100AC000002569682025696D202569730025696402
:100AD000202569682025696D2025697300256979BD
:100AE00020256964202569682025696D20256973A2
:100AF000005072696E742074696D653A20006F6BE6
:100B0000006F6666000002FB01F401ED01DF0144A5
:100B1000454255473A004D3131322053687574646F
:100B20006F776E004D3131332053004D6567612082
:100B30005A65726F204F46462E00434F4E46494736
:100B40005F4558504F5254004D4541545041434B1E
:100B500000434F4F4C45525F54454D504552415410
:100B6000555245004348414D4245525F54454D5012
:100B70004552415455524500424142595354455003
:100B800050494E470041524353004D4F54494F4E38
:100B90005F4D4F44455300544845524D414C5F50C2
:100BA000524F54454354494F4E00455854454E44C6
:100BB00045445F4D3230004C4F4E475F46494C45EF
:100BC0004E414D45004155544F5245504F52545F90
:100BD00053445F5354415455530053445F57524953
:100BE00054450052455045415400534443415244FA
:100BF0000050524F4D50545F535550504F52540077
:100C0000484F53545F414354494F4E5F434F4D4DFE
:100C1000414E445300454D455247454E43595F5060
:100C2000415253455200434153455F4C4947485454
:100C30005F4252494748544E45535300544F47472B
:100C40004C455F4C494748545300534F4654574115
:100C500052455F504F574552004255494C445F50F2
:100C6000455243454E54004C4556454C494E475F0E
:100C700044415441005A5F50524F42450052554E34
:100C80004F5554004155544F4C4556454C00505219
:100C9000494E545F4A4F420050524F4752455353BA
:100CA000004155544F5245504F52545F54454D509A
:100CB000004155544F5245504F52545F504F5300CE
:100CC000564F4C554D455452494300454550524F9F
:100CD0004D0042494E4152595F46494C455F54527E
:100CE000414E534645520053455249414C5F584F7F
:100CF0004E5F584F4646004649524D574152455F58
:100D00004E414D453A4D61726C696E20322E302E47
:100D1000392E332D6B6164312028446563203237CE
:100D200020323032312031333A34383A34352920C8
:100D3000534F555243455F434F44455F55524C3ADC
:100D40006769746875622E636F6D2F6B61642F4DD8
:100D500061726C696E2050524F544F434F4C5F5636
:100D6000455253494F4E3A312E30204D4143484968
:100D70004E455F545950453A4D656761205A65723A
:100D80006F2045585452554445525F434F554E5479
:100D90003A3120555549443A646266636364353597
:100DA0002D656262612D343631352D616264372DD7
:100DB0003139366161343338663330340A002F2FCD
:100DC000004D31343520533C696E6465783E206FA8
:100DD0007574206F662072616E67652028302D3132
:100DE000290A003F4A206F7574206F662072616E79
:100DF00067652028302E303120746F20302E332943
:100E00000A0020580020204D61783A200020002060
:100E1000204D696E3A2000203B200020204D3231C9
:100E20003120530046523A0020466C6F773A20003A
:100E3000206F7574206F662072616E67650A0053BB
:100E40006572766F20003A200020536572766F201D
:100E50000050726F6265204F6666736574205A0099
:100E600050726F6265204F6666736574205A006425
:100E7000697300656E0043290A0061626C65642035
:100E8000286D696E2074656D702000436F6C64205E
:100E900065787472756465732061726520004F46D1
:100EA00046004F4E006D6D00203B20446973746115
:100EB0006E6365200046696C616D656E74207275A5
:100EC0006E6F757420004F46460A004661646520C7
:100ED0004865696768742000426564204C657665E2
:100EE0006C696E6720004661696C656420746F20D0
:100EF000656E61626C6520426564204C6576656C48
:100F0000696E670A00496E76616C6964206D65736D
:100F1000682E0A004D34323120696E636F7272653B
:100F2000637420706172616D6574657220757361A0
:100F300067650A004D65736820706F696E74206F75
:100F40007574206F662072616E67650A00454550B2
:100F5000524F4D204F4B0A00290A0020746F200089
:100F60003F5A206F7574206F662072616E6765202E
:100F70002800290A0020746F20003F59206F7574E3
:100F8000206F662072616E676520282D00290A0097
:100F900020746F20003F58206F7574206F66207298
:100FA000616E676520282D004D383400446F6E65F2
:100FB000207072696E74696E672066696C650A00DC
:100FC0004D3737004D333100496E76616C696420CE
:100FD00065787472756465720A004361703A002026
:100FE000286D6D2900203B0020204D3835312058D8
:100FF000005A2D50726F6265204F666673657400EB
:10100000436F6F6C696E672E2E2E004865617469A0
:101010006E672E2E2E0045312025530020573A00B2
:1010200023646566696E652044454641554C545FAE
:10103000004B6420004B6920004B70200050494455
:10104000204175746F74756E652066696E6973688A
:101050006564212050757420746865206C61737418
:10106000204B702C204B6920616E64204B64206300
:101070006F6E7374616E74732066726F6D2062653B
:101080006C6F7720696E746F20436F6E6669677549
:10109000726174696F6E2E680A0050494420417570
:1010A000746F74756E65206661696C656421207467
:1010B000696D656F75740A00504944204175746FFD
:1010C00074756E65206661696C6564212054656D78
:1010D000706572617475726520746F6F20686967DE
:1010E000680A00504944204379636C6573002553B6
:1010F0002025692F256900204B643A2000204B6988
:101100003A2000204B703A200020436C61737369D1
:101110006320504944200A002054753A2000204B97
:10112000753A2000206D61783A2000206D696E3A92
:10113000200020643A200020626961733A20005741
:1011400061697420666F7220686561742075702E05
:101150002E2E00504944204175746F74756E6520C1
:1011600073746172740A00504944204175746F743D
:10117000756E65206661696C6564212054656D70CB
:101180006572617475726520746F6F206869676835
:101190000A00504944204175746F74756E6520666D
:1011A00061696C65642120426164206865617465D1
:1011B000722069640A00504944204175746F747547
:1011C0006E65004572723A207574663820666F6EDF
:1011D00074206E6F7420696E697469616C697A65D8
:1011E000642E004572723A207574663820666F6E00
:1011F00074206E6F7420696E697469616C697A65B8
:10120000642E004572723A207574663820666F6EDF
:1012100074206E6F7420696E697469616C697A6597
:10122000642E002568753A25303268750025303205
:1012300068753A2530326875002530326875272583
:101240003032687500256875642025303268753A3B
:1012500025303268750042656400456E636C6F73BB
:1012600075726500202020202020200020202020D2
:1012700000453A00523A00657272001FE0201020CB
:1012800010201010201020201020103030084004B2
:101290008003001FE03FF03FF03FF01FE01FE03F02
:1012A000F03FF03FF00FC0078003003FFFF0380031
:1012B0007030FC3020FC102078102030102C00D032
:1012C0002E31D02F7BD02F7BD02E31D02C00D020B0
:1012D000301020781020FC1030FC303800703FFFB8
:1012E000F03FFFF038007031863023871027879059
:1012F0002F87D02F03D02030102078102078102096
:1013000030102F03D02F87D0278790238710318666
:10131000303800703FFFF0001DC43F0000000C8615
:10132000198000000D0E198000000F0B19800000BD
:101330000D9F198000000DD3998000001CFBFF0059
:1013400000000000000000000000000000F380002A
:101350001F80007700001980005B1CF6131DAE5B38
:1013600035AB0635FB5B3DA70CBD9B4B30EB19B194
:101370009BE39D8E9F9D8E0001E0000000000120F8
:101380000000000001E0000000000C0F00FE07025A
:101390002503BB017FFE08FE08FE050808060000C5
:1013A00040F0C88888987810050808060000C0F842
:1013B0008888888888F80505050600012030F830FF
:1013C000200508080600002070F820202020E005F5
:1013D00009090600FF2070A8A8B8888870200705B2
:1013E00005070001D86C366CD80509090600FFF81E
:1013F000A88888888888A8F8050A0A0600FE205070
:1014000050505088A8A8887003030306000340A02A
:1014100040FFFFFFFFFFFFFFFFFFFFFFFFFFFFFF9B
:10142000FFFFFFFFFFFFFF0000000605FF010707AA
:10143000060200808080808000800303030601058F
:10144000A0A0A005060606000050F85050F8500570
:1014500009090600FF2070A8A07028A870200507C1
:1014600007060000C8C81020409898050707060026
:101470000040A0A040A890680103030602058080F8
:10148000800309090601FF20404080808040402001
:101490000309090601FF80404020202040408005CC
:1014A000070706000020A8702070A8200505050683
:1014B00000012020F820200203030601FFC0408025
:1014C000050101060003F8020202060100C0C00582
:1014D0000707060000081010204040800507070697
:1014E0000000708898A8C8887003070706010040AC
:1014F000C040404040E00507070600007088081023
:101500002040F8050707060000F80810300888702A
:1015100005070706000010305090F8101005070767
:10152000060000F880F0080888700507070600002C
:10153000304080F0888870050707060000F8081022
:101540001020202005070706000070888870888812
:10155000700507070600007088887808106002058B
:1015600005060100C0C000C0C00206060601FFC09B
:10157000C000C040800305050601012040804020D6
:10158000050303060002F800F803050506010180C3
:1015900040204080050707060000708810202000CA
:1015A000200507070600007088B8A8B880700507F6
:1015B00007060000708888F88888880507070600F5
:1015C00000F04848704848F005070706000070889A
:1015D0008080808870050707060000F0484848486A
:1015E00048F0050707060000F88080F08080F805C5
:1015F0000707060000F88080F08080800507070656
:1016000000007088808098887005070706000088B1
:101610008888F8888888030707060100E040404072
:101620004040E005070706000038101010109060D9
:101630000507070600008890A0C0A090880507074E
:10164000060000808080808080F805070706000083
:1016500088D8A8888888880507070600008888C871
:10166000A8988888050707060000708888888888F9
:1016700070050707060000F08888F0808080050765
:101680000706000070888888A8906805070706008C
:1016900000F08888F0A09088050707060000708891
:1016A0008070088870050707060000F820202020B9
:1016B000202005070706000088888888888870052C
:1016C000070706000088888888505020050707060D
:1016D000000088888888A8A85005070706000088A9
:1016E0008850205088880507070600008888502009
:1016F000202020050707060000F80810204080F889
:101700000309090601FFE080808080808080E00579
:101710000707060000804040201010080309090652
:1017200001FFE020202020202020E0050303060008
:10173000052050880501010600FEF8030303060199
:1017400005804020050505060000700878887805AA
:1017500007070600008080F0888888F005050506E8
:101760000000708080887005070706000008087870
:10177000888888780505050600007088F080700567
:101780000707060000304840E040404005070706D4
:1017900000FE7088888878087005070706000080BA
:1017A00080F0888888880307070601004000C04051
:1017B0004040E00409090601FE100030101010102E
:1017C000906005070706000080808890E0908803FD
:1017D0000707060100C04040404040E005050506FF
:1017E0000000D0A8A8A8A8050505060000B0C88874
:1017F0008888050505060000708888887005070739
:101800000600FEF0888888F080800507070600FE45
:1018100078888888780808050505060000B0C88023
:10182000808005050506000078807008F005070730
:101830000600002020F820202018050505060000DD
:1018400088888898680505050600008888885020E3
:101850000505050600008888A8A8500505050600AE
:101860000088502050880507070600FE88888850A9
:10187000204080050505060000F8102040F8030907
:10188000090601FF204040408040404020010909F6
:101890000602FF80808080808080808003090906A6
:1018A00001FF804040402040404080050303060087
:1018B0000248A890FF5045544700504C41005072D8
:1018C000696E742041626F72746564004D32350038
:1018D00050617573696E672E2E2E004D32340045AF
:1018E0004550524F4D2056657273696F6E20457298
:1018F000726F7200454550524F4D20496E646578B5
:10190000204572726F7200454550524F4D20435230
:1019100043204572726F72003F0049676E6F7265B7
:1019200000526573657400496E697469616C697A07
:101930006520454550524F4D0000FE0003FF8007D3
:10194000C7C00701E00000E00000F00000700400E4
:10195000700E00701F00703F80F00E00E00F01E07D
:1019600007C7C003FF8000FE0000FE0003FF8007E2
:10197000C7C00F01E00E00E03F80F01F00700E00B6
:10198000700400700000700000F00000E00701E04B
:1019900007C7C003FF8000FE000E000E000E000E01
:1019A000000E000E000E000E007FC03F801F000ED4
:1019B00000040004000E001F003F807FC00E000ED8
:1019C000000E000E000E000E000E000E00FFFFFFC6
:1019D0007F80FFC0FFC0FFC07F807F80FFC0FFC04F
:1019E000FFC03F001E000C0050726F6265205A203D
:1019F0004F6666736574002008204661637400209A
:101A000008204D6178002008204D696E004F666601
:101A1000004F6E004175746F74656D7000452073E2
:101A2000746570732F6D6D005A2053746570732F39
:101A30006D6D00592053746570732F6D6D005820C3
:101A400053746570732F6D6D00416476616E6365CC
:101A5000642053657474696E67730054656D7065B6
:101A60007261747572650053746570732F6D6D00CB
:101A7000436F6E66696775726174696F6E003F00CF
:101A80004E65787420436F726E657200446F6E65A8
:101A9000004E65787400486F6D696E672058595A1A
:101AA0000053746F72652053657474696E677300B8
:101AB0004C6F61642053657474696E67730042658E
:101AC00064205472616D6D696E670050726F62655B
:101AD000205A204F6666736574004661646520482D
:101AE0006569676874004F6666004F6E0042656402
:101AF000204C6576656C696E67004C6576656C2078
:101B0000426564004732394E0047323900417574EE
:101B10006F20486F6D65004D6F74696F6E0053578D
:101B20002D4D6F64650053746F77004465706C6F62
:101B3000790053656C662D54657374005265736546
:101B40007400436F6E66696775726174696F6E00C9
:101B5000526573746F72652044656661756C747349
:101B6000004C6F61642053657474696E6773005331
:101B7000746F72652053657474696E6773004F6685
:101B800066004F6E0052756E6F75742053656E73EC
:101B90006F7200424C546F7563680050726F6265DB
:101BA000205A204F666673657400416476616E63E7
:101BB00065642053657474696E6773004D61696E66
:101BC000003F004261636B0053746F70004D32320E
:101BD00000417474616368204D65646961004D3231
:101BE00031005072696E742066726F6D204D6564AD
:101BF00069610052656C65617365204D656469615A
:101C000000436F6E66696775726174696F6E005428
:101C1000656D7065726174757265004D6F74696F82
:101C20006E00526573756D65205072696E74005454
:101C3000756E650053746F70205072696E74005039
:101C400061757365205072696E7400496E666F200D
:101C500053637265656E000A4D3234004D32332095
:101C60002573003F005374617274205072696E7462
:101C70000043616E63656C005072696E740043616D
:101C80006E6E6F7420656E74657220737562646920
:101C9000723A200002202E2E000152656672657392
:101CA00068004D61696E002100486F74656E6420A4
:101CB000746F6F20636F6C64004261636B005072DD
:101CC0006F63656564004D6F74696F6E004469737E
:101CD00061626C65205374657070657273004D3875
:101CE00034004D34382050726F626520546573742F
:101CF000004732384F0A4D343820503130004265A9
:101D000064204C6576656C696E67004175746F2060
:101D1000486F6D6500473238004D61696E00BA1832
:101D2000B518436F6F6C646F776E005072656865AD
:101D3000617420240046616E205370656564004E16
:101D40006F7A7A6C65004D61696E0050726F6265E2
:101D5000205A204F666673657400466C6F770046A4
:101D6000616E205370656564004E6F7A7A6C650011
:101D70005370656564004D61696E00486F6D696EF2
:101D800067204661696C6564006F70656E0054522F
:101D900049474745524544003A200066696C616DE9
:101DA000656E74007A5F6D696E00795F6D696E00B3
:101DB000785F6D696E005265706F7274696E67202E
:101DC000656E6473746F70207374617475730A0048
:101DD00020746F6F206C6F6E6720657874727573F6
:101DE000696F6E2070726576656E7465640A002096
:101DF000636F6C6420657874727573696F6E2070A0
:101E0000726576656E7465640A00486F6D6520259D
:101E10007325732573204669727374005761726E5F
:101E2000696E673A20486F6D696E672042756D7004
:101E30002044697669736F72203C20310A000202E7
:101E4000040000E0C0000000C000000000000068C6
:101E5000430000634300007A430000A0400000A05C
:101E60004000000040FFFDFCFAF8F6F4F2F0EEEC62
:101E7000EAE9E7E5E3E1E0DEDCDAD9D7D5D4D2D090
:101E8000CFCDCBCAC8C7C5C3C2C0BFBDBCBAB9B726
:101E9000B6B4B3B2B0AFADACAAA9A8A6A5A4A2A18E
:101EA000A09E9D9C9A99989795949392908F8E8DD1
:101EB0008B8A8988878684838281807F7E7D7B7AF6
:101EC000797877767574737271706F6E6D6C6B6AFA
:101ED000696867666564636261605F5E5D5C5B5AEA
:101EE0005958585756555453525150504F4E4D4CC7
:101EF0004B4A4A4948474646454443424241403F8F
:101F00003E3E3D3C3B3B3A39383837363535343345
:101F100032323130302F2E2E2D2C2B2B2A292928EE
:101F2000272726252524232322212120201F1E1E8A
:101F30001D1C1C1B1B1A1919181817161615151419
:101F4000131312121111100F0F0E0E0D0D0C0C0B9E
:101F50000A0A090908080707060605050404030319
:101F600002020100000000000100000001000080EA
:101F700000555555000000400033333300AAAA2A0B
:101F8000004992240000002000C7711C0099991993
:101F900000D1451700555515003BB11300244912D7
:101FA0000011111100000010000F0F0F00E3380E98
:101FB0000043790D00CCCC0C00C3300C00E8A20B20
:101FC0000064210B00AAAA0A00703D0A009DD809EE
:101FD00000427B090092240900DCD30800888808AD
:101FE000001042080000000800F0C10700878707C2
:101FF0000075500700711C07003EEB0600A1BC06EF
:10200000006990060066660600703E0600611806CC
:102010000017F4050074D105005BB00500B290050F
:1020200000627205005555050078390500B81E0597
:1020300000050505004EEC040087D40400A1BD0492
:102040000090A7040049920400C17D0400EE6904D9
:1020500000C7560400444404005C32040008210414
:102060000041100400000004003FF00300F8E0030A
:102070000026D20300C3C30300CCB503003AA80373
:10208000000A9B0300388E0300C08103009F750384
:1020900000D0690300505E03001D53030034480361
:1020A00000913D03003333030016290300381F035A
:1020B0000097150300300C0300030303000BFA0222
:1020C0000049F10200BAE802005CE002002DD802EB
:1020D000002DD0020059C80200B0C0020031B90280
:1020E00000DAB10200AAAA0200A0A30200BC9C026E
:1020F00000FA9502005C8F0200DF880200828202F3
:1021000000457C02002776020027700200436A0225
:10211000007C640200D05E02003F590200C85302F6
:1021200000000061430000614300007A430000E0CA
:10213000C0000000C00000000053657474696E6741
:10214000732053746F726564000000FA430000FA54
:10215000430000A0400000C8410000A0420000A0D1
:10216000420000C8430080C043F4010000F40100B5
:1021700000640000008813000024F4D43050C38EA3
:1021800020C2A24017828B7011127A910D816CD9F6
:102190000AA861E108C7586607615143061E4B5DF6
:1021A00005C145A7041A411104093D98037139314D
:1021B000034036DB0265339102D4305402802E1D79
:1021C00002632CEE01752AC501B028A001102781F9
:1021D000018F2564012B244B01E0223401AC211F27
:1021E000018D200D01801FFC00841EED00971DDF76
:1021F00000B81CD200E61BC600201BBC00641AB24B
:1022000000B219A8000A19A0006A189900D1179104
:102210000040178B00B516840031167E00B3157987
:10222000003A157300C7146F0058146A00EE136665
:10223000008813630025135E00C7125B006C125701
:102240000015125400C111510070114F0021114BA3
:1022500000D61049008D104700461044000210427D
:1022600000C00F4000800F3E00420F3C00060F3BB5
:1022700000CB0E3800930E37005C0E3500270E346D
:1022800000F30D3200C10D3100900D3000600D2EB5
:1022900000320D2D00050D2C00D90C2B00AE0C29A1
:1022A00000850C29005C0C2700350C27000E0C263D
:1022B00000E80B2400C40B2400A00B23007D0B239B
:1022C000005A0B2100390B2100180B2000F80A1FBF
:1022D00000D90A1E00BB0A1E009D0A1D00800A1DAF
:1022E00000630A1C00470A1B002C0A1B00110A1A73
:1022F00000F7091A00DD091900C4091900AB091912
:1023000000920917007B091800630917004C091691
:102310000036091600200916000A091500F50815EF
:1023200000E0081400CC081400B8081400A4081435
:1023300000900813007D0812006B08130058081263
:102340000046081200340811002308110012081179
:102350000001081100F0071000E0071000D007107E
:1023600000C0071000B0070F00A107100091070E72
:102370000083070F0074070F0065070E0057070E54
:102380000049070E003B070D002E070E0020070D29
:102390000013070D0006070D00F9060C00ED060DF1
:1023A00000E0060C00D4060C00C8060C00BC060CAD
:1023B00000B0060C00A4060B0099060C008D060B5D
:1023C0000082060B0077060B006C060B0061060A04
:1023D0000057060B004C060A0042060A0038060A9F
:1023E000002E060A0024060A001A060A0010060932
:1023F0000007060A00FD050900F4050900EB0509C0
:1024000000E2050900D9050900D0050900C7050942
:1024100000BE050900B5050800AD050800A50509C1
:10242000009C050800940508008C05080084050838
:10243000007C050800740508006C050700650508A8
:10244000005D050700560508004E05070047050713
:10245000004005080038050700310507002A050778
:1024600000230507001C050600160507000F0507D9
:10247000000805060002050700FB040600F5040736
:1024800000EE040600E8040600E2040700DB040690
:1024900000D5040600CF040600C9040600C30406E4
:1024A00000BD040600B7040600B1040500AC040634
:1024B00000A6040600A00405009B04060095040580
:1024C00000900406008A04050085040500800406C7
:1024D000007A04050075040500700405006B04050E
:1024E0000066040500610405005C0405005704054E
:1024F00000520405004D040500480405004304058E
:10250000003E0404003A04050035040500300404CC
:10251000002C04050027040400230405001E040405
:10252000001A04040016040500110404000D04043C
:1025300000090405000404040000040400FC030472
:1025400000F8030400F4030400F0030400EC0304A7
:1025500000E8030400E4030400E0030400DC0304D7
:1025600000D8030400D4030400D0030400CC030407
:1025700000C8030300C503030024F404D9201BC4CE
:102580000C5C0E9804C4095F0265077101F405F93B
:1025900000FB04B30048048700C1036900580355D9
:1025A0000003034500BE023A008402310053022AB0
:1025B000002902250004022000E4011C00C80119C2
:1025C00000AF01170098011400840113007101107D
:1025D000006101100051010E0043010D0036010B96
:1025E000002B010B0020010B00150109000C010953
:1025F0000003010800FB000800F3000800EB0007DF
:1026000000E4000600DE000600D8000600D2000646
:1026100000CC000500C7000500C2000500BD000495
:1026200000B9000400B5000400B1000400AD0004CE
:1026300000A9000400A5000300A20003009F0004FD
:10264000009B000300980003009500020093000324
:1026500000900003008D0002008B00030088000240
:10266000008600020084000300810002007F000257
:10267000007D0002007B000200790002007700016B
:102680000076000200740002007200010071000276
:10269000006F0002006D0001006C0002006A000182
:1026A000006900020067000100660001006500018A
:1026B000006400020062000100610001006000018E
:1026C000005F0002005D0001005C0001005B000192
:1026D000005A000100590001005800010057000194
:1026E0000056000100550001005400010053000095
:1026F0000053000100520001005100010050000190
:10270000004F0001004E0000004E0001004D00018E
:10271000004C0001004B0000004B0001004A00018A
:102720000049000100480000004800010047000186
:102730000046000000460001004500000045000181
:10274000004400010043000000430001004200007B
:102750000042000100410000004100010040000172
:10276000003F0000003F0001003E0000003E00016D
:10277000003D0000003D0001003C0000003C000066
:10278000003C0001003B0000003B0001003A00005B
:10279000003A000100390000003900010038000053
:1027A0000038000000380001003700000037000149
:1027B0000036000000360000003600010035000041
:1027C0000035000000350001003400000034000036
:1027D000003400010033000000330000003300012A
:1027E0000032000000320000003200010031000021
:1027F0000031000000310001003000000030000016
:1028000000300001002F0000002F0000002F00000A
:10281000002F0001002E0000002E0000002E0001FD
:10282000002D0000002D0000002D0000002D0001F3
:10283000002C0000002C0000002C0000002C0001E7
:10284000002B0000002B0000002B0000002B0001DB
:10285000002A0000002A0000002A0000002A0001CF
:1028600000290000002900000029000000290000C4
:1028700000290001002800000028000000280000B6
:1028800000280000002800010027000000270000A9
:10289000002700000027000000270001002600009C
:1028A000002600000026000000260000002600018F
:1028B0000025000000250000002500000025000084
:1028C0000025000000250001002400000024000075
:1028D0000024000000240000002400010023000068
:1028E000002300000023000000230000002300005C
:1028F000002300000023000100220000002200004D
:10290000002200000022000000220000002200013E
:102910000021000000210000002100000021000033
:102920000021000000210000002100010020000023
:102930000020000000200000002000000020000017
:10294000002000000020000000200001001F000007
:10295000001F0000001F0000001F0000001F0000FB
:10296000001F0000001F0001001E0000001E0000EC
:10297000001E0000001E000000393000003325005A
:102980000087190000B00F0000DB080000BD040044
:1029900000740200003F01000020436F756E742038
:1029A000583A0045310045002C2073797374656DE9
:1029B0002073746F7070656421204865617465725E
:1029C0005F49443A200048656174696E672046613A
:1029D000696C65640048656174696E672066616949
:1029E0006C6564004572723A204D415854454D5013
:1029F000004D415854454D502074726967676572A7
:102A00006564004572723A204D494E54454D500060
:102A10004D494E54454D5020747269676765726523
:102A20006400202F0020403A007C3C3E5E2B3D3F5E
:102A30002F5B5D3B2C2A225C0043616E6E6F74201D
:102A40006F70656E20737562646972200053442054
:102A500063617264206F6B0A006F70656E526F6FF6
:102A600074206661696C65640A00766F6C756D65CB
:102A70002E696E6974206661696C65640A004E6F28
:102A800020534420636172640A002E0A006F70654F
:102A90006E206661696C65642C2046696C653A201D
:102AA0000046696C652073656C65637465640A0033
:102AB0002053697A653A200046696C65206F70651D
:102AC0006E65643A2000454E4420535542524F559E
:102AD00054494E450A002220706F73002220706115
:102AE00072656E743A2200535542524F5554494E06
:102AF000452043414C4C207461726765743A220052
:102B000053756263616C6C204F766572666C6F778B
:102B1000004578636565646564206D617820535570
:102B200042524F5554494E452064657074683A00CE
:102B3000667265736800646F696E67002066696C11
:102B4000653A20004E6F77200057726974696E678E
:102B500020746F2066696C653A20006D61726C6943
:102B60006E66772E6F726700322E302E392E332D1F
:102B70006B616431001FFFFFFFFFFFFF600000007B
:102B80000001FF400000000000FF80000000000086
:102B90007F83CF00000C303F87FF80000C301F8602
:102BA0007980000C000F8C30C7838C30E78C30CFDD
:102BB000C7CC31F38C30DCECEC33B98C30D86C6C96
:102BC00033198C30D06C0C33198C30D86C0C331911
:102BD0008C30DC6C0E3B198C30CF7C079F198C300D
:102BE000C77C038F19400000000000026000000055
:102BF0000000061FFFFFFFFFFFF870012C0190018E
:102C00002701B0012201C0011D01F00118011002CD
:102C1000130130020E016002090190020401C0029A
:102C2000FF000003FA004003F5008003F000D0032A
:102C3000EB002004E6007004E100E004DC00400545
:102C4000D700C005D2004006CD00D006C8008007DE
:102C5000C3003008BE00F008B900C009B400B00AD3
:102C6000AF00B00BAA00D00CA500000EA000500FC2
:102C70009B00C01096005012910000148C00C015EB
:102C80008700B0178200B0197D00D01B7800001EAD
:102C9000730040206E0090226900F02464004027F9
:102CA0005F0090295A00E02B5500102E5000203074
:102CB0004B0010324600E033410090353C001037A5
:102CC000370070383200A0392D00B03A2800A03B00
:102CD0002300603C1E00103D1900903D1400103E82
:102CE0000F00703E0A00C03E0500003F0000403F5C
:102CF000FBFF803FF6FFC03FF1FF2020506C616E6C
:102D00006E657242756666657242797465733A20C3
:102D1000002046726565204D656D6F72793A20001E
:102D200020436F6D70696C65643A2044656320329E
:102D30003720323032310A00204C617374205570D4
:102D400064617465643A20323032312D30392D306F
:102D500033207C20417574686F723A20286B61645F
:102D60002C20416E796375626963204D656761202F
:102D70005A65726F2041424C20313256290A004D6B
:102D800061726C696E20322E302E392E332D6B61BC
:102D900064310A0020536F66747761726520526552
:102DA0007365740A00205761746368646F6720520A
:102DB000657365740A002042726F776E206F7574B8
:102DC0002052657365740A002045787465726E61DF
:102DD0006C2052657365740A00506F776572557088
:102DE0000A0073746172740A004732385859004DF2
:102DF00031303031006572726F7220777269746998
:102E00006E6720746F2066696C650A00446F6E659A
:102E100020736176696E672066696C652E0A004DC5
:102E2000323900456E6473746F707300255320252A
:102E30006320256320256320256300205A3A002063
:102E4000593A0020583A00656E6473746F707320AD
:102E50006869743A2000000000010200090A0000BD
:102E6000000004030807000000000000000000004C
:102E7000000000000000004D6F76652025736D6D29
:102E8000004D6F766520302E316D6D004D6F76658B
:102E900020316D6D004D6F76652031306D6D004DC8
:102EA0006F76652041786973004D6F7665204578AF
:102EB000747275646572004D6F7665205A004D6FAF
:102EC00076652059004D6F76652058005072696E06
:102ED000742066726F6D204D6564696100FFFFFFAD
:102EE000205A3A200020593A200042656420583A7E
:102EF00020004D656761205A65726F2052656164DC
:102F0000792E005072696E74696E672E2E2E0050F5
:102F100072696E74205061757365640020450020ED
:102F20005A0020590020204D393220580053746532
:102F300070732070657220756E6974003B200022EA
:102F40000A00556E6B6E6F776E20636F6D6D616EEC
:102F5000643A2022006F6B00DB0FC93F45BCDA3FAB
:102F60008FB30240FCF0274056946140FE4B9B40DB
:102F700084A5D840E0231841346A5641E859974166
:102F800064DBD5416E271742B4B75542CE1A97423B
:102F9000C8AED542B5885A43D40684BFA65FA7BF42
:102FA0007443E0BF10B11AC01C2C58C0E8F697C09B
:102FB000B849D6C04E4E17C124D355C1802497C1FD
:102FC000A0B5D5C1121A17C244AE55C2781797C220
:102FD0006CACD5C267885AC320746F6F206C6F6E5B
:102FE0006720657874727573696F6E20707265768C
:102FF000656E7465640A0020636F6C642065787484
:10300000727573696F6E2070726576656E74656433
:103010000A006F6B0A00526573656E643A200020E7
:10302000453A00205A3A0020593A00583A00000028
:103030002200250028002B0000002100240027008A
:103040002A0002020202020202020404040404042E
:10305000040403030303030303030101010101014A
:103060000101010204081020408001020408102020
:103070004080010204081020408080402010080495
:1030800002014572726F722077726974696E6720EF
:10309000746F20454550524F4D210A005448455207
:1030A0004D414C2052554E4157415900546865726C
:1030B0006D616C2052756E6177617900ECDBB7E26F
:1030C00011241FBECFEFD0E4DEBFCDBF84B7809305
:1030D000521514BE0FB6F894A895809160008861CF
:1030E00080936000109260000FBE12E0A0E0B1E09B
:1030F000EAEDF3EE01E00BBF02C007900D92A83994
:10310000B107D9F725E1A8E9B2E001C01D92A235C7
:10311000B207E1F718E1CFE5D8E104C02197FE013D
:103120000E94C0EECE35D107C9F70E94A8DC0C94EE
:10313000E1F10C940000FC01A081B1811C92A281FC
:10314000B3818C918F5F8C930280F381E02D90810D
:103150008CE0989F800D1124EBE4F3E113AE84AF73
:103160000895FC0184910895FC01808108950097E1
:1031700051F0FC0180E09191992331F0907C9038DE
:10318000D1F38F5FF8CF80E00895119800C087FDDC
:1031900043C0419800C0119A00C000C0119800C0FF
:1031A00086FD46C0419800C0119A00C000C0119829
:1031B00000C085FD3BC0419800C0119A00C000C00E
:1031C000119800C084FD30C0419800C0119A00C021
:1031D00000C0119800C083FD25C0419800C0119A1D
:1031E00000C000C0119800C082FD1AC0419800C004
:1031F000119A00C000C0119800C081FD0FC0419815
:1032000000C0119A00C000C0119800C0419800C0D1
:10321000119A00C000C00895419ABCCF419AF0CFE6
:10322000419AE5CF419ADACF419ACFCF419AC4CFA4
:10323000419AB9CF90E080E00895CF93DF93DB010E
:10324000F9019C919130C1F0943080F094509C939E
:103250008830D1F480819181009771F0019791833A
:103260008083480F591FEA01188206C08C3539F453
:103270009C5F9C93943041F4DF91CF9108958B3300
:1032800039F781E08C93F8CF20813181B9016F5FEC
:103290007F4F71836083420F531FEA0188838081CF
:1032A00091818F3591056CF7E7CF0F931F9381E0E4
:1032B00000919D1410919E1420919F143091A014A0
:1032C0004091991450919A1460919B1470919C14A0
:1032D000041715072607370708F480E01F910F91A0
:1032E000089590E080E008952091FC03833021F45C
:1032F00025FD0CC024FD0CC030E0A90102C055958D
:1033000047958A95E2F7CA018170089581E0089592
:1033100080E008958091180484FD0BC080911A0408
:1033200087FD07C090911B04937081E019F480E041
:10333000089581E008952FEB280F2A3108F047C047
:10334000E22FF0E08091180490911904A0911A04E2
:10335000B0911B0404C0B695A795979587952A95BB
:10336000D2F780FD02C081700895E250FC4FE081E9
:10337000EE2341F180916A0790916B07E80FF92FD6
:10338000F11D808190ED980F9A3030F08E3251F41B
:10339000818180538A3098F4F093ED03E093EC033D
:1033A00081E008958D3211F08B3249F4818190EDE6
:1033B000980F9A3088F38E3211F48281EACFF0E0D0
:1033C000E0E0EACF1092ED031092EC03E9CF80E049
:1033D0000895CF93DF9385E4AEDF882309F188E079
:1033E000409118045091190460911A0470911B04C3
:1033F000972F9170C92F90E0D92FCC0FDD1F71FB53
:10340000222720F930E0220F331F220F331FC22B57
:1034100067FB442740F9C42B8C2BDF91CF91089593
:1034200080E0DECF88DF882341F081E02091EC034B
:103430003091ED03232B09F480E008951092B70337
:103440008091570190915801A0915901B0915A0172
:1034500080937F0590938005A0938105B0938205AA
:103460000895B0E0A0E0E7E3FAE10C94E4EE6B012C
:10347000E9014A3009F4D5C0453109F081C0DB01CA
:103480001296ED91FC91F28096818781139A00C08B
:103490000000E6E2F0E03197F0F7092F182FEF2C4B
:1034A000E29420EFE22230E1B32EBF0CE80188EF76
:1034B0006CDE00C0000086E290E00197F0F7BFE10B
:1034C000BF1508F49BC08F2D807780685EDE8E2D3F
:1034D0005CDE00C0000086E290E00197F0F780E833
:1034E00054DE80E052DE00C0000086E290E00197EA
:1034F000F0F78AEF4ADE00C0000086E290E0019714
:10350000F0F7005F1F4F8881807F3FDE89918295B1
:10351000807F3BDEC017D107B1F700C0000086E214
:1035200090E00197F0F7F394E0E1EE0EFB10BECFD0
:103530001398D6011296ED91FC9180819281980F9B
:1035400092832181921708F09FC194819F5F948399
:103550009381890F821710F08FEF820F838345814B
:1035600050E0440F551F70E060E0868197810E9413
:103570008DF181E0CDB7DEB7E9E00C9400EFDEC15C
:10358000FB0102811381423309F485C108F48DC126
:10359000463409F475C1473409F482C14B3349F705
:1035A00089812B81D80112967C91129713963C91B8
:1035B000213009F4BFC1233009F0A0C148EF480F02
:1035C000582F91E0341708F490E031E0541708F0D8
:1035D00030E0492F432B61E0571708F460E04623A1
:1035E00011F4932331F2FA8030E0F901E156FE4FF5
:1035F000D08025563E4FF901E08099C180EE8F0DB5
:103600008068807FC2DD8F2D8295807FBEDD00C007
:10361000000086E290E00197F0F780E8B6DD80E8F0
:1036200061CF0B9A1398399A4198099A119A139A73
:1036300000C0000086E290E00197F0F788E790E094
:10364000CEE9DFE0FE013197F1F70197D9F788EF76
:103650009CDD00C0000086E290E00197F0F780E278
:1036600094DD80E092DD00C0000086E290E00197EA
:10367000F0F780E08ADD80E888DD00C0000086E2A7
:1036800090E00197F0F780E080DD80E17EDD00C012
:10369000000086E290E00197F0F7CE010197F1F784
:1036A000CE010197F1F7CE010197F1F7CE01019715
:1036B000F1F7CE010197F1F7CE010197F1F7CE01B5
:1036C0000197F1F7CE010197F1F7CE010197F1F7DC
:1036D000CE010197F1F7CE010197F1F7CE010197E5
:1036E000F1F7CE010197F1F7CE010197F1F721979C
:1036F000F1F780E24ADD80E448DD00C0000086E2A8
:1037000090E00197F0F780E240DD80E63EDD00C00A
:10371000000086E290E00197F0F7D0E0C0E08C2F47
:103720008077806832DD8D2F30DD00C0000086E2BA
:1037300090E00197F0F780E828DD80E026DD00C00A
:10374000000086E290E00197F0F78AEF1EDD00C0EE
:10375000000086E290E00197F0F780E2119800C047
:10376000419800C0119A00C000C0119800C0419853
:1037700000C0119A00C000C0119800C0419800C05C
:10378000119A00C000C0119800C0419800C0119A61
:1037900000C000C0119800C0419800C0119A00C03C
:1037A00000C0119800C0419800C0119A00C000C02C
:1037B000119800C0419800C0119A00C000C0119833
:1037C00000C0419800C0119A00C000C0119800C00C
:1037D000419800C0119A00C000C0119800C04198E3
:1037E00000C0119A00C000C0119800C0419800C0EC
:1037F000119A00C000C0119800C0419800C0119AF1
:1038000000C000C0119800C0419800C0119A00C0CB
:1038100000C0119800C0419800C0119A00C000C0BB
:10382000119800C0419800C0119A00C000C01198C2
:1038300000C0419800C0119A00C000C000C0000044
:10384000E6E2F0E03197F0F7815009F087CF88EF9A
:103850009CDC00C0000086E290E00197F0F7CF5FAB
:10386000D05FC03209F05BCF80E08FDC80EC8DDC74
:1038700000C0000086E290E00197F0F7139879CE3F
:10388000F8018581888375CE80E0CDB7DEB7E9E0A9
:103890000C9400EF53C0B901C8010E9492CF69CEC9
:1038A000D80111968C91888364CE443191F04731D0
:1038B00009F05FCE1882D80112968C9112978983F5
:1038C00015968C91159781508A8313968C918B83D2
:1038D00050CED80115964C91159750E0440F551FC6
:1038E00070E060E016968D919C910E948DF1F80138
:1038F000128280818150838314823BCE381708F472
:1039000038CE871708F435CEFA80E12CD12C24303C
:1039100070F46ACEBE01C8010E9492CF898198815D
:103920009D0D98838E0D8983FF0C09F422CEF7FE3E
:10393000F6CFF0CF58E0580F482F43CEEF92FF92CA
:103940000F931F93CF93DF93EC018B017A018A854C
:103950009B858617970731F0888199810E947FD1D6
:103960001B870A87B701888199810E9482C92E81AD
:103970003F81820F932F911D9F838E8390E080E083
:10398000CDB7DEB7E6E00C9403EFB0E0A0E0EBECDF
:10399000FCE10C94E3EEEC017B018A018A859B85B6
:1039A0008617970731F0888199810E947FD1FB8625
:1039B000EA8688859985019609F5CC80DA808E8122
:1039C000D80EA880B980D5015596ED91FC91C5011E
:1039D0000995C80E780110E0F70121917F012111AE
:1039E0001FC08E819F81810F911D9F838E8390E0E8
:1039F00080E0CDB7DEB7EAE00C94FFEEEE80FF800A
:103A0000B801888199810E9482C98E0D9F2D911DD8
:103A1000288539852817390780F681E090E0E9CFBD
:103A20004C2D6D2DC5010E94D7D1D80E180FD4CFC3
:103A3000B0E0A0E0EEE1FDE10C94E6EEEC01D62E64
:103A40001CAD0BAD7C0184E0E80EF11CE98DFA8D14
:103A5000C7010995412F480F2D2D602FC7010E94E6
:103A6000D7D19BAD890F8BAF81E090E0CDB7DEB7AA
:103A7000E7E00C9402EFA6E0B0E0E1E4FDE10C9495
:103A8000DCEE7E836D83342EFC01408051806280A9
:103A90007380C301B20120E13EE040E050E00E94AB
:103AA00023EE49015A0189018CE3C82ED12CE12C67
:103AB000F12CC301B201A70196010E9423EE698394
:103AC0007A838B839C83CA01B901A70196010E9466
:103AD00023EE6B017C01332061F1C301B20120E8C8
:103AE00031E541E050E00E9423EE29013A015901FD
:103AF000DF92CF92C40168E170E00E9499EE9F933B
:103B00008F935F924F9285E492E19F938F93FE8112
:103B1000FF938D818F930E948EE70FB6F894DEBFDE
:103B20000FBECDBF88E0FAE04F165104D8F089E00F
:103B300019C081149104D1F48A818F9399819F9344
:103B4000DF92CF9289E392E19F938F93EE81EF937F
:103B5000FD81FF930E948EE70FB6F894DEBF0FBE83
:103B6000CDBF85E02696E1E10C94F8EE0436110510
:103B700068F4DF926F939F928F928DE292E19F9310
:103B80008F939E819F93ED81EF93E4CFDF926F93AC
:103B90009F928F9283E292E19F938F939E819F9356
:103BA000ED81EF930E948EE70FB6F894DEBF0FBE53
:103BB000CDBF86E0D7CF682F70E090E080E00C9416
:103BC0007FB08091EC039091ED03009731F04AE0D3
:103BD00050E070E060E00C9416E660E070E0CB012D
:103BE00008958091EC039091ED03009731F04AE045
:103BF00050E070E060E00C94E9E460E070E0CB013C
:103C00000895EFDF97FD0AC0ECDF6F3F7105810576
:103C1000910509F02CF4E5DF862F089580E00895E2
:103C20008FEF0895CF93C62FFDDB882311F0E9DFD6
:103C3000C82F8C2FCF9108958091EC039091ED03C4
:103C4000892B39F0DEDF91E0811101C090E0892FEE
:103C5000089591E0FCCFCF93DF93C82FD62FE2DBFE
:103C6000882321F0E9DFDF91CF9108958C2F63DB6A
:103C70008111F9CF8D2FF7CFB4DFCB010895CF930A
:103C8000DF93EB01CFDB882311F0F6DFEC01CE01EF
:103C9000DF91CF9108950F931F93CF938091EC0301
:103CA0009091ED030097D9F0FC018F01C1912C2F69
:103CB0002F7D81F0C53411F0C536B9F7F8011082B7
:103CC00070E060E00E9493E3F801C083CF911F9100
:103CD0000F91089570E060E00E9493E3F7CF60E0F9
:103CE00070E0CB01F3CFCF92DF92EF92FF926A01A7
:103CF0007B0198DB882319F0CEDF6B017C01C701C3
:103D0000B601FF90EF90DF90CF900895CF92DF92B1
:103D1000EF92FF92CF93C82F0E943ECE6B017C01A1
:103D200024EA30E74DE75FE36091310170913201A1
:103D300080913301909134010E94F5E787FD18C00E
:103D40008AEF90E0A0E0B0E08C0D9D1DAE1DBF1D80
:103D50008093670490936804A0936904B0936A0405
:103D6000C0932701CF91FF90EF90DF90CF900895FF
:103D700080E090E0DC01E8CFCF93809128048111AE
:103D800054C01092861310928713109288131092C9
:103D900054131092531310925613109255131092FD
:103DA000581381E08093571382E280935913109245
:103DB0005E1310925D13E2E7F3E120E833E18FEF49
:103DC00081932E173F07E1F7C1E0C0936F1323EBF8
:103DD0003EEA3093651320936413C09366131092E8
:103DE00067131092681390E49093691310926A130A
:103DF00022EB3EEA30938113209380132FE131E0D0
:103E000030935213209351139EE19093761391E1D6
:103E1000909377139CE19093741380937313809322
:103E200072130E94D1CFC093280481E080932704AD
:103E300084E692E190938212809381121092841210
:103E40001092831253985B9A52985A9A3898409AD3
:103E50000E9473AB10927704CF910895FC0180E02B
:103E6000309749F09491992331F0907C903809F083
:103E70008F5F3196F7CF0895B0E0A0E0E2E4FFE174
:103E80000C94E3EEEC015B018A01FB01099587FDCF
:103E900010C0C82ED12CF12CE12C2196F801C08243
:103EA000D182E282F382CE01CDB7DEB7EAE00C9494
:103EB000FFEE982F907E903CA9F48F7190E0B0E0D7
:103EC000A0E06C017D0156E0CC0CDD1CEE1CFF1C5B
:103ED0005A95D1F7CE010196F50109958F73C82A3D
:103EE0002296DCCF982F907F903E11F58F7090E056
:103EF000B0E0A0E06C017D0136E0CC0CDD1CEE1CD6
:103F0000FF1C3A95D1F7CE010196F50109958F7303
:103F1000C82A46E0CC0CDD1CEE1CFF1C4A95D1F7EC
:103F2000CE010296F50109958F73C82A2396B6CF64
:103F3000982F987F903F79F5877090E0B0E0A0E0EF
:103F40006C017D0186E0CC0CDD1CEE1CFF1C8A950B
:103F5000D1F7CE010196F50109958F73C82A96E035
:103F6000CC0CDD1CEE1CFF1C9A95D1F7CE010296FD
:103F7000F50109958F73C82A26E0CC0CDD1CEE1CD8
:103F8000FF1C2A95D1F7CE010396F50109958F7391
:103F9000C82A249683CF982F907C903841F4807C57
:103FA000803869F42196CE01F5010995F8CF8E7F0E
:103FB0008D3F28F02196CE01F5010995F8CFC12C4F
:103FC000D12C76016BCF9CE0899F802D112491E04C
:103FD000980F909326042CE0280F2093540730E08C
:103FE0002E5F3F4F409183134217130619F014F0D0
:103FF00080E00895209185139217D0F7662341F051
:104000008E5F0E94B6D0809154078E5F0E94B6D01A
:104010008091540790918313891750F32091851351
:1040200090912604291720F310928613809387130A
:1040300081E0089520912504022E000C330B821795
:10404000130641F08093250469E873E18FE493E15E
:104050000C947FD10895ACE0B0E0E1E3F0E20C9481
:10406000E5EE6F3F71058105910509F070F48BE471
:1040700093E1DEDCE0915313F09154133196849177
:1040800090E02C96E8E00C9401EFF0908613E0901D
:1040900087132091270421110FC043E052E16E2DB8
:1040A0008F2D0E9430D290E080E0F80EF0928613BF
:1040B000E09287139927E5CFC0905313D090541303
:1040C0002FE433E13A8329832F2D30E03C832B8387
:1040D0002E2D30E03E832D8318861F822FEF3FEF79
:1040E0003A8729871C861B8605EC1CE19E012F5F01
:1040F0003F4FAB01BC01C6010E94C1AFB6018FE4C6
:1041000093E10E947FD18F819885CFCF4F925F92AC
:104110006F927F928F929F92BF92CF92DF92EF9297
:10412000FF920F931F93CF93DF93CDB7DEB72897FE
:104130000FB6F894DEBF0FBECDBF7C016A01490106
:10414000FB0190818CE0989F800D1124982FF7013E
:104150002081822F880F820F880F8093861390937F
:1041600087134115510561F1FA82E9827C836B83E3
:1041700001111FC0AE014B5F5F4FB401C6017CDE71
:104180006C016D817E818F81988561157105810536
:104190009105B1F060DFF70180818F5F8083853109
:1041A00048F3CE0101960E949B18E4CFB12C860102
:1041B00029C08A01B12C26C0452846284728B1F7D6
:1041C00028960FB6F894DEBF0FBECDBFDF91CF911A
:1041D0001F910F91FF90EF90DF90CF90BF909F9035
:1041E0008F907F906F905F904F900895B39407C029
:1041F000B1102DC001151105C9F20F5F1F4F011538
:104200001105A9F2AE014B5F5F4FB401C60134DE68
:104210006C014D805E806F8078844114510461048C
:104220007104A9F0F0E24F1651046104710401F326
:10423000D301C2018D97A109B1090297A105B1056A
:1042400030F04BE2441651046104710479F6F70131
:104250008081482F4B0D5527551F4631510534F0AD
:10426000853020F0CE0101960E949B1881E0411418
:1042700051046104710409F480E0B80EF7018081F3
:104280008B0D8083BB2009F497CFBA94AE014B5FAE
:104290005F4FB401C801F0DD8C016D817E818F819B
:1042A0009885D9DEEFCFCF93DF93FC0125AD2111A7
:1042B00004C021E025AF0E94D1CFC0915113D0910D
:1042C0005213E0918013F091811382E00995E091FF
:1042D0008013F091811381E0099530E020E044E102
:1042E000BE018FE493E10E94CCCF22E833E147E1A5
:1042F000BE018FE493E10E94CCCFE0918013F09156
:10430000811380E00995DF91CF9108954F925F92DC
:104310006F927F928F929F92AF92BF92CF92DF92D5
:10432000EF92FF92CF93DF9300D000D0CDB7DEB7EE
:104330000E943ECE6B017C01809127018F3FC1F12D
:104340000E943ECE8090670490906804A09069041B
:10435000B0906A04681979098A099B0997FD28C0F9
:1043600080913713909138138F5F8F70891701F107
:10437000E0912701E53008F0DCC024E0E29FF00185
:104380001124ED55FE4F80819181A281B3818983F3
:104390009A83AB83BC8320E030E0A901BE016F5F4C
:1043A0007F4F87E791E00E94F5C38FEF809327014D
:1043B0000E9473AB8091780482FFC4C08091760420
:1043C00081111DC091E09093760480917D0489272E
:1043D0008093300710927D0483E080936C011092EB
:1043E00078040E943ECE6C507E4F8F4F9F4F60935B
:1043F000790470937A0480937B0490937C04809179
:10440000720490917304A0917404B0917504A70193
:104410009601281B390B4A0B5B0BDA01C901B7FF68
:1044200005C080917E04882309F4C5C1D701C60167
:104430008C599F4FAF4FBF4F80937204909373047A
:10444000A0937404B093750460917704062E000C59
:10445000770B77FF03C0719561957109909177048F
:1044600080917104981371C0633008F06EC010928F
:1044700077048091770480937104643008F075C0EC
:10448000809130078111F3C08091491390914A13B4
:104490008F519C4241F480912801882309F4F9C08E
:1044A0008150809328010E94047780908407909027
:1044B0008507A0908607B090870781110E94117729
:1044C000D501C4013AE0B695A795979587953A9599
:1044D000D1F7009741E0A407B10520F08FEF9FEFDF
:1044E000A0E0B0E09695879520916C012111E3C082
:1044F00030917E0431118BC18091491390914A1300
:104500008F519C4209F46AC180917F04811166C178
:1045100080916D0490916E04A0916F04B09170042D
:10452000C81AD90AEA0AFB0AF7FC66C10E94A38EE0
:1045300063C180916D0190916E01A0916F01B09166
:10454000700125CF109276045ACF633009F091CFD5
:104550008091770487FD07C081E0880F880F8093E2
:10456000770464E086CF8FEFF8CF8091530721E086
:1045700030E040E050E0882309F456C080904F07B7
:1045800090905007A0905107B09052078114910469
:10459000A104B104E9F170E090E080E00E94F9E745
:1045A00020E030E040E85EE30E945AE82B013C0145
:1045B000C701B601681979098A099B090E94F9E7C0
:1045C0009B01AC01C301B2010E948DEF20E030E0FD
:1045D0004AE754E40E945AE84B015C0120E030E0D5
:1045E00040EA52E40E94B2F024E630E040E050E0BD
:1045F00087FF12C020E030E040EF51E4C501B40174
:104600000E94B2F02AE030E040E050E087FF04C0B2
:1046100021E030E040E050E0C0924F07D0925007D8
:10462000E0925107F0925207A09177040A2E000CF5
:10463000BB0B0E946BEE24E030E040E050E00E94B3
:1046400045EE80914B0790914C07A0914D07B0919A
:104650004E07820F931FA41FB51F80934B079093A3
:104660004C07A0934D07B0934E0710927704D701E3
:10467000C6018856954CAF4FBF4F80936D04909301
:104680006E04A0936F04B093700481E080936C017A
:10469000FBCE8CE08093280180916B0490916C0498
:1046A000009729F0019790936C0480936B0481E04C
:1046B00080936C01F8CE009741F040916B045091CB
:1046C0006C044817590708F017CF80917E048111B8
:1046D00011C0223038F0243008F43FC0243011F4E7
:1046E00010926C018BE493E1DEDD81E080934A0758
:1046F00080937E0483E09EDC81E080936F13E091E1
:104700004913F0914A13099510924A0780917E044B
:10471000811127C0109230078091491390914A135C
:104720008F519C4209F0F0CE0E943ECEDC01CB01BD
:104730008C199D09AE09BF0980906B0490906C04A0
:10474000B12CA12C88169906AA06BB0608F0D4CE77
:1047500090936C0480936B04CFCE81E080936C01C6
:10476000C1CF8FE493E10E944FD191E0811101C04C
:1047700090E090937E04882369F280914913909190
:104780004A138F519C42B9F40E943ECEDC01CB010A
:104790008C199D09AE09BF09C0906B04D0906C04C0
:1047A000F12CE12CC816D906EA06FB0620F49093FA
:1047B0006C0480936B040F900F900F900F90DF911B
:1047C000CF91FF90EF90DF90CF90BF90AF909F90F0
:1047D0008F907F906F905F904F90089548E9C40E3E
:1047E0004AE3D41EE11CF11CC0926D04D0926E0409
:1047F000E0926F04F092700480917E048111DBCF0F
:1048000080916C018130B9F610926C01D4CF009781
:1048100009F470CF52CFACE0B0E0E1E1F4E20C94E7
:10482000E5EEF0908613E090871320912704211184
:1048300012C043EE51E16E2D8F2D0E9430D290E0D8
:1048400080E0F80EF0928613E092871399272C9659
:10485000E8E00C9401EFC0905313D09054132FE470
:1048600033E13A8329832F2D30E03C832B832E2D97
:1048700030E03E832D8318861F827A8769871C86E5
:104880001B8605EC1CE19E012F5F3F4F41EB58E179
:10489000BC01C6010E9456B0B6018FE493E10E94AC
:1048A0007FD18F819885CDCFA4E0B0E0EAE5F4E236
:1048B0000C94E1EE7C01062F5A01122F862F660F11
:1048C000990B9C0129563E4F690186E0882E912C58
:1048D00011160CF03DC0AE014F5F5F4F61EB78E108
:1048E000C701CADA7C0169817A818B819C8161155B
:1048F00071058105910561F16D33710581059105A2
:1049000009F450C06E3771058105910509F44AC05C
:104910006A3271058105910501F507FF11C08AE52D
:1049200092E10E3F11F086E592E136E01302B0010C
:10493000112471DF66E070E00E94ADEE161B60C0CE
:1049400065E470E080E090E086DB115069F510E0EE
:10495000812F2496ECE00C94FDEE64327105810504
:10496000910571F4A114B104D1F0E6E01E02B0018A
:104970001124C50150DFB4010E94ADEE161BA8CF73
:10498000603471058105910551F41150F601608183
:10499000062E000C770B880B990B5DDB99CF5BDB48
:1049A000115096CF07FDBBCF61E089819A81AB8121
:1049B000BC81CD97A105B10509F460E0600F6A30B4
:1049C000A4F01150862F6AE00E948CEE092F682F08
:1049D000880F770B605D7F4F072E000C880B990BBB
:1049E0003ADB112309F4B3CF602F062E000C770BAE
:1049F000605D7F4F072E000C880B990B2CDB11504C
:104A0000112309F4A4CF86E01802B0011124C701D4
:104A100002DF66E070E00E94ADEE161B99CFEBE47A
:104A2000F3E183AF64AF6FEF7FEFCA01F4CEACE088
:104A3000B0E0EDE1F5E20C94E5EEF0908613E09045
:104A4000871320912704211112C043EC51E16E2DF0
:104A50008F2D0E9430D290E080E0F80EF092861305
:104A6000E092871399272C96E8E00C9401EFC09010
:104A70005313D09054132FE433E13A8329832F2D1D
:104A800030E03C832B832E2D30E03E832D8318862F
:104A90001F827A8769871C861B8605EC1CE19E01B4
:104AA0002F5F3F4F44EB58E1BC01C6010E9456B056
:104AB000B6018FE493E10E947FD18F819885CDCF9D
:104AC0006FEF7FEFB4CFB0E0A0E0E9E6F5E20C9441
:104AD000E3EE5C016B01C2D9E82EC6010E94B71853
:104AE000F12C03E110E0081B1109C5E20E151F05AA
:104AF0000CF4CFE18C2F90E09C012E5F3F4F409152
:104B000083134217130609F08CF50997209185133A
:104B1000281719065CF1409156075091570760918C
:104B2000550710928613C093871325E1C501BCDE9B
:104B3000D1E0C114D104A9F06AE370E080E090E014
:104B40008ADA0E151F05A4F4C45F80918313C81779
:104B500040F0209185134C2F4950550B2417150612
:104B60004CF4CDB7DEB7EAE00C94FFEED0E0E1CF35
:104B7000DD23B9F3802F880F080F000F00938613F1
:104B8000C093871360E270E080E090E064DAC601D1
:104B900097DFE7CFACE0B0E0E0EDF5E20C94E1EEBA
:104BA000982F862F6A017901B02E692F0CDA88239D
:104BB00009F487C010912704C701002371F14ED971
:104BC000A82E8090531390905413111142C02FEFD0
:104BD0003FEF122F23E12A194091560750915707B2
:104BE00060915507C60160DEAA2009F46AC0B6E0EC
:104BF0008B9F600111246AE370E080E090E02BDA83
:104C000057E0C516D10408F442C060E270E080E0CD
:104C100090E021DAC81AD90AF3CF0E94B718A82E5B
:104C20008090531390905413112389F2FE01339610
:104C30008AE0DF011D928A95E9F78FE493E19A8378
:104C400089830EE91CE19E012F5F3F4F44EB58E141
:104C500012C0FE0133968AE0DF011D928A95E9F7C2
:104C60008FE493E19A8389830EE91CE19E012F5F13
:104C70003F4F41EB58E1B701C4010E9456B0B40167
:104C80008FE493E10E947FD12F813885A2CF40919C
:104C90005407212F30E0A6E0AA9EC00111242E5F08
:104CA0003F4F281739070CF49C0180E8821B809342
:104CB000861340938713BB2041F06FEF7FEFC7014E
:104CC000AADD2C96ECE00C94FDEEC701F9DEF9CFDD
:104CD0000C94DCB04F925F926F927F928F929F9272
:104CE000BF92CF92DF92EF92FF920F931F93CF93D9
:104CF000DF9310921D0410921C042FE320932004D4
:104D000010921F0410921E0410921804109219049D
:104D100010921A0410921B049C01F90190812F5FDC
:104D20003F4F9032D1F39E34C9F4818190ED980FBA
:104D30009A3020F08D3211F08B3281F432969F013F
:104D40002F5F3F4F808180538A3008F46DC09F01F0
:104D50002F5F3F4F8081803209F468C0F0936B076A
:104D6000E0936A078F010F5F1F4FC0816AE270E016
:104D7000C8010E94A7F1009731F0FC0131978081B2
:104D80008032E1F31182CD3421F0C43511F0C73403
:104D9000D9F5F80180810F5F1F4F8032D1F3805326
:104DA0008A3090F5C093200490E080E06AE0AF0183
:104DB0004F5F5F4F689F9001699F300D1124C901BB
:104DC000C0972081820F911D27FD9A95FA012081BD
:104DD00020532A3060F390931F0480931E04DF0158
:104DE00031962C912032D9F3CD3461F58E31910575
:104DF00039F0F0F48731910519F08C31910511F5F6
:104E0000B0931D04A0931C04DF91CF911F910F91CB
:104E1000FF90EF90DF90CF90BF909F908F907F900A
:104E20006F905F904F900895F90189CFF9018FCF6E
:104E30008537910538F08737910510F3803A13E0F4
:104E40009107F1F280906A0790906B0740E050E084
:104E5000BA0130E020E0C12CD12C7601C394FD01D1
:104E60003196DC91DD2309F484C0D132F1F4CD34E4
:104E7000E1F480329105C9F4409318045093190469
:104E800060931A0470931B04F0931D04E0931C04B8
:104E900063E270E0CF010E94A7F1009709F4B4CF5C
:104EA000FC011082B1CFDF01DACFD154DA3108F042
:104EB0005BC0DF011D91103291F0A0EDA10FAA306F
:104EC000E8F01E3271F4A181A053AA30B8F0211588
:104ED000310519F49F0121503109B12C13C0FD0196
:104EE000E8CF1D3211F01B3291F7A181B0EDBA0F5E
:104EF000BA3020F0AE3259F7A281E6CFBE2EB818F4
:104F0000309759F3AD2FB0E02601370104C0440CAF
:104F1000551C661C771CDA95D2F744295529662959
:104F20007729A250BC4FBC92A081A154AA3108F4A9
:104F3000BACFDF01D191DD2309F491CF00EDB02E7E
:104F4000BD0E19E01B15A8F713EDB12EBD0E11E033
:104F50001B1578F7DB3269F3FD013196DC91D03215
:104F600009F07DCFDF01F8CF21153105E9F69D016C
:104F7000DBCF30931D0420931C04409318045093FE
:104F8000190460931A0470931B043ECFFC016591D1
:104F9000759185919491089580E00C94CD898F92BC
:104FA0009F92AF92BF92CF92DF92EF92FF92CF93F8
:104FB000DF93EC018090990490909A04A0909B0458
:104FC000B0909C0420E030E0A901C501B4010E942A
:104FD000F5E7882309F452C0C880D980EA80FB80B5
:104FE000A7019601C501B4010E94F5E718160CF05F
:104FF0004AC02091E8033091E9034091EA035091BF
:10500000EB03C701B6010E94F5E7882321F1C092A6
:10501000E803D092E903E092EA03F092EB032091D7
:10502000E4033091E5034091E6035091E703C701A3
:10503000B6010E945AE89B01AC0160E070E080E894
:105040009FE30E9412EF6093140170931501809307
:1050500016019093170160911401709115018091D0
:10506000160190911701DF91CF91FF90EF90DF90A3
:10507000CF90BF90AF909F908F90089560E070E0C8
:1050800080E89FE3F0CF60E070E0CB01ECCFB0E0D0
:10509000A0E0EDE4F8E20C94DDEEEC012091610576
:1050A0003091620540916305509164056881798172
:1050B0008A819B810E9412EF4B015C012091650562
:1050C0003091660540916705509168056C817D813E
:1050D0008E819F810E9412EF6B017C01A5019401DA
:1050E00060910C0170910D0180910E0190910F0162
:1050F0000E94F5E7882309F454C080920C01909235
:105100000D01A0920E01B0920F012091DC033091AD
:10511000DD034091DE035091DF03C501B4010E941D
:105120005AE82B013C010E9426F04B015C0120E073
:1051300030E040EA50E40E94F5E7181634F4812C80
:10514000912CC0EAAC2EC0E4BC2E20E030E0A901D6
:10515000C501B4010E94B2F087FF03C0812C912CDD
:105160005401A5019401C301B2010E9412EF6093A2
:10517000D4037093D5038093D6039093D703C501CE
:10518000B4010E94F5EF6093D203062E000C770B5A
:105190006F5F7F4F6630710514F066E070E06093DA
:1051A000D003D0910A011091D203A701960160911A
:1051B00010017091110180911201909113010E94D0
:1051C000F5E7811123C0D11375C02091B803309148
:1051D000B9034091BA035091BB036091D40370911D
:1051E000D5038091D6039091D7030E945AE820916D
:1051F000BC033091BD034091BE035091BF030E9498
:1052000013EFCDB7DEB7E0E10C94F9EEC0921001D8
:10521000D0921101E0921201F09213012091E0036B
:105220003091E1034091E2035091E303C701B601DD
:105230000E945AE84B015C010E9426F06B017C0140
:1052400020E030E040EA50E40E94F5E7181634F41C
:10525000C12CD12CB0EAEB2EB0E4FB2E20E030E0E4
:10526000A901C701B6010E94B2F087FF03C0C12C9B
:10527000D12C7601A7019601C501B4010E9412EF5D
:105280006093D8037093D9038093DA039093DB0380
:10529000C701B6010E94F5EF6093D303062E000C00
:1052A000770B6F5F7F4F6630710514F066E070E03A
:1052B0006093D103C091D303D11305C080910B013A
:1052C0008C1709F470C08091D2039091D30390930E
:1052D0000B0180930A010C2E000CDD0B27E012035A
:1052E000C0011124FC01EC0FFD1FEE0FFF1FEE0F9C
:1052F000FF1FE356FB4F2081318142815381209370
:10530000CC033093CD034093CE035093CF03009151
:10531000D103002E000C110BFC01E00FF11FEE0F6A
:10532000FF1FEE0FFF1FE356FB4F608171818281EB
:1053300093810E9412EF6093C8037093C903809316
:10534000CA039093CB032091D00337E02303F001ED
:105350001124CE0FDF1FCC0FDD1FCC0FDD1FC35676
:10536000DB4F288139814A815B812093C4033093CC
:10537000C5034093C6035093C703E00FF11FEE0F20
:10538000FF1FEE0FFF1FE356FB4F6081718182818B
:1053900093810E9412EF6093C0037093C1038093C6
:1053A000C2039093C3038090D8039090D903A09038
:1053B000DA03B090DB032091C8033091C903409118
:1053C000CA035091CB03C501B4010E945AE8209151
:1053D000CC033091CD034091CE035091CF030E9476
:1053E00013EF6B017C01C092BC03D092BD03E0922D
:1053F000BE03F092BF032091C0033091C1034091DE
:10540000C2035091C303C501B4010E945AE8209120
:10541000C4033091C5034091C6035091C7030E9455
:1054200013EFA70196010E9412EF6093B8037093E7
:10543000B9038093BA039093BB03C7CEACE0B0E04E
:10544000E4E2FAE20C94EAEE182F882379F020E0E7
:1054500030E0A9016091690570916A0580916B0542
:1054600090916C050E94F5E78823F1F080919804F3
:105470008117D1F00E9430748CE0EBE8F1E0DE019E
:10548000119601900D928A95E1F7CE010196FFDD0C
:1054900080919804882361F087E791E00E948674E8
:1054A000109298040E947F872C96E3E00C9406EFFC
:1054B00081E08093980487E791E00E945274F2CFD4
:1054C000CF92DF92EF92FF9280E0B8DF10926505F5
:1054D000109266051092670510926805109261059A
:1054E00010926205109263051092640510926D058A
:1054F00010926E0510926F0510927005109269055A
:1055000010926A0510926B0510926C054DE954E0FB
:1055100027E0C12CD12C60ECE62E6FE7F62E90E050
:1055200080E0FC01EE0FFF1FEE0FFF1FE40FF51FE1
:10553000C082D182E282F38201968730910589F799
:105540002150445E5F4F2111EACFFF90EF90DF9032
:10555000CF9008954F925F926F927F928F929F9219
:10556000AF92BF92CF92DF92EF92FF921F93CF93B1
:10557000DF93EC01162F2091990430919A04409109
:105580009B0450919C04688179818A819B810E944F
:10559000F5E7882309F497C0B090980480E04EDFC7
:1055A000C880D980EA80FB8020E030E0A901C701F3
:1055B000B6010E94B2F087FF03C0C12CD12C760146
:1055C000C0929904D0929A04E0929B04F0929C04B9
:1055D0002DEB37E346E855EBC701B6010E94F5E72E
:1055E00087FD0BC02DEB37E346E855E3C701B60155
:1055F0000E94B2F018160CF076C0A701960160E088
:1056000070E080E89FE30E948DEF6093E403709365
:10561000E5038093E6039093E70380EF9FEFA9E70C
:10562000B4EC8093E8039093E903A093EA03B0936A
:10563000EB03BB2009F447C04090770150907801FC
:105640006090790170907A0180907B0190907C014C
:10565000A0907D01B0907E01C0907F01D09080012C
:10566000E0908101F090820181E0E8DE112359F1A0
:10567000A301920160917701709178018091790185
:1056800090917A010E94F5E781111BC0A501940158
:1056900060917B0170917C0180917D0190917E01F0
:1056A0000E94F5E781110DC020917F0130918001AA
:1056B0004091810150918201C701B6010E94F5E736
:1056C00081110E94CD87DF91CF911F91FF90EF90C4
:1056D000DF90CF90BF90AF909F908F907F906F9012
:1056E0005F904F90089560E070E0CB018ECF8F9275
:1056F0009F92AF92BF92CF92DF92EF92FF92C090B3
:105700006905D0906A05E0906B05F0906C0520E08B
:1057100030E0A901C701B6010E94F5E78823E1F155
:10572000A701960160E070E080E89FE30E948DEFA2
:105730006B017C0180906D0590906E05A0906F05C7
:10574000B090700520E030E0A901C501B4010E94CD
:10575000F5E7882329F1A501940160E070E080E875
:105760009FE30E948DEFC092DC03D092DD03E092B4
:10577000DE03F092DF036093E0037093E103809314
:10578000E2039093E303FF90EF90DF90CF90BF9000
:10579000AF909F908F900895C12CD12C7601CACFE5
:1057A00060E070E0CB01DFCFCF92DF92EF92FF920B
:1057B0006B017C0183E3C816D104E104F10470F0AD
:1057C00082E3C81AD108E108F10862E370E080E0E2
:1057D00090E00E94B5CD0E94E571ECCFC701B60103
:1057E0000E94B5CD0E94E571FF90EF90DF90CF90C1
:1057F0000895BC0190E080E00C947FB08091680730
:10580000813069F09091A11492FB882780F992FF72
:1058100007C097FB882780F991E08927089581E0E8
:1058200008959091A11494FB882780F994FF06C0F5
:1058300081E09091A712911101C080E00895ACE041
:10584000B0E0E5E2FCE20C94DDEE109253078091AB
:10585000300710923007882361F020E040E070E0CC
:1058600060E084E199EA0E94678D2C96E0E10C9457
:10587000F9EE2091390130913A0140914B07509156
:105880004C07CA01820F931F2436310509F0E9C382
:105890004730510544F006978A3091050CF0F0C36B
:1058A0008AE090E0F7C306964A3F5F4FACF38091E1
:1058B0004A07882309F4D0C1609193127091941221
:1058C000072E000C880B990B0E94FBE711E020913A
:1058D0008F123091901240919112509192120E9429
:1058E000B2F018160CF010E01093660480907F015F
:1058F00090908001A0908101B090820120E030E082
:10590000A901C501B4010E94F5E7C12CD12CE0EA40
:10591000EE2EE0ECFE2E87FD06C0C12CD12C70EAE5
:10592000E72E70E4F72E20E030E04AE754E4C501AA
:10593000B4010E945AE8A70196010E9413EF2DECD2
:105940003CEC4CEC5DE30E945AE80E94F5EF6B01E1
:105950007C0180E2F7FE09C0F094E094D094C094FA
:10596000C11CD11CE11CF11C8DE2409077015090CC
:1059700078016090790170907A0120917B013091DB
:105980007C0140917D0150917E0129873A874B87A8
:105990005C878093800460E230E1C31637E2D3066F
:1059A000E104F1048CF0C701B60120E137E240E0E8
:1059B00050E00E9445EECA01B9012AE030E040E023
:1059C00050E00E9445EE605D6093810460E248EE25
:1059D000C41643E0D406E104F1048CF0C701B6011B
:1059E00028EE33E040E050E00E9445EECA01B901E4
:1059F0002AE030E040E050E00E9445EE605D6093B8
:105A00008204C701B60124E630E040E050E00E9485
:105A100045EE6AE0862E912CA12CB12CCA01B90169
:105A2000A50194010E9445EE605D60938304C70167
:105A3000B601A50194010E9445EE6B01CA01B901AE
:105A4000A50194010E9445EECC2009F433C32EE257
:105A500020938404605D6093850450E3C50EC0927A
:105A6000860460E874E08EE594E00E94B2F120E0E4
:105A700030E0A901C301B2010E94F5E720E030E067
:105A800040E05FEB87FD04C020E030E040E05FE3F2
:105A9000C301B2010E9413EF0E94F5EFCB010E94F7
:105AA000478CBC0189E594E00E94B2F120E030E02F
:105AB000A90169857A858B859C850E94F5E720E0A0
:105AC00030E040E05FEB87FD04C020E030E040E0E4
:105AD0005FE369857A858B859C850E9413EF0E9420
:105AE000F5EFCB010E94478CBC0184E594E00E9455
:105AF000B2F18091A11400E117E283FD28C091DE8C
:105B0000882309F4E9C28091991490919A14A09184
:105B10009B14B0919C140097A105B10509F4DCC257
:105B2000BC01CD01615F784D8F4F9F4F20E137E27F
:105B300040E050E00E9423EE60919D1470919E140D
:105B400080919F149091A0140E9423EE89010E94DD
:105B50009D8B4B015C018D829E82AF82B886D62ED2
:105B6000809126018017C1F100932601C80164E6E7
:105B700070E00E9499EE7B0188E48E9DB0018F9DBC
:105B8000700D112490E080E00E94F9E72AE037EDE3
:105B900043E25CE30E945AE80E94FAEF60935304E8
:105BA0000115110509F09BC210924E041092440495
:105BB00080E8809343048EE494E0FC01019000208F
:105BC000E9F7CF018E549440982F990F890F880FD1
:105BD00090E8981B9093420480912501D816E1F13A
:105BE0008092250141E08D819E81AF81B88580380A
:105BF0009145A140B10508F440E062E374E0CE01B4
:105C000005960E943B1D982F990F990F891B880FAD
:105C1000805880933104282D2370822EE9F40115D9
:105C20001105A9F0A0E1B7E2A01BB10B2D813E81C7
:105C30004F8158850E9461EE980150E040E00E943B
:105C400023EE211531054105510509F06EC2109270
:105C5000440480E8809343040E943ECE00912A04CD
:105C600010912B0420912C0430912D046B017C01A8
:105C7000C01AD10AE20AF30A9701860137FD11C062
:105C8000209129042095209329046A547C4F8F4F3A
:105C90009F4F60932A0470932B0480932C0490935D
:105CA0002D04D090290411E0D11001C010E081E052
:105CB0000E941A2080918313873180F4809185138C
:105CC000843060F037E1E32E33E1F32E03E126E088
:105CD00044E069E08FE493E10E9455D28091831300
:105CE0008431B8F480918513823098F0DD2009F476
:105CF00035C280918807882309F430C281EE92E191
:105D00007C0102E123E042E068E68FE493E10E9437
:105D100055D2809183138C3108F06EC040908F1261
:105D2000509090126090911270909212A0909312E5
:105D3000B0909412843198F480918513883078F073
:105D40008091660480FF0DC283E992E17C010CE042
:105D500022E048E064E48FE493E10E9455D2809110
:105D60008313883040F4B7FEFFC147E752E167E094
:105D700082E40E940F25809183138C31B0F48091CE
:105D80008513843190F020E030E040E05FE3C30110
:105D9000B2010E9413EF0E94F5EF77FF0EC247E7B2
:105DA00052E16CE182E40E940F25809183138C31D3
:105DB00018F5809185138431F8F080918807882345
:105DC000D9F024E6829FC001112481589F4F6FEFC4
:105DD00070E00E94ADEECB010E94C68C27E62093B6
:105DE00086132CE1209387130E94602565E270E002
:105DF00080E090E00E942B2014DD882379F18091CF
:105E00008313843358F5809185138A3238F107E083
:105E100028E04AE26AE28FE493E10E94FCD005E0C8
:105E200022E04CE262E38FE493E10E94FCD024E0A4
:105E30004AE061E38AE20E94CCD0609151137091F4
:105E4000521382E380936B138BE280936C132BE6E7
:105E500033E142E38FE493E10E94CCCF809183133E
:105E6000853350F480918513813330F024E04AE487
:105E700061E386E30E94CCD080918313843368F47D
:105E800080918513823348F002E02091530442E36D
:105E900067E38FE493E10E94FCD080918313803309
:105EA00058F580918513883238F18091300481173C
:105EB00051F080912F04109330048F5F833008F0ED
:105EC000A5C180932F0480912F048111A2C18091DC
:105ED0004E04882389F0809142048093861380E3E6
:105EE000809387138EE494E00E94602565E270E061
:105EF00080E090E00E942B2080918313883208F08C
:105F00005DC0809185138D3108F458C02BE040E8C6
:105F10006DE180E00E94CCD080918313873208F03D
:105F20004DC0809185138F3108F448C083E0809381
:105F3000861306E20093871368E570E080E090E046
:105F40000E942B208BE08093861300938713DD2023
:105F500009F491C189E594E00E94602588E280936C
:105F6000861306E20093871369E570E080E090E015
:105F70000E942B2080E38093861300938713DD20FB
:105F800009F49EC184E594E00E9460258DE480932D
:105F9000861306E2009387136AE570E080E090E0E4
:105FA0000E942B2085E58093861300938713DD20C4
:105FB00009F4ABC18EE594E00E94602580918313C3
:105FC000833348F5809185138B3228F183E00E945A
:105FD0001A2083E08093861303E30093871366E01F
:105FE00070E080E090E00E942B2081E00E941A2067
:105FF0008091390190913A010E94C68C2CE0209347
:106000008613009387130E94602565E270E080E0AC
:1060100090E00E942B2080918313813408F025CCDE
:1060200080918513863308F420CC109286138EE37A
:106030008093871380E290E10E94B718082F863181
:1060400008F088C180E290E10E946025053109F4E2
:106050000CCC60E270E080E090E00E942B200F5FAB
:10606000F5CF243631054CF48536910504F58A3098
:10607000910534F48AE090E009C084369105BCF0C3
:10608000883EE3E09E0714F087EE93E02817390777
:1060900009F40DCC90933A018093390110924B078B
:1060A00010924C0710924D0710924E0700CC84E6D8
:1060B00090E0F0CF662351F02EE220938404605DDF
:1060C0006093850480E280938604CBCC80E2809349
:1060D000850480938404F6CF10E000E038CD2E2DA7
:1060E00080E2243628F08E2D64E60E9480EE805DEA
:1060F0008093840490E22A3040F03AE0822F632FAC
:106100000E9480EE0E9480EE905D90938504822F25
:106110006AE00E9480EE905D9093860464E874E0EB
:106120008EE494E00E94B2F146CD29833A834B83FA
:106130005C8381E0203831454140510508F480E01E
:10614000482F64E474E0CE0101960E943B1D982F15
:10615000990F990F891B880F80587CCD8BEA92E1AB
:10616000CFCD8BE792E1F2CDC5010E94C68CFC0138
:10617000808193E0803229F4818192E0803209F4B9
:1061800091E0892F880F880FE92EE81A8E2D855B04
:106190008093861387E08093871323E030E0291BE8
:1061A0003109CF01820F931F0E94602569E070E0E2
:1061B00080E090E00E942B20DECDCB010E94C68CB7
:1061C000FC01808193E0803229F4818192E0803269
:1061D00009F491E0892F880F880FF92EF81A8F2D76
:1061E000855B809386138CE18093871323E030E0F6
:1061F000291B3109CF01820F931F0E94602569E09E
:1062000070E080E090E00E942B20CFCD10922F0410
:106210005ACE8230B1F480914404882391F044E74F
:1062200052E160E386E30E940F258091430480934E
:10623000861380E38093871384E494E00E946025B2
:106240005BCE80913204882309F456CE86E3809396
:10625000861300E3009387136FEF7FEF81E792E1EE
:106260000E940B248091310480938613009387133E
:1062700082E394E0E3CF87E00E942C8380FF15C087
:1062800029E5E22E24E0F22EF70161917F016623D9
:1062900009F464CE6F320CF06FE3062E000C770B1E
:1062A000880B990B0E942B20EFCF8091580780FD1F
:1062B00051CE6FEF7FEF8CE692E10E940B244ECE21
:1062C00087E00E942C8381FF15C094E5E92E94E0BD
:1062D000F92EF70161917F01662309F457CE6F32E1
:1062E0000CF06FE3062E000C770B880B990B0E94C5
:1062F0002B20EFCF8091580781FD44CE6FEF7FEFC9
:106300008CE692E10E940B2441CE87E00E942C8310
:1063100082FF15C08EE5E82E84E0F82EF70161912A
:106320007F01662309F44ACE6F320CF06FE3062E2C
:10633000000C770B880B990B0E942B20EFCF8091DC
:10634000580782FD37CE6FEF7FEF84E692E10E941F
:106350000B2434CE80912E041817B1F000911F1039
:1063600010932E0480E290E10E94B718081708F0FD
:1063700050C00F5FE02FF0E0E05EFF4E8081807C38
:106380008038B9F300931F10E0901F10F12C970193
:10639000205E3F4E7901C9010E94B718182F60E8AE
:1063A00070E0C7010E941725153108F05ECA60E24F
:1063B00070E080E090E00E942B20143109F455CA6F
:1063C00060E270E080E090E00E942B20133109F43D
:1063D0004CCA60E270E080E090E00E942B20123115
:1063E00009F443CA212F30E02E5F3F4F4AEF4203AA
:1063F000B001439F700D112460587F4F80E290E1FF
:106400000E94172560E270E080E090E00E942B205F
:106410002CCA10921F10B8CF80916807823059F0B3
:1064200000DA882349F08091A11482FB882780F943
:1064300091E08927089581E0089581E00895DC01C5
:10644000EC918E2F90E0FC01EE0FFF1FE80FF91F7B
:10645000E250FD4E80818F7780830895892B79F4F7
:106460001092900082E0809391001092950010921B
:106470009400C19A809171008260809371000895A8
:10648000B0E0A0E0E6E4F2E30C94E0EEEC017B0186
:1064900088818C3008F0A4C090E0FC01EE0FFF1F53
:1064A000E80FF91FE250FD4E80818F770E9407B3FD
:1064B00019821A8288812CE0622F0E9480EE829FCE
:1064C000B001112430E020E0AB01420F531FFA016C
:1064D000EE0FFF1FE40FF51FE250FD4E908197FD78
:1064E00007C02F5F3F4F2C30310571F790E0B6DFCA
:1064F0007880072D10E06801CC0CDD1CF601E00F60
:10650000F11FE250FD4E80818068808377FC68C077
:1065100080E2E81682E0F8060CF03FC08A8128E5A8
:1065200032E0281B310987FD3395220F331F220FDC
:10653000331F032E000C440B550B898178E8872EFE
:10654000912C881A910887FD9394880C991C880CCB
:10655000991C092C000CAA08BB0860E070E0CB0174
:10656000F7FC0AC0B701653B710514F064EB70E0FD
:10657000072E000C880B990B281939094A095B0969
:106580000E9414EE24EB30E040E050E00E9445EE23
:10659000820E931EA41EB51E74018BE08715D8F0E1
:1065A000298188E890E0821B910927FD9395880F47
:1065B000991F880F991FE816F906BCF402972FB7A8
:1065C000F894E601C00FD11FC250DD4E880F991F0D
:1065D0009A8389832FBF62E370E080E090E0E4D883
:1065E000CDB7DEB7EDE00C94FCEE2A8188E592E0B1
:1065F000821B910927FD9395880F991F880F991F7A
:10660000E816F906DCF6C701D9CFCF93DF93EB018B
:10661000682F70E083E293E133DF688179818A81BA
:106620009B81643F21E072078105910520F464EFAE
:1066300071E080E090E0B8D886B182958170DF91FA
:10664000CF910895A4E0B0E0E8E2F3E30C94EBEE20
:106650008EEE92E0A0E0B0E089839A83AB83BC83A6
:10666000BE016F5F7F4F8AE5D0DF2496E2E00C9495
:1066700007EFA4E0B0E0EFE3F3E30C94EBEE8EEE73
:1066800092E0A0E0B0E089839A83AB83BC83BE0133
:106690006F5F7F4F8AE0B9DF2496E2E00C9407EF4A
:1066A000A4E0B0E0E6E5F3E30C94EBEE84EF91E0D8
:1066B000A0E0B0E089839A83AB83BC83BE016F5FA7
:1066C0007F4F8CE3A2DF2496E2E00C9407EFA4E076
:1066D000B0E0EDE6F3E30C94EBEE84EF91E0A0E0A4
:1066E000B0E089839A83AB83BC83BE016F5F7F4F29
:1066F00080EA8BDF2496E2E00C9407EF1F920F9262
:106700000FB60F9211240BB60F922F933F934F9316
:106710005F936F937F938F939F93AF93BF93EF9309
:10672000FF938091A80387FF27C0109295001092D5
:1067300094008091A8038F5F8093A8038091A803A1
:10674000082E000C990B209122132817190629F006
:1067500024F08091A8038C30DCF18091940090911A
:106760009500049680349C4908F47DC08091940083
:1067700090919500049679C08091A803082E000C92
:10678000990B209122132817190699F294F2E0919F
:10679000A8038E2FEE0F990BFC01EE0FFF1FE80FE1
:1067A000F91FE250FD4E808187FFC3CFE091A8031F
:1067B0008E2FEE0F990BFC01EE0FFF1FE80FF91F54
:1067C000E250FD4E808160E08F770E9459CDB1CFBD
:1067D0002091940030919500E091A8038E2FEE0F48
:1067E000990BFC01EE0FFF1FE80FF91FE250FD4E61
:1067F00081819281820F931F9093990080939800DA
:10680000E091A8038E2FEE0F990BFC01EE0FFF1FF6
:10681000E80FF91FE250FD4E808187FF11C0E09123
:10682000A8038E2FEE0F990BFC01EE0FFF1FE80F50
:10683000F91FE250FD4E808161E08F770E9459CDB3
:10684000FF91EF91BF91AF919F918F917F916F9148
:106850005F914F913F912F910F900BBE0F900FBE04
:106860000F901F90189580E49CE990939900809375
:1068700098008FEF8093A803E3CF9091C00095FF1D
:10688000FCCF8093C6000895CF93DF93EC018991EC
:10689000882311F0F2DFFBCFDF91CF910895CF93E2
:1068A000DF93EC018991882311F0E7DFFBCF8DE0C6
:1068B000E4DF8AE0E2DFDF91CF910895CF93DF93A9
:1068C000EC01FE0184912196882311F0D6DFF9CFE7
:1068D000DF91CF9108950F931F93CF938C01C62F13
:1068E0008AED9FE0EBDFC801E9DF8AE3C6DF80E3E2
:1068F0008C0FC3DF8AE0C1DFCF911F910F91089504
:10690000CF92DF92EF92FF926A017B01D7DF42E0E4
:10691000C701B6010E9426B3FF90EF90DF90CF90A1
:106920000895CF93DF9361EF7FE00E9473C4C0911D
:106930003213D0913313488159816A817B8188EE6B
:106940009FE0DEDF4C815D816E817F8182E29FE28C
:10695000D7DF40912E1350912F1360913013709117
:1069600031138FE19FE2CCDF85EE9FE0A7DF8FED53
:106970009FE0A4DF8AE081DFDF91CF910895C0DF3F
:106980008AE07BCFAEE4B0E0E8ECF4E30C94DBEE1D
:1069900070E060E085E40E943F1E9AA789A78111FC
:1069A0007CC26EEB70E083E50E943F1E3C0165E017
:1069B00070E083E40E943F1E8C0160E085E50E9448
:1069C0002B1E8DAF60E086EB91E10E9409A20E9430
:1069D0003ECE69877A878B879C87809169019091E9
:1069E0006A010E976816790654F087E691E166DF32
:1069F0000E94F7C4C25BDF4FE2E10C94F7EE2985F9
:106A00003A854B855C85205E314B4F4F5F4F2BABFA
:106A10003CAB4DAB5EAB83E591E150DF0E945C7116
:106A20008FE78093951281E080936B0160E08FE3A4
:106A300091E10E9409A289859A85AB85BC85898BE5
:106A40009A8BAB8BBC8B8BA79CA7ADA7BEA7198ECF
:106A50001A8E1B8E1C8E19A21AA21BA21CA21982AE
:106A60001A821B821C822FE730E040E050E02D8725
:106A70003E874F87588B80E090E4ACE1B6E48D838D
:106A80009E83AF83B8871D8A1E8A1F8A188EFFE7F0
:106A9000CF2ED12CE12CF12C2F961FAE2F971FA6B5
:106AA00018AA19AA1AAA1DA21EA21FA218A691E02E
:106AB0009FAB312C212C812C912C54019301072C5C
:106AC000000C440B550B22962CAF3DAF4EAF5FAF81
:106AD0002297402F002E000C550B5CAF4BAFC3012B
:106AE0004E969C01092E000C440B550B26962CAF9C
:106AF0003DAF4EAF5FAF2697CC979C01990F440BEB
:106B0000550B2A962CAF3DAF4EAF5FAF2A9736E0BC
:106B1000631A7108C301072C000CAA0BBB0B2E963D
:106B20008CAF9DAFAEAFBFAF2E9780916B01882326
:106B300009F48DC00E943ECE2B013C0110918805C6
:106B4000112309F473C00E94AC71109288058090E3
:106B50008F1290909012A0909112B0909212A50175
:106B600094016D897E898F89988D0E94B2F087FF8C
:106B700004C08D8A9E8AAF8AB88EA50194016D816A
:106B80007E818F8198850E94F5E7181624F48D8206
:106B90009E82AF82B88622966CAD7DAD8EAD9FADE4
:106BA00022970E94FBE76D8F7E8F8F8F98A39FA9FE
:106BB0002D8D3E8D4F8D58A1992309F472C1C501C9
:106BC000B4010E94B2F018168CF5D301C2012989D4
:106BD0003A894B895C89821B930BA40BB50BAC01E2
:106BE000BD01485853416109710977FD1FC04D85AA
:106BF0005E856F8578894C195D096E097F097595E9
:106C0000679557954795409395128DA39EA3AFA383
:106C1000B8A78D8D9E8DAF8DB8A18D8B9E8BAF8BC0
:106C2000B88F49865A866B867C861FAA26966CADDD
:106C30007DAD8EAD9FAD26970E94FBE7A501940127
:106C40000E94F5E787FF21C088EB90E137DE1092C4
:106C50006B010E945C71CCCE4BEEC42ED12CE12C8A
:106C6000F12C76C124E130E040E050E02D873E87F2
:106C70004F87588B34E1C32ED12CE12CF12C76C1F7
:106C8000CD86DE86EF86F88A71C1D301C2012BA5BD
:106C90003CA54DA55EA5821B930BA40BB50BB7FDC0
:106CA00047C089A50E94D1708AE0E7DDD301C20107
:106CB0008053984FAF4FBF4F8BA79CA7ADA7BEA7E0
:106CC0002F969FAD2F9791116FC02FA538A949A975
:106CD0005AA9C501B4010E94B2F018160CF050C0B8
:106CE00020E030E040E050E4C501B4010E9413EF21
:106CF0006FA778AB89AB9AABA3019201205E314BB1
:106D00004F4F5F4F2BAB3CAB4DAB5EAB2E966CAD9C
:106D10007DAD8EAD9FAD2E970E94FBE7A50194013E
:106D20000E94F5E7881F8827881F2F968FAF2F971F
:106D300089859A85AB85BC858D8F9E8FAF8FB8A3D3
:106D400029893A894B895C89281739074A075B07E3
:106D500020F42D8F3E8F4F8F58A38D8D9E8DAF8D3C
:106D6000B8A1481A590A6A0A7B0A91E849169FE4B1
:106D7000590692E16906710460F18AE990E166CFF3
:106D8000D301C2012BA93CA94DA95EA9821B930B7B
:106D9000A40BB50B46EC59E265ED79E2B7FDC8CF1F
:106DA00080E00E946B71C4CF2A966CAD7DAD8EAD34
:106DB0009FAD2A970E94FBE79B01AC01C501B4017E
:106DC0000E94F5E787FFB4CF4CE950E36CEA70E32B
:106DD000E7CFABADBCADA215B3050CF05BC0B3E023
:106DE0002B1631040CF456C08DE390E167DD80E290
:106DF00090E164DD49815A816B817C8189E390E176
:106E0000BEDD80E290E15ADD49A15AA16BA17CA1CF
:106E100085E390E1B4DD80E290E150DD498D5A8D4B
:106E20006B8D7C8D81E390E1AADD2DAD222309F4E9
:106E3000DFCD89819A81AB81BC818093961290933A
:106E40009712A0939812B09399122CEA35EC47E26E
:106E50005EE369A17AA18BA19CA10E945AE860938C
:106E60009A1270939B1280939C1290939D1220E033
:106E700030E543EC50E4698D7A8D8B8D9C8D0E94BA
:106E80005AE860939E1270939F128093A012909381
:106E9000A112AECD0E94862148CE82E991E10EDD9D
:106EA000A9CDC501B4010E94F5E787FFBFCED3018C
:106EB000C20129853A854B855C85821B930BA40B07
:106EC000B50BAC01BD01485853416109710977FD0B
:106ED000ADCE2114310409F4FCC02DA13EA14FA177
:106EE00058A5280F391F4A1F5B1F298B3A8B4B8BE4
:106EF0005C8B2DA13EA14FA158A5281B390B4A0B35
:106F00005B0BC701B6010E9414EE29893A894B89AF
:106F10005C890E9445EECD84DE84EF84F888C20E41
:106F2000D31EE41EF51E34E1C316D104E104F104BE
:106F30000CF498CE4CEEC416D104E104F1040CF02C
:106F40008BCE50E8C516D104E104F1040CF498CEC0
:106F5000CD86DE86EF86F88A8EEF90E0A0E0B0E086
:106F60008C199D09AE09BF096C017D0187E391E190
:106F7000A5DC6D857E858F8598890E94682682E3D1
:106F800091E19CDCC701B6010E9468264D815E81BB
:106F90006F8178858BE291E1B3DC4D895E896F89E1
:106FA000788D84E291E1ACDC33E0231631040CF4FB
:106FB00090C0C701B6010E94FBE720E030E040E846
:106FC00050E40E945AE869837A838B839C832D81E5
:106FD0003E814F8158856D897E898F89988D0E9469
:106FE00012EF2BED3FE049EC5FE30E945AE89B0172
:106FF000AC0169817A818B819C810E948DEF6FAB9E
:1070000078AF89AF9AAF69897A898B899C890E9408
:10701000FBE72FE632E143E85AE30E945AE86D832A
:107020007E838F8398872AE939E949E15FE36FA975
:1070300078AD89AD9AAD0E945AE869837A838B83D3
:107040009C839B01AC010E9413EF2D813E814F81F7
:1070500058850E948DEF69A37AA38BA39CA320E09F
:1070600030E040E05EE36D817E818F8198850E94F3
:107070005AE829813A814B815C810E945AE8698FE4
:107080007A8F8B8F9C8F4FA958AD69AD7AAD8EE109
:1070900091E136DC4D815E816F81788588E191E1F7
:1070A0006EDC89E091E10ADC49815A816B817C8147
:1070B00083E091E125DC49A15AA16BA17CA18DEF70
:1070C00090E11EDC498D5A8D6B8D7C8D87EF90E1B0
:1070D00056DC8D859E85AF85B8898C0D9D1DAE1DB6
:1070E000BF1DB595A79597958795809395124CAD43
:1070F0004F930F933F922F9283EE90E19F938F9344
:107100002EEE30E13F932F931F920E94ECA15FEF90
:10711000251A350A0FB6F894DEBF0FBECDBF2D8DF0
:107120003E8D4F8D58A12D833E834F835887498ACA
:107130005A8A6B8A7C8A1FAB79CD63E378E00E9420
:1071400073C460915A0D70915B0D80915C0D9091AC
:107150005D0D0E94F9E7AB01BC018AE298E0D0DB4B
:1071600040918A0D50918B0D60918C0D70918D0D19
:1071700087E298E0C5DB40918E0D50918F0D6091B4
:10718000900D7091910D84E298E0BADB40916C070C
:1071900050916D0760916E0770916F0781E298E0E2
:1071A000EECBCF93DF9367ED77E00E9473C4CAE420
:1071B000DDE04CA95DA96EA97FA98EEC97E0A0DB6C
:1071C00048AD59AD6AAD7BAD8BEC97E099DB4CAD2A
:1071D0005DAD6EAD7FAD84E298E0D1DBDF91CF9104
:1071E0000895CF93DF9363EB77E00E9473C4CAE402
:1071F000DDE04CA15DA16EA17FA18AEA97E080DB72
:1072000048A559A56AA57BA582E29FE279DB4CA53A
:107210005DA56EA57FA58FE19FE272DB48A959A904
:107220006AA97BA98CE19FE2AADBDF91CF91089547
:10723000CF93DF936EE877E00E9473C4CAE4DDE089
:10724000688179818A819B810E94F9E7AB01BC0149
:1072500085E897E055DB6C817D818E819F810E945E
:10726000F9E7AB01BC0182E29FE24ADB68857985E0
:107270008A859B850E94F9E7AB01BC018FE19FE203
:107280003FDB6C857D858E859F850E94F9E7AB018C
:10729000BC018CE19FE273DBDF91CF910895AF9247
:1072A000BF92CF92DF92EF920F931F93CF93DF9312
:1072B0005B01EA016901882309F452C08EE797E077
:1072C000FDDAF501608171818281938146E00E943F
:1072D00026B3E1100AC085E797E0F0DA688179818A
:1072E0008A819B8146E00E9426B38EE697E0E6DA2B
:1072F000F601608171818281938143E00E9426B30F
:1073000087E697E0DBDAF801608171818281938101
:1073100043E00E9426B38EE597E0D0DAF6012081A3
:10732000318142815381F801608171818281938131
:107330000E9412EF43E00E9426B3EE2099F08AE00B
:107340009CDA89E497E0BADA688179818A819B8145
:1073500046E00E9426B38AE090DA8AE08EDA02C024
:10736000E110EFCFDF91CF911F910F91EF90DF9060
:10737000CF90BF90AF900895A6E5B0E0E2ECF9E3BE
:107380000C94DBEE2DB63EB687E00E944783811158
:107390000AC061E086E50E94121E8DA3853090F040
:1073A00084E297E08BDA0FB6F8943EBE0FBE2DBE96
:1073B0000FB6F8943EBE0FBE2DBECA5ADF4FE2E1B3
:1073C0000C94F7EE2DA1222319F084E097E076DAF1
:1073D0006AE080E50E94121E182F8CEF810F8F3219
:1073E00018F080EE96E0DECF60E085E40E942B1E70
:1073F000882309F447C031E038AFE0903213F090B1
:107400003313D7012D913D914D915C91609177019E
:10741000709178018091790190917A010E9413EF27
:10742000AB01BC0188E50E94731E69877A878B8750
:107430009C87F701248135814681578160917B01CA
:1074400070917C0180917D0190917E010E9413EFEB
:10745000AB01BC0189E50E94731E6D877E878F8713
:10746000988BBE01635F7F4FCE0109960E9439C59C
:1074700081110BC063E68CEC96E00E9409A284EBBC
:1074800096E090CF83E088AFB8CF8CE40E949B1940
:10749000082F882309F44EC10E94011E8EA380315B
:1074A00018F08DE896E07ECFFEA1F13009F444C1DA
:1074B00060E083E50E942B1E22968FAF22978823DF
:1074C00021F0011102C037E03EA38DA1833018F0F6
:1074D00083E796E0F3D99091980429969FAF299776
:1074E00080E00E941E2A0E94B2861D8A1E8A1F8A80
:1074F000188E198E1A8E1B8E1C8E83EF9FE4A3ECC0
:10750000B7E48D8F9E8FAF8FB8A383EF9FE4A3EC7A
:10751000B7EC89A39AA3ABA3BCA3A12FB0E0BBABEC
:10752000AAABEDB7FEB724E0129FE019F1091124D0
:107530000FB6F894FEBF0FBEEDBF8DB79EB7019694
:1075400024969FAF8EAF24972DA148ADBE01635FF7
:107550007F4FCE0109960E946FC60E943ECE6115F4
:1075600071058105910511F00E948AE319AA1CAAF0
:107570001DAA1EAA1FAAAEA1A150BB0B6396BFAF46
:10758000AEAF6397812F90E0B0E0A0E067968CAF3C
:107590009DAFAEAFBFAF6797B9A9AB2FB0E0BCA7A7
:1075A000ABA7EAA9FBA9AE17BF070CF07BC21196E7
:1075B000B8A7AFA3FF93EF93BF93AF938FE596E088
:1075C0009F938F9389E696E09F938F931F920E94DB
:1075D000ECA12DB73EB7275F3F4F0FB6F8943EBFE3
:1075E0000FBE2DBF3EA1332309F48CC10E943BE3A3
:1075F0002AE030E040E050E00E9445EE0E94FBE7C8
:1076000020E030E040EA50E40E94B2F00FEF1FEFBC
:10761000181614F001E010E00E943BE328E631E088
:1076200040E050E00E9445EE0E94FBE72B013C0148
:107630000E943BE327E130E040E050E00E9445EE4D
:107640006B5F7F4F8F4F9F4F0E94FBE769AF7AAF11
:107650008BAF9CAF8DA18430B9F449AD5AAD6BAD01
:107660007CAD81E596E04CD9B301A20189E496E0B6
:1076700047D983E496E022D90130110511F483E45F
:10768000FCD88FE396E01AD9B801110F880B990B3B
:107690000E94FBE721966CAF7DAF8EAF9FAF219725
:1076A00020E030E040E153E40E945AE82D966CAFB0
:1076B0007DAF8EAF9FAF2D971FA6EFA56396AEADA2
:1076C000BFAD6397EA171B060CF01CC12296FFADF5
:1076D0002297F11134C00E943BE324E130E040E006
:1076E00050E00E9445EE675E7F4F8F4F9F4F0E9494
:1076F000FBE721962CAD3DAD4EAD5FAD21970E94CD
:107700005AE89B01AC01C301B2010E9413EF2B01A7
:107710003C0120E030E044EB53E40E94F5E718160A
:10772000ACF420E030E044EB53E4C301B2010E942A
:1077300012EFEDCF1EA2BCCE22E02EA3B9CE2D9625
:107740002CAD3DAD4EAD5FAD2D97DDCF20E030E0EF
:10775000A901C301B2010E94B2F087FF0BC020E073
:1077600030E044EB53E4C301B2010E9413EF2B015C
:107770003C01ECCF0091321310913313D8011496D1
:107780002D913D914D915C9117976D857E858F85EB
:1077900098890E9412EF61966CAF7DAF8EAF9FAF5C
:1077A000619726E33AEF4EE85CE3C301B2010E9421
:1077B0005AE86B017C010E948AEF28966CAF7DAF7E
:1077C0008EAF9FAF2897F80120813181428153818C
:1077D00069857A858B859C850E9412EF4B015C013F
:1077E00029AD3AAD4BAD5CAD28966CAD7DAD8EAD9F
:1077F0009FAD28970E945AE89B01AC01C501B401D6
:107800000E9413EF4B015C0189829A82AB82BC8299
:10781000C701B6010E94E7F029AD3AAD4BAD5CADB2
:107820000E945AE861962CAD3DAD4EAD5FAD6197BB
:107830000E9413EF6B017C01CD82DE82EF82F8861D
:1078400020E030E040EE50ECC501B4010E94F5E7C5
:1078500087FF3AC080E090E0A0EEB0EC89839A8385
:10786000AB83BC8320E030E040E050ECC701B601C0
:107870000E94F5E787FF37C080E090E0A0E0B0EC21
:107880008D839E83AF83B887FDA1F43071F4498165
:107890005A816B817C8183E396E032D84D815E8191
:1078A0006F81788582E29FE26AD8198A1A8A1B8AD8
:1078B0001C8ABE016F5E7F4FCE0101960E94DEC71B
:1078C0002FA52F5F2FA7F9CE20E030E041E653E44B
:1078D000C501B4010E94B2F0181624F680E090E0D1
:1078E000A1E6B3E4BBCF20E030E041E653E4C701BA
:1078F000B6010E94B2F018163CF680E090E0A1E6D6
:10790000B3E4BECF20E048ADBE01635F7F4FCE0140
:1079100009960E946FC64B015C01EBA5FCA5EE0F1A
:10792000FF1FEE0FFF1F24968EAD9FAD2497E80F2B
:10793000F91F80829182A282B382A50194016D8D8C
:107940007E8D8F8D98A10E94B2F0181624F48D8E32
:107950009E8EAF8EB8A2A501940169A17AA18BA1D8
:107960009CA10E94F5E787FF04C089A29AA2ABA25E
:10797000BCA2A50194016CA97DA98EA99FA90E9412
:1079800013EF6CAB7DAB8EAB9FAB8FA198A5092E8F
:10799000000CAA0BBB0B8FA398A7A9A7BAA7BC0181
:1079A000CD010E94FBE76BA77CA78DA79EA79B013B
:1079B000AC016CA97DA98EA99FA90E948DEF2B0116
:1079C0003C014D8A5E8A6F8A788E2496AEADBFAD3B
:1079D0002497B8ABAFA710E0C12CD12C7601EFA54E
:1079E000F8A96191719181919191F8ABEFA7A301F1
:1079F00092010E9412EF9B01AC010E945AE89B0188
:107A0000AC01C701B6010E9413EF6B017C011F5F3F
:107A1000F9A9F11720F72BA53CA54DA55EA50E945D
:107A20008DEF0E94F1F0698F7A8F8B8F9C8F2DA143
:107A30002230A0F16FA178A589A59AA50E94DCB09B
:107A40008EE296E00E945E3467966CAD7DAD8EADA1
:107A50009FAD67970E94DCB088E296E00E945E349A
:107A600043E0C501B4010E9426B380E20E943D3488
:107A700081E03DA133300CF480E0E12C8E010F5DFC
:107A80001F4F9E01235E3F4FAE01475E5F4FBE0119
:107A90006B5E7F4F04DC8AE00E943D3489A98F5FD2
:107AA00089AB7ACD0E94CC278DE196E00E945E34AE
:107AB00081E09DA119160CF080E0EE24E3948E0184
:107AC0000F5D1F4F9E01235E3F4FAE01475E5F4F2C
:107AD000BE016B5E7F4FE3DB698D7A8D8B8D9C8D54
:107AE0000052110926E042E00E94D2E29F938F9358
:107AF0008CE096E09F938F9386E196E09F938F931F
:107B00001F920E94ECA10E94998629968FAD299719
:107B10000E941E2A0E94CD8746CC8F929F92AF92E0
:107B2000BF92EF92FF920F931F93CF93DF9383EC5B
:107B300094E00E945E34C0E0D7E0D15021F080E2B2
:107B40000E943D34FACF8C2F0E94DB1DCF5FC730DF
:107B500099F78AE00E943D340DE914E0C0E080E22C
:107B60000E943D348C2F0E94DB1D7801D7E080E21B
:107B70000E943D34F70180809180A280B38020E094
:107B800030E0A901C501B4010E94B2F087FD03C035
:107B90008BE20E943D3443E0C501B4010E9426B34C
:107BA000D150FCE1EF0EF11CD111E1CF8AE00E942F
:107BB0003D34CF5F0C5F1F4FC73089F68AE00E94CB
:107BC0003D34DF91CF911F910F91FF90EF90BF90C7
:107BD000AF909F908F900895811107C08EE99EE02D
:107BE0000E945E348AE00C943D3482EA9EE0F8CF35
:107BF0008CEB94E00C945E3486EB94E00C945E3451
:107C0000CF9384E50E94121AC0E08823F1F00E940D
:107C1000011EC82F1816CCF4EFDF8DE40E943D340E
:107C200080911E0490911F040E94F92B81E999E034
:107C30000E945E346C2FCC0F770B880B990B0E943F
:107C4000DCB08AE00E943D34CFEF8C2FCF910895B5
:107C5000CF93C82F67E978E00E945CC4C11101C0CE
:107C6000CBDF4091961250919712609198127091CB
:107C700099128EE898E00E94803420E030E543ECD1
:107C800050E460919A1270919B1280919C12909195
:107C90009D120E945AE8AB01BC018BE898E00E945B
:107CA00080342CEA35EC47E25EE360919E127091DD
:107CB0009F128091A0129091A1120E945AE8AB01EC
:107CC000BC0188E898E00E9480348AE00E943D343C
:107CD000CF910895B0E0A0E0E0E7FEE30C94E5EE7C
:107CE00061E083E50E942B1EC1E0C82764E879E0CB
:107CF0008C2F0E945CC4C11101C07EDF8CE799E02B
:107D00000E945E348FED9FE00E945E348AE00E9404
:107D10003D346AE679E08C2F0E945CC4C11101C039
:107D20006BDF8DE499E00E945E348C2F0E947CC44E
:107D30008C2F57DA8C2F7CDA8C2F33DA8C2FFDD9ED
:107D400066ED78E08C2F0E9473C4D09198048DEC7E
:107D500098E00E945E346D2F70E090E080E00E9419
:107D6000DCB04091990450919A0460919B04709109
:107D70009C048FE19FE20E94803480EC98E00E9496
:107D80005E348091980428DF20E030E0A901609102
:107D9000690570916A0580916B0590916C050E9450
:107DA000F5E7882399F18DE9E82E84E0F82E10E0BC
:107DB000670100E0C11101C01FDF83E499E00E9468
:107DC0005E34802F0E94DB1D80E499E00E945E34C7
:107DD000812F0E94DB1D8FE19FE20E945E34F6013D
:107DE000608171818281938145E00E9426B38AE09F
:107DF0000E943D340F5FFCE1CF0ED11C0730D1F65D
:107E00001F5F84E0E80EF11C173091F667EF78E011
:107E10008C2F0E945CC401E715E0D0E0C11101C0C5
:107E2000EBDE8EEE98E00E945E348D2F0E94DB1D0B
:107E3000F80160817181072E000C880B990B0E945C
:107E4000FBE7AB01BC018BEE98E00E948034F801A7
:107E5000E280F38088EE98E00E945E34C7010E94C1
:107E6000F92B8AE00E943D340C5F1F4FD13071F531
:107E70008C2FEEDE8C2F0E94913469E279E08C2FFA
:107E80000E9473C4C0915B0180E299E00E945E345D
:107E90006C2F70E090E080E00E94DCB040915701D0
:107EA000509158016091590170915A018DE199E00A
:107EB0000E94803482E199E00E945E3480915B01EF
:107EC0008BDECDB7DEB7E8E00C9401EFD1E0A6CFB2
:107ED000CF93DF93EB010E945E34BE01DD0F880B70
:107EE000990B0E94DCB0DF91CF9108950E945C71E4
:107EF0000E94328C80912B07813099F079DE8FE3DC
:107F000094E00E945E3460E085E394E00E9409A260
:107F10006EE571E080E090E00E94D42B81E08093D8
:107F20002B070895CF92DF92EF92FF921F93CF938A
:107F3000DF9300D000D0CDB7DEB78EEEC82E82E042
:107F4000D82EE12CF12CC982DA82EB82FC82BE01B0
:107F50006F5F7F4F8AE50E94053381110EC010E0EC
:107F6000812F0F900F900F900F90DF91CF911F9165
:107F7000FF90EF90DF90CF9008950E946733C98201
:107F8000DA82EB82FC82BE016F5F7F4F8AE50E943E
:107F90000533182F882319F32BDE89E195E00E9421
:107FA0005E34A4DFDDCFCF92DF92EF92FF921F937A
:107FB000CF93DF9300D000D0CDB7DEB78EEEC82EC2
:107FC00082E0D82EE12CF12CC982DA82EB82FC828D
:107FD000BE016F5F7F4F8AE00E94053381110EC0A2
:107FE00010E0812F0F900F900F900F90DF91CF91A5
:107FF0001F91FF90EF90DF90CF9008950E9467331C
:108000000E9422330E9439330E942233C982DA82CD
:10801000EB82FC82BE016F5F7F4F8AE00E940533D6
:10802000182F8823E9F2E4DD8CED94E00E945E34A1
:108030005DDFD7CFEC018B01F42E0E945C7120979D
:1080400009F47CC0D9DDCE010E945E348AE00E9432
:108050003D340115110511F406E71EE20E94BC1E15
:108060001F930F93DF93CF9385E094E09F938F93BB
:1080700081E08F930E94ECA10E94A38EC0915013C7
:10808000C695C6958BE493E10E945321DC2FDD0F4A
:108090001D2F1C0F8DB79EB707960FB6F8949EBF85
:1080A0000FBE8DBF83E00E941A2010928613C093EA
:1080B000871380E290E10E94602510928613D0938E
:1080C00087136FEF7FEF86EF93E00E940B241092EF
:1080D0008613109387136FEF7FEF89EE93E00E9472
:1080E0000B248FE493E10E944FD18111DBCF80DD1F
:1080F00085E194E00E945E3489EE93E0019739F0C7
:1081000000C00000EEE5F9E03197F0F7F7CFF89402
:1081100089EE93E0019739F000C00000E6EEF3E04D
:108120003197F0F7F7CF0E945C71FF2021F00E9499
:10813000A873A895FECF0E946373FBCF01151105AC
:1081400011F406E71EE2CCE0D4E088CF8091940DD4
:108150009091950D2FEF3FEF981751F0E92FF0E038
:10816000EC56F24F228130E09F5F9F779093950D00
:10817000C90108951F920F920FB60F9211240F900C
:108180000FBE0F901F9018951F920F920FB60F926F
:1081900011240BB60F922F938F939F93EF93FF931E
:1081A0009091C6002091950DE091940D81E08E0F85
:1081B0008F77281729F0F0E0EC56F24F9283E82FE2
:1081C000E093940DFF91EF919F918F912F910F90DC
:1081D0000BBE0F900FBE0F901F9018958EBD0DB463
:1081E00007FEFDCF08958FEF8EBD0DB407FEFDCFC6
:1081F0008EB50895909164009B7F90936400982FB2
:10820000906A96959CBD80FD03C091E0863009F48C
:1082100090E09DBD0895A8E0B0E0E1E1F1E40C94A8
:10822000DBEEB82E80917D0E843008F0F6C131E689
:10823000D32E80917D0E843008F021C18091940D61
:108240009091950D891B8F7709F419C17FDF97FFF6
:108250000AC0CEDC81E393E00E945E348091940DED
:108260008093950DE6CF8A3019F08D3009F0FEC06D
:1082700010927C0E80911A0E90911B0EFC01EA5E0A
:10828000F14F1682892B19F40E94E571D2CF10921A
:108290001B0E10921A0E0CE11EE0F8018191803243
:1082A00009F446C08E3409F09DC06CE273E0C80149
:1082B0000E9474E77C01892B41F06EE470E0C801F4
:1082C00004960E94A7F1009709F4C8014AE050E023
:1082D00070E060E001960E94E9E42B013C0180918E
:1082E000160E9091170EA091180EB091190E0196CE
:1082F000A11DB11D481659066A067B0629F060E0EB
:1083000089EF92E0EF2851F16AE270E0C8010E9423
:10831000D6F19C01009729F1982F901BF12C9923FD
:1083200049F09150F801E90FF11D8081F826F7CF4F
:108330008F01B3CF4AE050E070E060E0C9010196E0
:108340000E94E9E42F2D30E050E040E0621773070F
:108350008407950751F060E08AED92E00E94C6C361
:1083600068CF60E080EB92E0F9CF4092160E509219
:10837000170E6092180E7092190E80912B078130A3
:10838000E1F467E470E0C8010E94A7F10097A9F04A
:108390004AE050E070E060E001960E94E9E462305B
:1083A00071058105910548F48FE092E00E945E34EA
:1083B00060E085E092E00E9409A2F80180818D349E
:1083C00081F58381823309F445C0883301F180331C
:1083D00041F58181843329F58281813311F50E9431
:1083E000A9871FC08091A11480FFC7CF6FE17EE2F3
:1083F000C8010E9474E7009731F0FC01838180532B
:108400008A3008F0BACF60E086E892E0A7CF828198
:10841000803339F48181813321F410926B01109201
:108420007D0480911C0E8B3309F403CF80917D0E67
:10843000843008F0FECE80917F0E8D9DC001112406
:108440006CE17EE08058914F0E94B2F180E00E9482
:1084500086C3EFCE8281813321F78181813309F791
:1084600041E070E060E086E19BE0E4DD2AE13EE08F
:108470004CE15EE06CE77EE00E941D19DACE80914F
:10848000A11483FDCAC082FFC8C087FDC6C01A827E
:10849000198281E6F82E94E0E92E29E6D22E809109
:1084A0007D0E843008F0B9C00E9455198111B5C005
:1084B00041E050E0BE016D5F7F4F84EA92E10E948F
:1084C000CAD70B8110E0019711F00FEF1FEF8091D9
:1084D000AC129091AD12A091AE12B091AF128093F8
:1084E0009D1490939E14A0939F14B093A0140E9487
:1084F00055190F3F100741F4811106C079DB89E45B
:1085000093E00E945E34CBCF40917F0E242F30E069
:108510000A3061F00D3051F0882309F470C0898170
:108520009A81009719F001969A8389831092A90382
:1085300089819A81F29EF001F39EF00D1124E35897
:10854000F14FDF01A80FB91F13961C92892BA9F5D3
:108550000E94E5710E945519882309F4A0CF84EA8E
:1085600092E10E94146D809198148823F1F181505A
:10857000809398148D9DC001112462E08758994F13
:108580000E94D1D9E091981424E0E29FF0011124D7
:10859000EB58F94F408151816281738140939D1462
:1085A00050939E1460939F147093A01484EA92E1F8
:1085B0000E94CFD60E94AAD272CF1A8219828381DA
:1085C0008D3479F48481823361F48581853349F473
:1085D000868180538A3028F08091A1148B7F80930C
:1085E000A11481E00E9486C3B5CF0E949CD28091E5
:1085F000A11488608093A114E0922B0750CF4F9D67
:10860000A00111244058514F9E012F5F3F4F69EA4E
:1086100073E0802F0E941D1942CF0E943ECE6B0155
:108620007C01BB2041F0C0922104D0922204E09250
:108630002304F09224048091F8039091F903A0910F
:10864000FA03B091FB030097A105B10529F1409110
:108650002104509122046091230470912404840F1A
:10866000951FA61FB71FA7019601281B390B4A0BA0
:108670005B0BDA01C901B7FD0FC0BADA60916A0776
:1086800070916B0788E593E00E948ED240E070E025
:1086900060E090E080E0E9CE8091190190911A01AC
:1086A000A0911B01B0911C01892B8A2B8B2B79F097
:1086B0009091371380913813981709F4C4C0C09271
:1086C0002104D0922204E0922304F09224048091A9
:1086D000AE039091AF03A091B003B091B1034601F6
:1086E0005701881A990AAA0ABB0AD501C401B7FD25
:1086F000C0C19091371380913813209108019817C9
:1087000009F4D5C0E09138133BE5E39FF001112453
:10871000E151F84F8081281799F0809308010E9459
:108720003ECEB09008010B2D10E084E00E9407B30C
:108730000115110509F0BEC060E084E00E9459CD2A
:1087400080918705882309F487C100912F0110913A
:108750003001C8010297209193123091941228178A
:1087600039070CF479C1809038138C82812C912CBC
:108770005401809137132C81821709F4FDC0822F98
:1087800090E03BE5389FF001399FF00D1124E7564A
:10879000F84F458956896789708D452B462B472BA5
:1087A00081F4418D528D638D748D452B462B472B63
:1087B00041F4458D568D678D70A1452B462B472B77
:1087C000E9F14BE5489F9001499F300D1124C90103
:1087D0008756984F1C01FC016181728183819481CD
:1087E0000E94F1F06D837E838F839887F10161A1F0
:1087F00072A183A194A10E94F9E72B013C01F10130
:1088000065A176A187A190A50E94F9E79B01AC0123
:10881000C301B2010E948DEF2D813E814F815885A9
:108820000E945AE82B013C01AC019B01C501B40137
:108830000E94B2F087FF02C0530142018C818F5F1A
:108840008F708C8396CFBB2019F01092B2033FCF6C
:108850000E943ECE00912104109122042091230415
:10886000309124048090190190901A01A0901B016E
:10887000B0901C01080D191D2A1D3B1D601B710BBA
:10888000820B930B97FDE1CF8091B20381111FCF33
:1088900081E08093B20380E00E94787381E00E94BF
:1088A000787382E00E9478730E94637310CF809186
:1088B000880731CF0F3F110511F461E03ECFEAE5A3
:1088C000FEE2E491E150EA3008F051C0F0E0E559F1
:1088D000FB4B0C94C0EE75447A447F448944B74402
:1088E000B74493449B44A344AD4484B5806884BD9D
:1088F000B7BC26CF84B5806284BDB8BC21CF80913F
:108900008000806880938000109389000093880025
:1089100017CF8091800080628093800010938B003D
:1089200000938A000DCF8091B00080688093B000E2
:10893000B092B30005CF8091B00080628093B00008
:10894000B092B400FDCE809190008068809390003A
:108950001093990000939800F3CE8091900080626C
:108960008093900010939B0000939A00E9CE00380A
:1089700011050CF0A2CFE0CEB801110F880B990BB6
:108980000E94FBE72B013C012091290130912A0133
:1089900040912B0150912C01C501B4010E945AE86D
:1089A000A30192010E9413EF4B015C0100912D0184
:1089B00010912E01AC019B01C301B2010E94B2F0E3
:1089C00018168CF0B801012E000C880B990B0E9430
:1089D000FBE72B013C01A50194010E94F5E7181665
:1089E00014F4240135018090AA039090AB03A09069
:1089F000AC03B090AD03A3019201C501B4010E9484
:108A0000B2F01816D4F420E037ED43EA5CE3C3017A
:108A1000B2010E945AE82B013C0128E431EE4AE7FA
:108A20005FE3C501B4010E945AE89B01AC01C30198
:108A3000B2010E9413EF2B013C014092AA03509215
:108A4000AB036092AC037092AD03C301B2010E940C
:108A5000F5EFCB010E947FCEF4E6CF0ED11CE11CD6
:108A6000F11CC092AE03D092AF03E092B003F0923B
:108A7000B1030E94E57180912B07882309F40AC194
:108A800080915B018823B1F18091B703811132C0DD
:108A90000E94FE2B882371F1F894029B10C08091F4
:108AA000570190915801A0915901B0915A018093BA
:108AB0007F0590938005A0938105B0938205609116
:108AC0007F05709180058091810590918205789451
:108AD00020E030E0A9010E94F5E787FF0BC081E0AC
:108AE0008093B70385E993E09093E9068093E806C5
:108AF0000E94307410910901113061F18091A1142C
:108B000080648093A11481E08093090164EF71E097
:108B100080E090E00E94D42B0E94BFD48091A114E9
:108B200084FFD0C0123028F460E089E993E00E940D
:108B300009A283E080936C010E943ECE6C597F4F66
:108B40008F4F9F4F609372047093730480937404EB
:108B5000909375040E943ECE6B017C011091180128
:108B60001123F1F08091FD038823D1F04091B303EC
:108B70005091B4036091B5037091B603460157015B
:108B8000841A950AA60AB70AB501A40177FD1AC08E
:108B9000833009F492C00CF081C081300CF086C0A3
:108BA000212F30E0A8EEB3E00E9471EEC60ED71E72
:108BB000E81EF91EC092B303D092B403E092B5034D
:108BC000F092B6030E9486218091F703882379F101
:108BD0000E943ECE6B017C018091F3039091F403DF
:108BE000A091F503B091F603A7019601281B390B5C
:108BF0004A0B5B0BDA01C901B7FD19C02091F703DD
:108C000030E0A8EEB3E00E9471EEC60ED71EE81E5B
:108C1000F91EC092F303D092F403E092F503F092B0
:108C2000F60380E00E94D1708AE00E943D3480917A
:108C3000F203882379F10E943ECE6B017C01809182
:108C4000EE039091EF03A091F003B091F103460180
:108C50005701881A990AAA0ABB0AD501C401B7FDAF
:108C600019C02091F20330E0A8EEB3E00E9471EE4B
:108C7000C60ED71EE81EF91EC092EE03D092EF0377
:108C8000E092F003F092F1030E9493B389E393E141
:108C90000E94AA722896E2E10C94F7EE843009F063
:108CA0007FCF0E94FC3D88EA93E004C00E94FC3D17
:108CB00087ED93E00E945E3473CF0E94FC3D80EC10
:108CC00093E0F8CF112309F445CF33CFA2E1B0E010
:108CD000ECE6F6E40C94DCEE9091490D93FD7FC038
:108CE000082F0E94003E182F87FD79C089E40E945A
:108CF000121A882309F48BC00E94011E282F30E02D
:108D00001216130614F421E030E0220F331F220F55
:108D1000331FF901EF58FA4F80819181198A0E941F
:108D20007FCE80919312909194128635910574F0C4
:108D3000002381F00E94EA8B0DC082E50E94121A86
:108D4000882309F46CC00E943C1EE9CF0E94328C3B
:108D50000E94F7C46091931270919412072E000C38
:108D6000880B990B0E94FBE720918F123091901293
:108D700040919112509192120E94B2F0181644F054
:108D8000298980E090E1222329F049894A8B48C053
:108D90008BE090E19F938F9386E190E19F938F9377
:108DA0001F920E94ECA10F900F900F900F900F90C8
:108DB00031E03A8B35C060E070E0CB014FC0C701B5
:108DC000B6010E94F5E787FF0EC080916B018823F2
:108DD00021F010926B010E94F7C4309287056296D1
:108DE000E1E10C94F8EE4601570100E098C08FE3F2
:108DF0000E943D34CFC020E030E040E450E40E94C7
:108E0000B2F018160CF004C12601370101C183E548
:108E10000E94121A898B811196CF01118ECF1A8A66
:108E200083E50E94121A882331F00E943C1E909321
:108E3000300180932F0182E40E94121A882331F0BE
:108E40000E943C1E90932E0180932D0186E40E9487
:108E50009B19882309F4AFCF0E944B1E6093290110
:108E600070932A0180932B0190932C013324339427
:108E700020E030E0A9010E94F5E7811101C0312C0A
:108E800030928705002309F4AACF5A89552309F4A3
:108E9000A6CF1092870581E080936B011D821E8210
:108EA0001F82188619861A861B861C8680E09CE322
:108EB000ACE1B6E48D879E87AF87B88B812C912C6F
:108EC00090E8A92E9FEBB92E00E0412C512C3201E5
:108ED0006091931270919412072E000C880B990BDD
:108EE0000E94FBE76B017C01A50194010E94F5E75C
:108EF0008823A9F020918F12309190124091911205
:108F000050919212998991115ACFC701B6010E94CE
:108F1000F5E7082F001F0027001F460157010E9498
:108F20003ECE6B017C01DC01CB0129853A854B8566
:108F30005C85821B930BA40BB50BB7FD2EC0D7012C
:108F4000C60188519C4FAF4FBF4F89879A87AB8727
:108F5000BC87812F0E94D1708CE190E10E945E3429
:108F6000411451046104710409F441CFC301B201F9
:108F7000605F784D8F4F9F4F6C197D098E099F0957
:108F800028EE33E040E050E00E9423EECA01B90130
:108F90000E9468268AE00E943D3480E03CD90E940D
:108FA0003ECE609321047093220480932304909317
:108FB000240420918F12309190124091911250917F
:108FC000921229833A834B835C83C501B4010E94CA
:108FD00012EF9F77411451046104710409F00BCF23
:108FE00020E030E040E85FE30E94F5E787FF10C033
:108FF0003A89412C512C3201332331F085E0482E3F
:109000008DE0582E612C712C4C0C5D1C6E1C7F1C4D
:109010000023C1F18D819E81AF81B885892B8A2B78
:109020008B2B61F0D701C6012D813E814F81588580
:10903000821B930BA40BB50BB7FD24C029813A8189
:109040004B815C816D857E858F8598890E9412EFAA
:1090500020E030E040EC5FE30E94F5E787FDB5CE0D
:10906000D701C601805A9541AF4FBF4F8D839E8374
:10907000AF83B88729813A814B815C812D873E87F8
:109080004F87588B80916B01882309F49ECE411441
:1090900051046104710461F030E1C31A37E2D30A6C
:1090A000E108F108C418D508E608F708F7FE8DCEE8
:1090B0001A8A0ECFA5E4B0E0E0E6F8E40C94DBEE0B
:1090C00026968FAF26972091FD0328AB81E08093F1
:1090D000FD03809120048D3409F48CC3843511F490
:1090E0000C94795C873491F480911E0490911F0454
:1090F0008D31910509F4FBC108F082C084309105DF
:1091000009F4A2C130F4029708F4FBC00E9446C4DF
:1091100073C18531910509F46FC14C97B9F787E0A8
:109120000E942C83811111C0809118049091190420
:10913000A0911A04B0911B04EEE0B695A7959795FF
:109140008795EA95D1F780FD57C10E94307410923F
:109150003C01609198048CE40E942B1E982E80E0C4
:109160000E941E2A0E943ECE609321047093220426
:1091700080932304909324040E94B28681E080931C
:10918000E4060E94BE88C0901804D0901904E090B4
:109190001A04F0901B0479E1F694E794D794C794ED
:1091A0007A95D1F7C0FE0DC081E00E942C83182F64
:1091B00082E00E942C8311110C94265E11E0811133
:1091C00001C010E08091180490911904A0911A0434
:1091D000B0911B0467E1B695A795979587956A9519
:1091E000D1F780FF02C00C949C5C112311F40C9405
:1091F0009F5CA12E10E04C2D4170B42E0C94B85CF5
:109200008A35910509F4E7C250F58E31910509F4CC
:1092100071C18A9709F07ACF80912B07833008F4C7
:10922000EBC089E40E94121A082FF12C882319F050
:109230000E943C1EF82E8AE40E94121AE82E88230F
:1092400009F4C7C10E943C1E182F0111C5C1173077
:1092500008F4C8C182EE99E00E945E34CDC08B351F
:10926000910509F4BBC28C35910509F04FCF47E950
:10927000242E41E0342E57E7E52E51E0F52EC12C87
:10928000D12C10E0F10181911F010E94121A082FC8
:10929000882349F10E944B1E2B013C01D7012D91DF
:1092A0003D914D915C910E9412EF4B015C012DEBC1
:1092B00037E346E855EB0E94F5E787FD0AC02DEB42
:1092C00037E346E855E3C501B4010E94B2F0181631
:1092D00054F4133011F0C02E0D2DF701408251824D
:1092E00062827382D02E1F5FF4E0EF0EF11C143007
:1092F00049F6CC2009F476C20E947F870E94CD8770
:109300007BC080912B07833008F476C0F8E8CF2E1D
:10931000F4E0DF2EA7E7EA2EA1E0FA2E10E088E5C0
:10932000810F0E94121A882309F472C00E944B1EFA
:109330004B015C01812F0E947419882359F0D701D9
:109340002D913D914D915C91C501B4010E9413EFA7
:109350004B015C01F60180829182A282B3821F5F81
:10936000F4E0CF0ED11C24E0E20EF11C1330B9F66C
:1093700085E40E94121A882309F455C00E944B1EEE
:109380006B017C0183E00E947419882371F02091A5
:109390008301309184014091850150918601C7017C
:1093A000B6010E9413EF6B017C01C0929404D0922D
:1093B0009504E0929604F092970440E050E0BA01E0
:1093C00086E40E94731E20E030E0A9010E94B2F002
:1093D000181684F40E944B1E29E838E848E85CE33C
:1093E0000E945AE8609335017093360180933701EB
:1093F000909338010E948A8326969FAD26979111FB
:1094000002C00E9433C4A8A9A093FD030C9420536A
:10941000F70180819181A281B381F60180839183DC
:10942000A283B3839CCF8091830190918401A0910A
:109430008501B09186018093940490939504A09344
:109440009604B0939704B9CF80E50E94121AC12CFC
:10945000D12C7601882321F00E94E11D6B017C0153
:1094600083E50E94121A882361F00E944B1E20E0BF
:1094700030E04AE754E40E945AE80E94FAEF6B0198
:109480007C010E94307480912010811105C060E041
:1094900084EA99E00E9409A20E943ECEC60ED71E21
:1094A000E81EF91E0E943ECE6C197D098E099F09A7
:1094B00097FFA2CF80E00E940B41F4CF60E070E004
:1094C00080EA90E40C94C15CA3019201C701B6014B
:1094D0000C940D5D60E08FEB99E00E9409A20E9460
:1094E000FC3D8DEA99E00E945E340C94FE5D0E9482
:1094F000825E82CF0091321310913313F8012081E4
:10950000318142815381609177017091780180911E
:10951000790190917A010E9413EFAB01BC0188E5BB
:109520000E94731E69837A838B839C83D80114966F
:109530002D913D914D915C91179760917B017091B8
:109540007C0180917D0190917E010E9413EFAB011F
:10955000BC0189E50E94731E6D837E838F8398878B
:10956000BE016B5F7F4FCE0101960E9439C58823F3
:1095700009F442CF80E00E941E2A0E94B28661E078
:1095800085E40E942B1E21E0482FBE016B5F7F4FB8
:10959000CE0101960E946FC66B017C0149815A8100
:1095A0006B817C818AED99E00E9480344D815E81DF
:1095B0006F81788585ED99E00E948034B701A6011E
:1095C00080ED99E00E94BF340E9499860E94CD8769
:1095D00013CF10E0002331F0B6E0BF1508F43ACE07
:1095E000E11035CE80E1E7E7F1E0A8E8B4E00190D2
:1095F0000D928A95E1F7002319F16F2DFF0C770B7F
:10960000880B990B0E94FBE72091690530916A0550
:1096100040916B0550916C050E945AE820916105BC
:109620003091620540916305509164050E9413EFEB
:10963000609388047093890480938A0490938B04C8
:10964000EE2019F1612F110F770B880B990B0E94F7
:10965000FBE720916D0530916E0540916F055091AB
:1096600070050E945AE82091650530916605409189
:109670006705509168050E9413EF60938C04709306
:109680008D0480938E0490938F0460E080E50E94A7
:109690002B1E8823C1F10023D1F0E0913213F09109
:1096A000331320813181428153816091880470910C
:1096B000890480918A0490918B040E9412EF609338
:1096C00088047093890480938A0490938B04EE201D
:1096D000D1F0E0913213F09133132481358146812A
:1096E000578160918C0470918D0480918E049091CB
:1096F0008F040E9412EF60938C0470938D0480930A
:109700008E0490938F0440E050E0BA0186E40E94FA
:10971000731E6B017C0120E030E0A9010E94B2F0D1
:1097200087FF03C0C12CD12C760129E838E848E82E
:109730005CE3C701B6010E945AE86B017C0180908E
:10974000350190903601A0903701B090380120E0AB
:1097500030E0A9010E94F5E7882341F0C09235016D
:10976000D0923601E0923701F09238010091390130
:1097700010913A0184E690E090933A018093390188
:10978000C0907101D0907201E0907301F09074016B
:1097900080E090E0A0E8BFE38093710190937201B4
:1097A000A0937301B09374010E948A838092350163
:1097B00090923601A0923701B092380110933A018D
:1097C00000933901C0927101D0927201E09273014D
:1097D000F092740111CE1092FC030ECE8FE08093B4
:1097E000FC030ACEDD2009F489CD83E891E00E94D4
:1097F000838184CD80911E0490911F04823791054E
:1098000011F40C943C5508F06FC18B34910509F4A8
:10981000EFC608F0E9C08831910509F40FC508F0DA
:10982000BAC08231910509F4F6C708F06EC08230E3
:10983000910508F479C4419709F068CC0E948A190F
:10984000882309F4CDC40E94E91900917A05102FEC
:109850001095182309F4D0CDF12CE12CD12CA12E98
:10986000B12CC5010E2C02C0959587950A94E2F79C
:1098700080FF08C08E2D0E94AF73F701EC5DFD4F95
:109880008081D82A8FEFE81AF80A93E0E916F104EC
:1098900041F713FF05C00E947173AD2DA360DA2E4E
:1098A000102B10951D2109F4A7CD88E20E943D34AC
:1098B000F12CE12CC12ED12CC6010E2C02C09595A5
:1098C00087950A94E2F780FF09C0F701E956FE4F39
:1098D00080810E943D3480E20E943D34BFEFEB1A4C
:1098E000FB0AE3E0EE16F10439F713FF09C085E443
:1098F0000E943D3480E30E943D3480E20E943D346A
:109900008EE09AE00E945E3477CD8531910509F4AE
:109910007FC458F5449709F0F9CB8091A11484FFD6
:1099200070C48FE39AE00E945E348091A11484FF9A
:1099300017C08AED92E10E94436E8BE1EAEDF2E1FD
:10994000DE01119601900D928A95E1F770E060E0DA
:10995000CE0101960E9403DBCE0101960E94137096
:1099600080E39AE00E945E3447CD8631910509F488
:1099700052C4479709F0CACB80911C0490911D04F2
:10998000FC012191222309F455C42032D1F7DF01D3
:1099900011971C92F6CF8D31910509F4DDC4A0F426
:1099A0008A31910509F463C408F453C48B319105DD
:1099B00009F478C44C9709F0A9CB80911C049091CC
:1099C0001D040E9485D918CD8F31910509F46AC50F
:1099D00008F4C8C48032910509F41FC5C09709F086
:1099E00095CB0E94BC3908CD8836910509F40CC688
:1099F00008F046C08235910509F4FDC6F0F48D34B7
:109A0000910509F4FDC508F4F7C58135910509F004
:109A10007DCB0E944174109288070E945C710E9465
:109A2000328C68EE73E080E090E00E94D42B60E01E
:109A30008BE29BE00E9409A2DFCC8435910509F4FA
:109A4000EAC608F4E0C68535910509F47EC78C3571
:109A5000910509F05BCB0E94003E87FDCDCC809143
:109A6000180484FD97C780911A0487FD93C78091DD
:109A70001B04837009F08EC781E00E947CC4BCCCBB
:109A80008D36910509F4C5C598F48A36910509F417
:109A9000DCC508F4C3C58B36910509F40FC68C36B6
:109AA000910509F033CB10927D0410926B01A4CC88
:109AB0008F36910509F420C608F40BC6803791054E
:109AC00009F456C68137910509F020CB83E50E9441
:109AD000121A882309F458C60E94011E8D3308F01B
:109AE0004EC68093180188CC8D3221E0920711F484
:109AF0000C94A75808F0F4C18B39910509F454C6A9
:109B000008F0F4C08737910511F40C948D5508F0D6
:109B1000BAC08537910509F4B7C708F0C5C78337C0
:109B2000910509F0F3CA87EF9CE00E945E3460E083
:109B300087EE9CE00E946B3460E082ED9CE00E9426
:109B40006B3461E08BEC9CE00E946B3460E080EC55
:109B50009CE00E946B3461E081EB9CE00E946B34DE
:109B600061E081EA9CE00E946B3460E088E99CE05F
:109B70000E946B3461E08EE89CE00E946B3461E0EF
:109B800084E89CE00E946B3461E08DE79CE00E94D9
:109B90006B3461E085E79CE00E946B3461E087E60E
:109BA0009CE00E946B3460E089E59CE00E946B348D
:109BB00060E08AE49CE00E946B3460E08CE39CE00F
:109BC0000E946B3460E086E29CE00E946B3460E0AF
:109BD00085E19CE00E946B3460E080E09CE00E94A4
:109BE0006B3460E081EF9BE00E946B3461E08AEEB1
:109BF0009BE00E946B3460E083EE9BE00E946B343C
:109C000061E08AED9BE00E946B3460E085EC9BE0B4
:109C10000E946B3460E087EB9BE00E946B3460E055
:109C20008AEA9BE00E946B3461E087E99BE00E9436
:109C30006B3460E08AE89BE00E946B3460E085E86A
:109C40009BE00E946B3461E088E79BE00E946B34EC
:109C500060E084E69BE00E946B3460E081E59BE07D
:109C60000E946B3460E080E892E10E947119682FD5
:109C7000617088E49BE00E946B3460E08AE39BE0C3
:109C80000E946B34B9CB8937910509F453C708F4A6
:109C900048C78139910509F455C78A39910509F0FA
:109CA00035CA83E50E94121A882309F4A5CB0E94C5
:109CB000011E182F8C3308F08CE38093F2030E946E
:109CC0003ECE6B017C01212F30E0A8EEB3E00E9474
:109CD00071EEC60ED71EE81EF91EC092EE03D0929A
:109CE000EF03E092F003F092F10386CB833D910500
:109CF00011F40C940657C0F58B3C910509F4A1C7EB
:109D0000B0F4893C910509F001CA8091180484FDE2
:109D10006EC780911A04887809F069C780911B0486
:109D2000837009F064C781E00E94183965CB8C3CD0
:109D3000910509F4BAC78D3C910509F0E7C98091F6
:109D4000180481FF02C00C94AA568091190481FF67
:109D500002C00C94AA5680911A048C7009F0FAC7BC
:109D600081E00E949D3848CB8D3D910511F40C9403
:109D70009A5708F045C08C3D910509F0C7C982E4A7
:109D80000E949B19882341F08091390190913A01FA
:109D900090931E0180931D0182E50E949B198823E8
:109DA00041F080911D0190911E0190933A018093A2
:109DB000390183E50E94121A882331F00E943C1E6B
:109DC00090933A018093390180911804909119047D
:109DD000A0911A04B0911B04892B8A2B8B2B09F0BC
:109DE0000BCB6091390170913A0184E29EE00E94B0
:109DF000683F85E20E943D348AE00E943D34FCCAFF
:109E0000883141E0940711F40C94E7578232914075
:109E100009F07CC98AE50E94121A882311F40C9477
:109E200082580E944B1E20E030E040E050EC0E943F
:109E3000B2F0C12CD12CE12C50ECF52E87FD13C0D3
:109E40000E944B1E20E030E040E050E40E94F5E725
:109E5000C12CD12CE12C40E4F42E181624F00E94E1
:109E60004B1E6B017C012091660D3091670D409176
:109E7000680D5091690DC701B6010E945AE80E9411
:109E8000F5EFCB010E941AC561E080E50E942B1E10
:109E9000882311F40C948858A701960160912E1321
:109EA00070912F1380913013909131130E9413EF12
:109EB00060932E1370932F1380933013909331136C
:109EC0000E94FC3D40912E1350912F13609130134E
:109ED0007091311380E69EE00E94BF340C94885844
:109EE000843FA1E09A0711F40C94705B08F0ADC0B8
:109EF0008239E1E09E0711F40C943F59F0F48F325F
:109F000021E0920711F40C94375910F40C94F15895
:109F1000803941E0940711F40C943B598139914008
:109F200009F0F4C883E50E949B19811165CA81E09C
:109F30000E94CD890E94CD875FCA8C39A1E09A0723
:109F400011F40C94455938F48A39914009F0DEC86F
:109F50000E94A98751CA843AF1E09F0711F40C943A
:109F6000AD59853A914009F0D1C86FEF7FEF89E490
:109F70000E943F1E8C016FEF7FEF8AE40E943F1E1C
:109F80007C018AE50E94121AD12C811108C081E55A
:109F90000E94121AD82E882311F40C941E5EC02E33
:109FA00081E0800F883010F00C94685BBE2C81E05B
:109FB0008E0D883010F00C94685B102F0E944B1EA1
:109FC0002B013C01A02E07FDA12C17FF02C046E08B
:109FD000C42E8E2DE7FCE12C87FF02C036E0B32EA5
:109FE00027E0322ECA1408F407CAFE2C3A9C40011E
:109FF0001124BF1410F40C94655B0F2D10E020E0C9
:10A0000030E0A901DD2069F0F401E00FF11FEE0F4F
:10A01000FF1FEE0FFF1FE356FB4F2081318142816E
:10A020005381080D191D000F111F000F111F03563A
:10A030001B4FC301B2010E9413EFD8016D937D93B2
:10A040008D939C931397F394D4CF8C3032E0930785
:10A0500011F40C94805B20F5863F51E0950711F4D4
:10A060000C94785B10F40C94745B873FB1E09B0711
:10A0700011F40C947C5B883F914009F047C881E063
:10A08000809379050E94388F10927905882309F40E
:10A09000B3C90E94FC3D8DE49FE00E945E34ACC9D0
:10A0A000803AF3E09F0709F4EFC1A0F483359340B1
:10A0B00009F02CC880911A0487FF02C00C94985BA9
:10A0C00080911B04837011F00C94985B81E00E94D6
:10A0D000913492C9873E43E0940711F40C94695C73
:10A0E000893E934009F012C80E9430748091A114F7
:10A0F000877F8B7F8093A1140E949D8B6D337105A8
:10A100008105910520F084EC9FE00E942A5E80EC9E
:10A110009FE00E942A5E8CEA9FE00E945E3488EAFB
:10A120009FE00E942A5E68C980E50E94121AC12C35
:10A13000D12C7601882321F00E94E11D6B017C0166
:10A1400083E50E94121A882361F00E944B1E20E0D2
:10A1500030E04AE754E40E945AE80E94FAEF6B01AB
:10A160007C010E94307480911C0490911D04009722
:10A1700011F10E9481C21091FD0383E08093FD03E1
:10A1800081E080937D04C114D104E104F10431F035
:10A190000E943ECEC60ED71EE81EF91E80917D0499
:10A1A0008823B9F0C114D104E104F10451F480E032
:10A1B0000E940B41F3CF60E08BEF99E00E9409A26F
:10A1C000DACF0E943ECE6C197D098E099F0997FD5A
:10A1D000EECF10927D041093FD030E94F7C40CC9CA
:10A1E00060E08DE19AE00E9409A280E00E94AF73D6
:10A1F00081E00E94AF7382E00E94AF730E9471738E
:10A20000FBC80E94FC3D86E29AE00E945E34F4C8DE
:10A210000E94BFD4F1C88091A11482FF02C087FFC1
:10A22000EBC80E949CD28091A1148F7E80648093A1
:10A23000A114E2C860E00E94D1D9DEC80E94112CAE
:10A24000882321F00E94AAD20E94EA8B0E94F7C4C0
:10A25000D3C88091A11482FF05C087FD03C08B7F06
:10A260008093A1140E941D8C0E94F7C4C5C88091E0
:10A27000A11484FFC1C883E50E94121A882309F43F
:10A28000BBC80E94F11DAB01BC0140939D145093CB
:10A290009E1460939F147093A01484EA92E10E942C
:10A2A000CFD6AAC88091180490911904A0911A04DD
:10A2B000B0911B0432E0B695A795979587953A958E
:10A2C000D1F780FF1CC08DE79AE00E945E34809138
:10A2D000A712882379F0BE016F5F7F4F84EA92E175
:10A2E0000E94376DCE0101960E9444348AE00E949C
:10A2F0003D3482C880E59AE00E945E34F7CF8091B9
:10A30000A11482FF24C0C0909D14D0909E14E090B0
:10A310009F14F090A0148BE69AE00E945E34C7016F
:10A32000B6010E947FB08FE20E943D346091991483
:10A3300070919A1480919B1490919C140E947FB00C
:10A340008DE00E943D348AE00E943D3455C88AE584
:10A350009AE00E945E3450C88091A1148E7F809351
:10A36000A1144AC88091A11484FF46C80E94B9D69E
:10A370008091A11484FF40C840911C0450911D0499
:10A38000BE01645E7F4F80E00E94A6C28C010097F0
:10A3900009F432C86C8D7D8D19821C8222E0AC01DB
:10A3A000CE0101960E941870811115C0F12CCE01CA
:10A3B00001960E941370FF2019F1B80187EA9AE014
:10A3C0000E948ED210929D1410929E1410929F148F
:10A3D0001092A01411C8CE0101960E9454D7882370
:10A3E00029F361E0CE0101960E941D6D0097F1F204
:10A3F00025EEDC012C931C820E94E6D2F82ED7CFEA
:10A400008FE89AE00E945E34C8010E9444348CE8D0
:10A410009AE00E945E340C94FC498091A11482FF62
:10A4200003C087FF0E9430748091A11484FD02C094
:10A430000C94FC4960E080E50E942B1E182F682FC9
:10A4400080911C0490911D040E94D1D983E50E9443
:10A45000121A882381F00E94F11DAB01BC014093C8
:10A460009D1450939E1460939F147093A01484EADB
:10A4700092E10E94CFD60E94AAD211110C94FC49FD
:10A480000E94EA8B0C94FC4920911C0430911D041D
:10A490009091A11492609093A114C9010E9485D952
:10A4A0000C94FC490E949D8B6B017C0120E831E5F6
:10A4B00041E050E00E9423EEC9016DE671E00E9488
:10A4C00099EE4B015C01C701B60120E13EE040E09E
:10A4D00050E00E9423EECA01B90128E130E040E0DB
:10A4E00050E00E9423EE2B013C011B01C701B60185
:10A4F0002CE330E040E050E00E9423EE6B017C0151
:10A50000CA01B9012CE330E040E050E00E9423EEA4
:10A510008E010F5F1F4F8114910419F1DF92CF92CA
:10A520007F936F935F924F92BF92AF929F928F9261
:10A530008DED9AE09F938F931F930F930E948EE768
:10A540000FB6F894DEBF0FBECDBFC8010E9481C216
:10A550000E94FC3DB80181EF9AE00E948ED20C94DB
:10A56000FC49A114B10489F0DF92CF927F936F93DD
:10A570005F924F92BF92AF928DEC9AE09F938F9330
:10A580001F930F930E948EE7DBCF4114510479F0A3
:10A59000DF92CF927F936F935F924F9281EC9AE01C
:10A5A0009F938F931F930F930E948EE7C9CF6115DE
:10A5B000710569F0DF92CF927F936F9389EB9AE0F8
:10A5C0009F938F931F930F930E948EE7B9CFDF92D3
:10A5D000CF9285EB9AE09F938F931F930F930E94E6
:10A5E0008EE70F900F900F900F900F900F90ADCFC0
:10A5F0000E94EA8B0C94FC490E941D8C0C94FC492F
:10A600000E94328C0C94FC4980E00E9466460C94B7
:10A61000FC4981E00E9466460C94FC490E94003E81
:10A62000182F87FD0AC08EEF9AE00E945E34812FBA
:10A630000E94D1708AE00E943D3498A99093FD0356
:10A64000CB5BDF4FE2E10C94F7EE60E080E50E9427
:10A65000121E81110C94FC498091180490911904E8
:10A66000A0911A04B0911B0460918807062F10E096
:10A6700080FD02C00FEF10E089E40E94121A8823C7
:10A6800011F40C94125E0E94011E90E01816190637
:10A6900014F481E090E0880F991F880F991FFC0146
:10A6A000EF58FA4F028113810F3F110519F010F096
:10A6B0000FEF10E0009388070C94FC4960E080E500
:10A6C0000E94121E81110C94FC49109288070C9470
:10A6D000FC498EE40E94121A882311F40C94FC4960
:10A6E0000E94F11D6093160E7093170E8093180E42
:10A6F0009093190E0C94FC4983E50E94121A88234A
:10A7000021F00E94011E8093490D0E94FC3D8FE0C4
:10A710009BE00E945E348091490D882331F110E066
:10A7200000E020E08091490D90E0002E02C0959558
:10A7300087950A94E2F780FF12C0FF24F394F20E8B
:10A74000222319F08CE20E943D34F801EE0FFF1F26
:10A75000EB5FF44F859194910E945E342F2D0F5F33
:10A760001F4F05301105F1F6C1CD81E09BE0C4CD4E
:10A7700041E070E060E086E19BE00E941A408CE3DB
:10A78000809318010C94FC490E94FC3D1091180123
:10A7900084E29BE00E945E34812F0E94DB1D8AE0F0
:10A7A0000E943D340C94FC4983E50E94121A8823D0
:10A7B00011F40C94FC490E94011E182F8C3308F0F0
:10A7C0008CE38093F7030E943ECE6B017C01212F26
:10A7D00030E0A8EEB3E00E9471EEC60ED71EE81E70
:10A7E000F91EC092F303D092F403E092F503F092C5
:10A7F000F6030C94FC498091FC038F7D806180936B
:10A80000FC030C94FC498091FC038F7E8062809352
:10A81000FC030C94FC4983E50E94121A8823F1F092
:10A820000E943ECE609321047093220480932304FF
:10A83000909324040E944B1E20E030E04AE754E449
:10A840000E945AE80E94FAEF6093190170931A016E
:10A8500080931B0190931C010C94FC490E948A195F
:10A86000882309F46EC00E9430740E94E919082FF1
:10A8700010917A05182311F40C94FC49F12CE12C69
:10A88000C82ED12CAA24A394B12CC6010E2C02C030
:10A89000959587950A94E2F780FF12C08E2D0E944D
:10A8A0007873882369F0F701EC5DFD4F8081950195
:10A8B0000E2C01C0220F0A94EAF7822B80951823F0
:10A8C000AFEFEA1AFA0AB3E0EB16F104F1F603FF70
:10A8D00004C00E9463738111147FF12CE12CC12EFE
:10A8E000D12CC6010E2C02C0959587950A94E2F7EB
:10A8F00080FF0FC0F701E956FE4F80810E943D3472
:10A90000F701EC5DFD4F908180917A0589230E94CB
:10A91000B2DBEFEFEE1AFE0AF3E0EF16F10409F7EF
:10A9200013FD02C00C94FC4985E40E943D3480E391
:10A930000E943D3480917A0583700E94B2DB0C94B2
:10A94000FC490E9441740C94FC4983E50E949B19C8
:10A95000882311F40C94FC490E943ECE609321049C
:10A960007093220480932304909324040E944B1E2E
:10A9700020E030E04AE754E40E945AE80E94FAEFEF
:10A980006093F8037093F9038093FA039093FB03A9
:10A990000C94FC49B7E9CB2EB1E0DB2E1AE4E12E92
:10A9A0001DE0F12E10E0D6018D916D010E94121A6A
:10A9B000882349F0133089F00E944B1EF701648B05
:10A9C000758B868B978B1F5FF4E0EF0EF11C1430B4
:10A9D00051F70E9408740C94FC490E944B1E4B01D5
:10A9E0005C0120E030E040EA51E40E94F5E787FF97
:10A9F0003AC0A501940160916A0D70916B0D809130
:10AA00006C0D90916D0D0E948DEF2B013C01AC01FE
:10AA10009B0160917A0D70917B0D80917C0D9091DE
:10AA20007D0D0E945AE860937A0D70937B0D8093A0
:10AA30007C0D90937D0D60917C0770917D078091D6
:10AA40007E0790917F070E94F9E7A30192010E947F
:10AA50005AE80E94FAEF60937C0770937D07809319
:10AA60007E0790937F0780926A0D90926B0DA09263
:10AA70006C0DB0926D0DA7CF0E9493B389E393E163
:10AA80000E94AA720C94FC4980911C0490911D04B0
:10AA9000009709F4DBCBDC012C91222309F4D6CBFF
:10AAA0000E9481C20C94FC4900911C0410911D0469
:10AAB00094E0F12C40E09150F9F0F8018081282FCA
:10AAC0002B7F213499F421812133B1F4813411F1A8
:10AAD000853409F441E098012E5F3F4F89012F5FD3
:10AAE0003F4FF80180818032C9F3E5CF803521F4F2
:10AAF000818180538A3078F341110E94FC3DFF2010
:10AB000021F08EEB9DE00E945E34C8010E944F341C
:10AB10000C94FC49FF24F394DECF0E9478880C94B7
:10AB2000FC4981E08093E4068093E3060E94BE889E
:10AB30000C94FC491092E4061092E3060E94BE8831
:10AB40000C94FC4970E060E083E50E943F1E823077
:10AB500040F00E94F83D81EC9DE00E945E340C9430
:10AB6000FC498C01112788E40E94121A8823A9F05D
:10AB70000E943C1E8A3A910574F10E943C1E863F59
:10AB8000910564F50E943C1EF801EE0FFF1FEE0FC9
:10AB9000FF1FEF58FA4F9183808386E40E94121AB8
:10ABA000882311F40C94FC490E943C1E97FD19C0A7
:10ABB0000E943C1E8F3F910509F0B4F40E943C1E98
:10ABC000000F111F000F111FF801EF58FA4F938368
:10ABD00082830C94FC498AEA90E0D6CF85EF90E01E
:10ABE000D3CF90E080E0ECCF8FEF90E0E9CF0E94F0
:10ABF000003E87FF02C00C94FC4907E911E05AE4CB
:10AC0000E52E5DE0F52E6BE9C62E61E0D62ED8016B
:10AC10008D918D010E94121A882359F00E944B1EBB
:10AC20000E94FAEFF70160837183828393830E940D
:10AC3000C473F4E0EF0EF11CC016D10641F70C947A
:10AC4000FC498091180484FD0DC080911A04887815
:10AC500049F480911B04837029F481E00E94F1384B
:10AC60000C94FC490E94003E87FF02C00C94FC49F2
:10AC700047E9E42E41E0F42E10E000E0D7018D9189
:10AC80007D010E94121A882349F00E944B1EF80190
:10AC9000E65BF24F64A375A386A397A30C5F1F4FD7
:10ACA0000031110559F70C94FC498091190487FD76
:10ACB00009C080911A048E7029F481E00E94D13875
:10ACC0000C94FC4983E50E94121A882391F00E949B
:10ACD0004B1E60937E0D70937F0D8093800D90933B
:10ACE000810D6093860D7093870D8093880D9093EE
:10ACF000890D80E50E94121A882351F00E944B1E94
:10AD000060937E0D70937F0D8093800D9093810DE5
:10AD100082E50E94121A882351F00E944B1E609314
:10AD2000820D7093830D8093840D9093850D84E53F
:10AD30000E94121A882311F40C94FC490E944B1EA5
:10AD40006093860D7093870D8093880D9093890D85
:10AD50000C94FC4982E40E94121A882351F00E944C
:10AD6000E11D60935A0D70935B0D80935C0D909381
:10AD70005D0D83E50E94121A882351F00E944B1E3C
:10AD800060938A0D70938B0D80938C0D90938D0D35
:10AD900084E50E94121A882351F00E944B1E609392
:10ADA0008E0D70938F0D8093900D9093910D8AE48A
:10ADB0000E94121A882311F40C94FC490E944B1E25
:10ADC0006B017C012AE037ED43E25CE30E94B2F0C4
:10ADD00087FD14C02AE939E949E95EE3C701B601F4
:10ADE0000E94F5E7181654F0C0926C07D0926D07D8
:10ADF000E0926E07F0926F070C94FC490E94F83DB8
:10AE000083EE9DE00E945E340C94FC4983E50E9431
:10AE10009B19882331F00E941C1E80933B010C94E7
:10AE2000FC4910913B01105D8BE19EE00E945E3475
:10AE3000812F0E943D3487E19EE00E945E34809124
:10AE40003B010E94EC3D20913D0130913E0140913B
:10AE50003F01509140012CA33DA34EA35FA340901E
:10AE600041015090420160904301709044018090F4
:10AE7000450190904601A0904701B0904801C090D4
:10AE80004901D0904A01E0904B01F0904C01809133
:10AE90004D0190914E01A0914F01B091500188A7B2
:10AEA00099A7AAA7BBA720915101309152014091C7
:10AEB0005301509154012CA73DA74EA75FA78FE0E7
:10AEC0009EE00E945E344CA15DA16EA17FA182E054
:10AED0009EE00E948034B301A20182E29FE20E94C0
:10AEE0008034B501A4018FE19FE20E9480348DE09F
:10AEF0009EE00E945E3485E09EE00E945E34B701D1
:10AF0000A60182E09EE00E94803448A559A56AA56A
:10AF10007BA582E29FE20E9480344CA55DA56EA5D0
:10AF20007FA58FE19FE20E9480348AE00E943D3439
:10AF30000C94FC490E94003E082F87FF02C00C942D
:10AF4000FC4983E50E94121A002E000C110B7801B7
:10AF5000EE0CFF1C882309F10E943C1EF701EB5AFE
:10AF6000FE4F91838083000F111F000F111F0F5898
:10AF70001E4FBC01990F880B990B0E94FBE72AE03A
:10AF800037ED43E25CE30E945AE8D8016D937D936C
:10AF90008D939C9313970C94FC490E94FC3D85E48F
:10AFA0000E943D3480E3800F0E943D34F701EB5A4C
:10AFB000FE4F6081718188E29EE00E94683F85E2D9
:10AFC0000E943D348AE00E943D340C94FC4980E5A7
:10AFD0000E94121A882311F40C94FC490E943C1E12
:10AFE0008C01892B09F081C083E50E94121A882305
:10AFF00089F00E943C1E97FD07C0BC0183E293E1EB
:10B000000E9440320C94FC4983E293E10E941F327B
:10B010000C94FC490E94FC3D70E060E089E49EE0F5
:10B020000E94683F80912513F8E5CF2EF2E0DF2ED5
:10B03000C81AD10887FDD394CC0CDD1CCC0CDD1CC8
:10B040000D2C000CEE08FF0880912413B8E88B2E1D
:10B05000912C881A910887FD9394880C991C880C70
:10B06000991C092C000CAA08BB088091231390E0BE
:10B070008F3FC9F1FC01EE0FFF1FE80FF91FE250EF
:10B08000FD4E8181928173E0880F991F7A95E1F7D7
:10B09000B0E0A0E0E4E0B595A79597958795EA958F
:10B0A000D1F702969C012F5F3F4F032E000C440BFB
:10B0B000550B281939094A095B09A4EBB0E00E9435
:10B0C00061EEA7019601281939094A095B090E9416
:10B0D00045EEB90186E49EE00E94683F8AE00E9446
:10B0E0003D340C94FC4980E0DDCF0E94F83DB8016E
:10B0F0008FE39EE00E94683F80E39EE00E945E3402
:10B100000C94FC4983E50E94121A81110C94114F92
:10B1100080911A0487FD14C080911B04837081F410
:10B120000E94FC3D40912E1350912F1360913013DB
:10B130007091311381E59EE00E94BF340C94FC496C
:10B1400082E50E949B198111EBCF0C94FC49809100
:10B15000180483FD09C080911904817829F481E0E5
:10B160000E94283E0C94FC4980E50E94121A882314
:10B1700051F00E944B1E6093961270939712809329
:10B1800098129093991289E40E94121A882381F0F0
:10B190000E944B1E2CEA35EC47E25EE30E945AE81F
:10B1A00060939A1270939B1280939C1290939D12BD
:10B1B00084E40E94121A882311F40C94FC490E9422
:10B1C0004B1E20E030E543EC50E40E945AE86093C7
:10B1D0009E1270939F128093A0129093A1120C94D0
:10B1E000FC4983E50E949B19182F882369F00E946F
:10B1F0003C1E9C01909376018093750191E0232B76
:10B2000009F090E090937D1280E50E949B198823BD
:10B2100061F02091750130917601232B11F00E948D
:10B220001C1E80937D120C94FC4911110C94FC4956
:10B230000E94FC3D8BE89EE00E945E3480917D126E
:10B24000882391F083E79EE00E945E34609175014F
:10B25000709176018AE79EE00E94683F86E79EE053
:10B260000E945E340C94FC498FE69EE0EDCF0E9474
:10B27000C2340C94FC490E9430740C94FC490E9426
:10B28000CC270E94CD870C94FC498091180483FD43
:10B290002AC080911A04867031F50E94FC3D85EB2E
:10B2A0009EE00E945E3480915B018823C9F082EAAF
:10B2B0009EE00E945E344091570150915801609188
:10B2C000590170915A0188EA9EE00E94803485EA13
:10B2D0009EE00E945E348AE00E943D340C94FC495A
:10B2E0008EE99EE0E6CFC0901804D0901904E0905B
:10B2F0001A04F0901B0431E1F694E794D794C794B4
:10B300003A95D1F7B1E0CB22DD24EE24FF2483E58A
:10B310000E949B19182FC114D104E104F10411F407
:10B32000882341F00E941E1A112321F00E941C1E46
:10B3300080935B0184E40E949B19882311F40C9490
:10B34000FC490E944B1E60935701709358018093F3
:10B35000590190935A010C94FC4983E50E949B1972
:10B36000182F882309F426C10E941C1E8CA320914B
:10B370007701309178014091790150917A012DAB9C
:10B380003EAB4FAB58AF80917B0190917C01A09177
:10B390007D01B0917E0189AF9AAFABAFBCAF209178
:10B3A0007F0130918001409181015091820121966D
:10B3B0002CAF3DAF4EAF5FAF2197112331F03CA1D1
:10B3C000311103C080E00E941E2A809118049091E0
:10B3D0001904A0911A04B0911B0425E1B695A79514
:10B3E000979587952A95D1F79C01AD012170332758
:10B3F0004427552729AB3AAB4BAB5CAB20E030E0A0
:10B40000A9016091690570916A0580916B05909121
:10B410006C050E94F5E7882309F4D0C083E40E94FC
:10B420009B19882309F49AC00E944B1E25966CAF85
:10B430007DAF8EAF9FAF25974DE954E059A748A740
:10B440008A0157E05CA7412C512CE8EC6E2EE2EC0F
:10B450007E2E812C912CF8ECAF2EF2E4BF2E312CF5
:10B46000212CF101EE0FFF1FEE0FFF1FE00FF11F68
:10B47000C080D180E280F380A7019601C501B401AC
:10B480000E94F5E7181614F446015701A70196012A
:10B49000C301B2010E94B2F087FF02C0260137014A
:10B4A0008FEF281A380A97E029163104D1F6ACA597
:10B4B000A150ACA7045E1F4FA111D1CFA3019201EF
:10B4C000C501B4010E9413EF20E030E040E05FE3EB
:10B4D0000E945AE825962CAD3DAD4EAD5FAD259747
:10B4E0000E9413EF4B015C012DEB37E346E855EB6F
:10B4F0000E94F5E787FD0AC02DEB37E346E855E3E8
:10B50000C501B4010E94B2F0181644F580E00E9413
:10B510001E2A67E0F62E08A519A557E0E52EF801CA
:10B5200061917191819191918F016F01F4E0CF1A36
:10B53000D108A50194010E9412EFD6016D937D936D
:10B540008D939C931397EA94E110E9CFFA94E8A5C0
:10B55000F9A57C96F9A7E8A7F110DDCF89A99AA9EA
:10B56000ABA9BCA9892B8A2B8B2B81F020E030E082
:10B57000A9016091690570916A0580916B059091B0
:10B580006C050E94F5E781110E948D3D8AE50E94BD
:10B590009B19882359F00E944B1E69837A838B8301
:10B5A0009C8360E0CE0101960E94AA2A8CA10E9491
:10B5B0001E2A15C0E0919804ECA3D9CEFCA1F1118C
:10B5C00008C029A93AA94BA95CA9232B242B252B18
:10B5D000E9F20E94FC3D85E09FE00E945E349CA160
:10B5E000992351F080919804811106C00E94F83D82
:10B5F00086EE9EE00E945E340E94FC3D88ED9EE057
:10B600000E945E34809198040E94EC3D0E94FC3DB3
:10B610008BEC9EE00E945E34C0909904D0909A0416
:10B62000E0909B04F0909C0420E030E0A901C70169
:10B63000B6010E94B2F018160CF042C042E0C701F9
:10B64000B6010E9426B38DE00E943D348AE00E943C
:10B650003D342091770130917801409179015091EA
:10B660007A016DA97EA98FA998AD0E94F5E7811195
:10B670000C947E4920917B0130917C0140917D01A9
:10B6800050917E0169AD7AAD8BAD9CAD0E94F5E71E
:10B6900081110C947E4920917F013091800140916D
:10B6A00081015091820121966CAD7DAD8EAD9FAD33
:10B6B00021970E94F5E781110C947E490C94FC4976
:10B6C00086EC9EE00E945E34C4CFA3940C94F24FAB
:10B6D0000E94F83D84E39FE00E945E340C94FC4994
:10B6E0000E9442A20C94FC490E9432920C94FC49A4
:10B6F0000E94C8880C94FC490E946A3E0C94FC4944
:10B700008091A11482FF0CC087FD0AC00E94112CF9
:10B710009091A11480FB97F99093A1140C94FC498B
:10B7200084FD02C00C94FC490E94B9D60C94FC49DB
:10B73000409026135090271360902813709029137F
:10B7400020912A1330912B1340912C1350912D13DB
:10B750002CA33DA34EA35FA3C0902E13D0902F1314
:10B76000E0903013F090311388E50E94121A182FE0
:10B77000882309F482C00E944B1E4B015C0120E02B
:10B7800030E041E653EC0E94B2F087FD0BC020E0B0
:10B7900030E041E653E4C501B4010E94F5E7181614
:10B7A0000CF06DC061EE70E085E99FE00E94683F9B
:10B7B00061EE70E080E99FE00E94683F8DE89FE0C5
:10B7C0000E945E3410E089E50E94121A882341F13C
:10B7D0000E944B1E4B015C0120E030E041E653EC3F
:10B7E0000E94B2F087FD0BC020E030E041E653E458
:10B7F000C501B4010E94F5E718160CF043C061EED4
:10B8000070E08AE79FE00E94683F61EE70E085E7A4
:10B810009FE00E94683F82E79FE00E945E3410E054
:10B820008AE50E94121A882391F10E944B1E6B0137
:10B830007C0120E030E040EA51EC0E94B2F087FD4C
:10B840000AC020E030E040EA51E4C701B6010E949E
:10B85000F5E71816E4F46CEE7FEF80E69FE00E94B7
:10B86000683F64E170E08BE59FE00E94683F88E5F7
:10B870009FE00E945E340C94FC4911E0A4CF2401A7
:10B880003501A1CF8CA29DA2AEA2BFA2C9CF112328
:10B8900011F40C94FC4940922613509227136092A5
:10B8A0002813709229138CA19DA1AEA1BFA18093F2
:10B8B0002A1390932B13A0932C13B0932D13C092A3
:10B8C0002E13D0922F13E0923013F09231130C9478
:10B8D000FC4983E080932B071092751060E083E5AC
:10B8E0000E942B1E81110C94FC490E949DC30C9454
:10B8F000FC4900911E0410911F040E943ECE6093EB
:10B900002104709322048093230490932404002341
:10B9100011F40C94FC490E94FC3D84E50E943D34E6
:10B92000802F0E94DB1D80E20E943D3488EC9FE066
:10B930000E945E340C94FC4911110FC011E08091FB
:10B94000180490911904A0911A04B0911B043B2F84
:10B950003170A32E31130C94FB488C2D8170A12ED5
:10B9600081130C94FB4811E0AA24A394BB24B39444
:10B9700082E50E94121A882311F40C945E4A0E94F8
:10B980004B1E68A379A38AA39BA320E030E0A90102
:10B990000E94F5E7882379F0111105C0A11003C0BA
:10B9A000BB2009F42BC1CE0180960E94A9C40E943D
:10B9B00067330E942233112309F48AC0AA2009F4B4
:10B9C00084C0109277011092780110927901109240
:10B9D0007A0110927B0110927C0110927D011092ED
:10B9E0007E010E947F878DE49EE10E94C6276B0145
:10B9F0007C0181E59EE10E94C6272B013C01AC0140
:10BA00009B01C701B6010E94B2F0181614F00C9405
:10BA1000644AA7019601C301B2010E948DEF9B0108
:10BA2000AC010E945AE820E030E040E85FE30E9469
:10BA300013EF0E94F1F021E030E048E452E40E946C
:10BA40005AE869837A838B839C8380917F019091EC
:10BA50008001A0918101B09182018CA39DA3AEA32E
:10BA6000BFA320E030E040EC5FE3C301B2010E94DD
:10BA70005AE82B013C0177FA709477F8709420E033
:10BA800030E040EC5FE3C701B6010E945AE89058ED
:10BA9000DE0111966D01ECA0FDA00EA11FA1A30176
:10BAA00092010E94D1860E94678B109277011092BA
:10BAB00078011092790110927A0110927B01109214
:10BAC0007C0110927D0110927E0180E00E94358AF7
:10BAD000AA2019F081E00E94358ABB2009F48EC0AB
:10BAE00083E00E944783811189C00E947F878091F3
:10BAF0007F0190918001A0918101B091820180939A
:10BB0000940490939504A0939604B09397040091A5
:10BB1000321310913313F801C080D180E280F3809A
:10BB2000A701960160E070E080EE92E40E9412EFBF
:10BB3000609388047093890480938A0490938B04A3
:10BB4000D80114964D905D906D907C901797A3014D
:10BB5000920160E070E080EE92E40E9412EF609348
:10BB60008C0470938D0480938E0490938F042DE049
:10BB700030E044EE52E4C301B2010E94B2F0181664
:10BB800014F40C946A4A2EE030E042EE52ECC30109
:10BB9000B2010E94F5E787FF02C00C946A4A2DE0CB
:10BBA00030E04EEE52E4C701B6010E94F5E71816E8
:10BBB00014F40C946A4A2EE030E042EE52ECC701D5
:10BBC000B6010E94B2F087FF02C00C946A4A1C8E34
:10BBD0001D8E1E8E1F8E88E0E8E8F4E0DE011196CF
:10BBE00001900D928A95E1F7BE01645E7F4FCE0110
:10BBF00001960E94DEC782E00E94358A0E947F87FC
:10BC00008091E3068093E406992019F081E00E9478
:10BC10001E2A0E94998683E080936C010E94CD8742
:10BC20000C94FC4983E50E94121A882311F40C94A9
:10BC300054530E94F11D8B010C9454530E94F83D03
:10BC400084E19FE00E945E340C94FC49882309F44F
:10BC500075CE89CEB0E0A0E0E0E3FEE50C94DDEE29
:10BC60007C014DB65EB660906A0770906B078DB62A
:10BC70009EB66AE070E0C7010E9432E76C018C0159
:10BC80000E191F09892B21F4C7010E9444E78C017A
:10BC9000C80101962DB73EB7281B390B0FB6F89493
:10BCA0003EBF0FBE2DBF8DB79EB701965C01A801A8
:10BCB000B7010E9465E7F501E00FF11F1082C50191
:10BCC0000E946A2681E00E945A48C114D10451F0B2
:10BCD00076019FEFE91AF90A0FB6F8949EBE0FBEDF
:10BCE0008DBEC5CF0FB6F8949EBE0FBE8DBEC301EC
:10BCF0000E946A260FB6F8945EBE0FBE4DBEE0E10C
:10BD00000C94F9EEA2E4B0E0E8E8FEE50C94DBEE7A
:10BD10000E943ECE609321047093220480932304FA
:10BD20009093240480919804811145C08091180457
:10BD300090911904A0911A04B0911B043DE0B695AE
:10BD4000A795979587953A95D1F780FF03C086E030
:10BD500096E080DF87E00E944783811133C08091A5
:10BD60009804888B8091180490911904A0911A046A
:10BD7000B0911B04AC01BD0126E1769567955795FE
:10BD800047952A95D1F740FFEDC020E030E0A901AA
:10BD90006091690570916A0580916B0590916C05C1
:10BDA0000E94F5E7811113C00E94F83D84EF95E0F1
:10BDB0000E945E3407C060E08FE40E942B1E88233F
:10BDC00009F4B4CFCE5BDF4FE2E10C94F7EE8AE5E5
:10BDD0000E94121A8823E9F00E944B1E6B017C011D
:10BDE00020E030E040E251ECC701B6010E94F5E7E7
:10BDF00087FD0AC020E030E040E251E4C701B6010F
:10BE00000E94B2F0181674F40E94F83D87EE95E097
:10BE1000CFCFC0907F01D0908001E0908101F09061
:10BE20008201DECF40E050E060EC7FE788E50E94D1
:10BE3000731E2B013C0140E050E060EC7FE789E598
:10BE40000E94731E6BAB7CAB8DAB9EAB6FEF89E436
:10BE50000E94121E6FEF8AE40E94121E8BA09CA00B
:10BE6000ADA0BEA020E030E040E05FE3C501B4013A
:10BE70000E945AE820916105309162054091630566
:10BE8000509164050E9412EFA30192010E9413EFEA
:10BE9000A50194010E948DEF0E94F5EF2B013C015A
:10BEA000162F8FA098A4A9A4BAA420E030E040E007
:10BEB0005FE3C501B4010E945AE820916505309105
:10BEC000660540916705509168050E9412EF2BA905
:10BED0003CA94DA95EA90E9413EFA50194010E94FF
:10BEE0008DEF0E94F5EF062F042C000C550857FC2F
:10BEF00031C027E0421651047CF5062E000C770B6A
:10BF000077FD2CC0673071055CF5173008F05ACF0B
:10BF1000073008F057CF80E00E941E2A37E0130256
:10BF2000F0011124E00FF11D07FDFA95EE0FFF1F40
:10BF3000EE0FFF1FE356FB4FC082D182E282F382F5
:10BF400088890E941E2A8889882309F43BCF0E9491
:10BF5000CD8738CF10E0D1CF16E0CFCF00E0D5CFDE
:10BF600006E0D3CFE9E0B695A79597958795EA9532
:10BF7000D1F780FD0CC070E060E086E50E943F1EB6
:10BF80009A838983059730F082EC95E011CF0E9467
:10BF9000602A18CF60E084E40E942B1E8F8740E067
:10BFA00050E0BA018AE50E94731E6BA77CA78DA79B
:10BFB0009EA740E050E669EF75E483E50E94731E9A
:10BFC00029E838E848E85CE30E945AE860936D018C
:10BFD00070936E0180936F0190937001E090321323
:10BFE000F0903313D7014D905D906D907C9020E0E0
:10BFF00030E040EE50E4C301B2010E9412EF4B0169
:10C000005C0120E030E040E251E40E94B2F087FFA2
:10C0100006C0812C912C70E2A72E71E4B72E20E08F
:10C0200030E041E653E4C301B2010E9413EF6FAB6D
:10C0300078AF89AF9AAF20E030E047E553E40E9443
:10C04000F5E7181644F480E090E0A7E5B3E48FAB81
:10C0500098AFA9AFBAAFD7011496CD90DD90ED900F
:10C06000FC90179720E030E040E050E4C701B601B3
:10C070000E9412EF2B013C0120E030E040E251E44D
:10C080000E94B2F087FF06C0412C512C60E2662E60
:10C0900061E4762E20E030E041E653E4C701B601CA
:10C0A0000E9413EF6BAB7CAB8DAB9EAB20E030E01E
:10C0B00047E553E40E94F5E7181644F480E090E069
:10C0C000A7E5B3E48BAB9CABADABBEAB88E40E9401
:10C0D0009B19882309F4F8C10E944B1E0E94F5EFBA
:10C0E00023966CAF7DAF8EAF9FAF239721966EAD39
:10C0F0007FAD219777FF02C06F5F7F4F7595679582
:10C1000071956195710960597F4F072E000C880B5E
:10C11000990B0E94FBE76B017C01CBAEDCAEEDAE70
:10C12000FEAEA30192010E94B2F087FF04C04BAEA5
:10C130005CAE6DAE7EAEA5019401C701B6010E9452
:10C14000B2F087FF02C075016401CB8ADC8AED8AF8
:10C15000FE8A8BAD9CADADADBEAD8F8B988FA98F98
:10C16000BA8F2196AEADBFAD2197BD01BB0F880B35
:10C17000990B0E94FBE74B015C01A70196010E940D
:10C1800013EF6B017C012FA938AD49AD5AAD0E9468
:10C19000F5E7181624F4CFA8D8ACE9ACFAACCB8EEE
:10C1A000DC8EED8EFE8E2BAD3CAD4DAD5EADC50192
:10C1B000B4010E9413EF6B017C012BA93CA94DA98E
:10C1C0005EA90E94F5E7181624F4CBA8DCA8EDA818
:10C1D000FEA8CF8ED8A2E9A2FAA2BE01695E7F4F67
:10C1E000CE0143960E9439C5882309F496C1BE0149
:10C1F000615E7F4FCE014B960E9439C5E82E8823A1
:10C2000009F48BC12F89388D498D5A8D6F8D78A196
:10C2100089A19AA10E9412EF2BEA3AEA4AE25EE370
:10C220000E945AE84B015C012B893C894D895E894B
:10C230006B8D7C8D8D8D9E8D0E9412EF2BEA3AEADC
:10C240004AE25EE30E945AE86BA37CA38DA39EA3FF
:10C250008FA298A6A9A6BAA689819A81181619064E
:10C2600074F480E995E00E945E348F85882321F084
:10C2700086E895E00E945E348AE00E943D340E9488
:10C2800030740E94B28680E00E941E2A80E090E016
:10C29000A0E2B1E48FA798ABA9ABBAABCE018F9661
:10C2A0000E94A9C42091690530916A0540916B05EF
:10C2B00050916C056BA17CA18DA19EA10E94F5E718
:10C2C000811130C020916D0530916E0540916F0550
:10C2D000509170056FA178A589A59AA50E94F5E7F0
:10C2E000811120C020916105309162054091630564
:10C2F000509164056B897C898D899E890E94F5E740
:10C30000811110C020916505309166054091670547
:10C31000509168056F89788D898D9A8D0E94F5E717
:10C320008823A9F00E94602A88E0FE01B396A9E65E
:10C33000B5E001900D928A95E1F788E0FE017396D1
:10C34000A1E6B5E001900D928A95E1F7188A60E0C8
:10C3500085E40E942B1ECC24C394811102C043E0CB
:10C36000C42E1B861C861D861E861A8ADE2C97E02C
:10C37000792E26E5A22E25E0B22E34E6832E35E076
:10C38000932E8A8987300CF0D4C0DD2009F4C8C010
:10C3900066246394B7E0BBAB90E021E0D226879D92
:10C3A000F02C1124F394998B19896A89FBA91F1722
:10C3B00009F4BCC0062E000C770B880B990B0E9469
:10C3C000FBE72FA138A549A55AA50E945AE82F8955
:10C3D000388D498D5A8D0E9413EF1B012C01612F5E
:10C3E000110F770B880B990B0E94FBE72BA13CA147
:10C3F0004DA15EA10E945AE82B893C894D895E8936
:10C400000E9413EF6B837C838D839E832F823886FB
:10C4100049865A8689819A81892B89F082E795E03D
:10C420000E945E348F2D0E94DB1D61E370E080E787
:10C4300095E00E94683F8DE695E00E945E341F9271
:10C4400021E32F931F92FF92BF92AF929F928F9200
:10C450001F920E94ECA129814C2DBE01695F7F4F84
:10C46000CE0103960E946FC69B01AC012B873C87CF
:10C470004D875E8709898A89672D0603800111240B
:10C48000080F111D87FD1A95000F111F000F111FB6
:10C4900003561B4F6BA57CA58DA59EA50E9413EF8F
:10C4A000D8016D937D938D939C931397188A81E0A7
:10C4B0000E940B41F3948989860D898B0FB6F894FD
:10C4C000DEBF0FBECDBF70CFB301A20186E40E94D4
:10C4D000731E6B017C01B501A4018CE40E94731EE4
:10C4E0006B8B7C8B8D8B9E8BCF8AD88EE98EFA8E50
:10C4F0004BA95CA96DA97EA982E40E94731E6B0101
:10C500007C014FA958AD69AD7AAD82E50E94731EDA
:10C510006B8F7C8F8D8F9E8F5CCE86EA95E048CCAA
:10C5200066246A94EFEFEBAB96E037CF6F5F6A8BD0
:10C5300028CF0E94F7C40E94CC27882359F088890D
:10C540000E941E2A80E090E0A0ECBFE78B879C87CA
:10C55000AD87BE870E948D3D0E94772B8F8581110C
:10C5600022C08FE791E00E94CF274B015C0187E753
:10C5700091E00E944728A50194010E945AE89B017E
:10C58000AC0160917F017091800180918101909157
:10C5900082010E9412EF60937F017093800180936B
:10C5A0008101909382018F858111E888E09298043F
:10C5B0000E94998680919804882309F4C8CC0E942F
:10C5C0007F87C5CCCF93DF93C0917E0E81E6C89F55
:10C5D000E0011124C058D14F8091490D80FF05C062
:10C5E0000E94FC3DCE010E944F34CE010E946A267B
:10C5F00080E00E945A48DF91CF910895A0E1B0E019
:10C60000E4E0F3E60C94E9EE8C01DC01ED91FC91A1
:10C610000280F381E02DBE016F5F7F4F0995882373
:10C6200009F45DC08981807C91F56F81637070E051
:10C63000762F6627770F770F8885B4E08B9FC00130
:10C640001124682B792B8985829586958695837030
:10C65000682B6F5F7F4F90E080E02A852370220F68
:10C660003B8537FB332730F9232B3E813F70230F67
:10C670003327331F2750310904C0660F771F881FE7
:10C68000991F2A95D2F76096E4E00C9405EF803468
:10C6900019F568856695669570E090E080E0CB01BD
:10C6A000772766272A85622B098510E0102F00273F
:10C6B000012E000C220B330B602B712B822B932B42
:10C6C0006F5F7F4F8F4F9F4F4AE0660F771F881F26
:10C6D000991F4A95D1F7D7CF8BE0F801848360E0AA
:10C6E00070E0CB01D0CF0895FC0182810895FC0158
:10C6F00090E1A0E6B6E001900D929A95E1F70895D9
:10C70000EF92FF920F931F93E0927B05F0927C05CE
:10C7100000937D0510937E05B62F172F022FF32E61
:10C72000242F582FB09383051093840550938505CB
:10C730006FEFFF27B01B1F09520B30F45095109577
:10C74000B195160B560B66276093A402A6E0BA9F1C
:10C7500000929802712DEE271A9F700DE11D5A9FCD
:10C76000E00D70939902E0939A02AFE0BA9F0092B5
:10C770009C02712DEE271A9F700DE11D5A9FE00D4E
:10C7800070939D02E0939E02AAE0BA9F0092A002DD
:10C79000712DEE271A9F700DE11D5A9FE00D7093C9
:10C7A000A102E093A2021F910F91FF90EF900895D4
:10C7B000A5E0B0E0EEEDF3E60C94E2EE6F36710525
:10C7C0008105910578F4FB01EE0FFF1FEE0FFF1FAF
:10C7D000EB59F04E65917591859194912596EBE01A
:10C7E0000C94FEEEF62EE72E282FE5E6FEE100275C
:10C7F000BB275F2D8E2D922F992341F4982F852FE3
:10C80000B85F992319F4982F8827B85F903138F4CE
:10C8100082959295582F5F70807F952BBC5F9034E6
:10C8200028F4880F991F880F991FBE5F903818F45D
:10C83000880F991FB395880F991FE90FF01F549126
:10C8400081E09927B85079F1C0F0B0FF02C0550FD0
:10C85000881FB1FF04C0550F881F550F881FB2FFF6
:10C8600006C082955295152F1F70507F812BB3FF04
:10C870001AC0982F852F552716C0B195B0FF02C05A
:10C8800085955795B1FF04C0859557958595579522
:10C89000B2FF05C08295507F5295582B8F70B3FF21
:10C8A00002C0582F8827BB247727AA27B2E0F59E1D
:10C8B000B0187109A00BB00BE59E7019A109B00B5F
:10C8C000259FA019B109F89E7019A109B00BE89E27
:10C8D000A019B109289FB019F99EA019B109E99EC4
:10C8E000B0195B9DA12C99244427662733278B9D83
:10C8F000A00C911C401F601F301F9B9D900C411D80
:10C90000601F301F579FA00C911C401F601F301FDD
:10C91000879F900C411D601F301F979F400D611D28
:10C92000301F5A9F900C411D601F301F8A9F400D81
:10C93000611D301F9A9F600D311D5B9F400D611D71
:10C94000301F8B9F600D311D9B9F300DB1E0AA27DA
:10C950007727BB24F49EB0187109A00BB00BE49E9E
:10C960007019A109B00B249FA019B109F69E701986
:10C97000A109B00BE69EA019B109269FB019F39E3C
:10C98000A019B109E39EB019BF187E09A20B20F0CF
:10C99000B1E04B0F601F301F1124762F642F90E001
:10C9A000832F1CCFFC017081472F50E0062E02C060
:10C9B000559547950A94E2F740FF14C04091F80559
:10C9C00050E0062E02C0559547950A94E2F740FFC5
:10C9D00009C021E030E001C0220F6A95EAF72095F6
:10C9E0002723208308958F929F92AF92BF92CF9278
:10C9F000DF92EF92FF92FC01C080D180E280F38051
:10CA000020E030E048EC52E4C701B6010E945AE849
:10CA10004B015C0120E030E0A901C701B6010E9492
:10CA2000F5E720E030E040EA50E487FF04C020E072
:10CA300030E040EA50ECC501B4010E9413EF2DEC48
:10CA40003CEC4CEC5DE30E945AE80E94F5EF9B0140
:10CA50008BE237FF05C022273327261B370B8DE2D9
:10CA600080938104C90168EE73E00E94ADEECB01B2
:10CA7000EAE0F0E0BF010E94ADEE805D80938204A9
:10CA8000C90164E670E00E94ADEECB01BF010E94D7
:10CA9000ADEE805D80938304C901BF010E94ADEEBD
:10CAA0009C01CB01BF010E94ADEE805D80938404A8
:10CAB0008EE280938504205D2093860481E894E0D3
:10CAC000FF90EF90DF90CF90BF90AF909F908F90AE
:10CAD00008954F925F926F927F928F929F92AF9242
:10CAE000BF92CF92DF92EF92FF92FC01C080D18083
:10CAF000E280F38020E030E04AE754E4C701B60169
:10CB00000E945AE84B015C0120E030E040E251EC29
:10CB1000C701B6010E94F5E7181654F420E030E092
:10CB200048EC52E4C701B6010E94B2F087FD8AC00A
:10CB300020E030E0A901C701B6010E94F5E787FFB8
:10CB400072C060E070E080EA90ECA50194010E9460
:10CB500013EF2DEC3CEC4CEC5DE30E945AE80E9494
:10CB6000F5EF6B017C01F7FC63C020E137E240E0A8
:10CB700050E00E9445EECA01B9012AE030E040E0F1
:10CB800050E00E9445EE605D60938104C701B601EC
:10CB900028EE33E040E050E00E9445EE9AE0892E16
:10CBA000912CA12CB12CCA01B901A50194010E94BC
:10CBB00045EE605D60938204C701B60124E630E073
:10CBC00040E050E00E9445EECA01B901A501940180
:10CBD0000E9445EE605D609383048EE2809384043E
:10CBE000C701B601A50194010E9445EE6B01CA017F
:10CBF000B901A50194010E9445EE605D6093850432
:10CC0000F0E3CF0EC092860481E894E0FF90EF90AD
:10CC1000DF90CF90BF90AF909F908F907F906F905C
:10CC20005F904F90089560E070E080EA90E48DCFCF
:10CC3000F094E094D094C094C11CD11CE11CF11C70
:10CC40006DE2A2CF20E030E0A901C701B6010E9449
:10CC5000F5E787FF6BC060E070E080EA90ECA5012B
:10CC600094010E9413EF2DEC3CEC4CEC5DE30E9430
:10CC70005AE80E94F5EF4B015C0120E030E0A90189
:10CC8000C701B6010E94F5E787FD0BC020E030E048
:10CC900040E251E4C701B6010E94B2F060E287FDB4
:10CCA00013C0B7FC48C0C501B40128EE33E040E032
:10CCB00050E00E9445EECA01B9012AE030E040E0B0
:10CCC00050E00E9445EE605D60938204C501B401AE
:10CCD00024E630E040E050E00E9445EE8AE0482E35
:10CCE000512C612C712CCA01B901A30192010E943F
:10CCF00045EE605D609383048EE280938404C501F9
:10CD0000B401A30192010E9445EE6B01CA01B90171
:10CD1000A30192010E9445EE605D6093850480E36B
:10CD2000C80EC092860482E894E070CF60E070E0A4
:10CD300080EA90E494CFB094A09490948094811C65
:10CD4000911CA11CB11C6DE2BFCF282F81E32436BA
:10CD500009F080E28093830490E22A3040F03AE0C8
:10CD6000822F632F0E9480EE0E9480EE905D909350
:10CD70008404822F6AE00E9480EE905D9093850487
:10CD800085E28093860483E894E0089560915501DC
:10CD900070915601072E000C880B990B0E94FBE73F
:10CDA0002AE037ED43E25CE30E945AE860937101A8
:10CDB0007093720180937301909374010895CF93DF
:10CDC000DF93EC01CB01BA010E94FBE723E333E3DD
:10CDD00043E250E40E945AE820E030E040E05FE3A4
:10CDE0000E9413EF0E94FAEF6883DF91CF910895BC
:10CDF0000E94FBE723E333E343E250E40E945AE856
:10CE000020E030E040E05FE30E9413EF0E94FAEF81
:10CE100024E6629FC001112481589F4F6FEF70E09C
:10CE20000E94ADEE862F91CF80915507811104C0ED
:10CE300080912C0780938807089580919714882308
:10CE4000C1F0815080939714EAEDF2E1882351F00C
:10CE50008150990B2BE1289FF001299FF00D11249F
:10CE6000E757FC4E8BE1AFEBB2E101900D928A9552
:10CE7000E1F720919714211105C08091A1148064DD
:10CE80008093A11481E090E0A0E0B0E0211103C004
:10CE900080E090E0DC0180934B0790934C07A093D7
:10CEA0004D07B0934E071092460781E080934807E4
:10CEB00083E080936C010895CF93DF93EC01CB0165
:10CEC000BA010E94FBE7688379838A839B83DF91A1
:10CED000CF910895CF93DF93EC01CB01BA010E946B
:10CEE000FBE72DEC3CEC4CEC5DE30E945AE86883D8
:10CEF00079838A839B83DF91CF910895CF93DF93CA
:10CF0000EC01CB01BA010E94FBE72AE037ED43E2D6
:10CF10005CE30E945AE8688379838A839B83DF916C
:10CF2000CF910895CF92DF92EF92FF92CF93DF934C
:10CF300000D000D0CDB7DEB70E94FBE72AE037ED86
:10CF400043E25CE30E945AE86B017C0120E030E0A0
:10CF5000A9010E94F5E72DEB37E346E055E387FF93
:10CF600004C02DEB37E346E055EBC701B6010E9444
:10CF700013EF69837A838B839C83CE010196A9DDAD
:10CF80000F900F900F900F90DF91CF91FF90EF9047
:10CF9000DF90CF900895CF93DF93EC01CB01BA01DE
:10CFA0000E94FBE70E94F5EF79836883DF91CF91C0
:10CFB00008958F929F92AF92BF92CF92DF92EF929D
:10CFC000FF92FC01C080D180E280F38020E030E05D
:10CFD000A901C701B6010E94F5E787FD99C06DEB75
:10CFE00077E386E095E3A70196010E9413EF9F7710
:10CFF00020E030E048EC52E40E945AE820E030E0C3
:10D0000040EA50E40E9413EF2DEC3CEC4CEC5DE365
:10D010000E945AE80E94F5EF6B017C0180E2809348
:10D02000800460E2F0E1CF16F7E2DF06E104F104EC
:10D030008CF0C701B60120E137E240E050E00E94E9
:10D0400045EECA01B9012AE030E040E050E00E941C
:10D0500045EE605D6093810460E288EEC81683E06F
:10D06000D806E104F1048CF0C701B60128EE33E0E4
:10D0700040E050E00E9445EECA01B9012AE030E0EC
:10D0800040E050E00E9445EE605D6093820460E203
:10D09000E4E6CE16D104E104F1048CF0C701B60138
:10D0A00024E630E040E050E00E9445EECA01B901BC
:10D0B0002AE030E040E050E00E9445EE605D609381
:10D0C00083048AE0882E912CA12CB12CC701B601D3
:10D0D000A50194010E9445EE6B01CA01B901A501A9
:10D0E00094010E9445EE605D609384048EE280931B
:10D0F0008504F0E3CF0EC092860480E894E0FF90B0
:10D10000EF90DF90CF90BF90AF909F908F90089559
:10D110006DEB77E386E095EB66CFA4E0B0E0E3E962
:10D12000F8E60C94EBEE0E94FBE72DEC3CEC4CECAB
:10D130005DE30E945AE869837A838B839C83CE01E6
:10D14000019637DF2496E2E00C9407EFCF93DF934C
:10D15000EC018D810E94FA4060E08B810E9459CDE4
:10D16000DF91CF910895CF92DF92EF92FF920F93CC
:10D170001F93CF938C01C62F69017A01E7DF0E94CC
:10D1800028CF8C2F80640E94EE408F2D0E94EE40AD
:10D190008E2D0E94EE408D2D0E94EE408C2D0E941F
:10D1A000EE4087E8C11101C085E90E94EE40CC3015
:10D1B00011F40E94F340C0E00E94F340F80186831E
:10D1C00087FF04C0CF3F11F0CF5FF6CFCF911F9103
:10D1D0000F91FF90EF90DF90CF90089561E0FC01F8
:10D1E00083810E9459CD8FEF0C94EE400F931F93D3
:10D1F000CF938C01ABDF0E9428CFC82F882369F022
:10D200008DEF0E94EE400E9428CFC82FC801E6DFB4
:10D210008C2FCF911F910F91089582E1F8018483A3
:10D22000F5CFB0E0A0E0E7E1F9E60C94E1EEEC0127
:10D230006A017B014801590120E030E0A90167E360
:10D2400092DFA501980167E1CE018DDF81111DC03C
:10D250008F81833039F089E0CC0CDD1CEE1CFF1C83
:10D260008A95D1F7A701960169E1CE017CDF11E033
:10D27000882319F010E087E08C83CE01AFDF812F87
:10D28000CDB7DEB7ECE00C94FDEE89E08C8310E0C6
:10D29000F4CFCF93DF93EC016EBDFA01CA019E5F1C
:10D2A0000DB407FEFDCF20812EBD0DB407FEFDCFCE
:10D2B00021812EBD3296E817F90791F70DB407FECC
:10D2C000FDCF8FEF0E94EE408FEF0E94EE400E9454
:10D2D000F3408E838F71853041F083E18C83CE01E2
:10D2E0007DDF80E0DF91CF91089581E0FBCF0F9348
:10D2F0001F93CF93DF93EC018B0128DF0E9428CF8F
:10D3000081110BC085E18C8310E0CE0167DF812F96
:10D31000DF91CF911F910F910895A8016CEFCE017D
:10D32000B8DF182F882371F3F0CF0F931F93CF939B
:10D33000DF93EC0189018F81833039F089E0440F5C
:10D34000551F661F771F8A95D1F79A01AB0168E1D7
:10D35000CE0109DF811127C0A8016EEFCE0199DF50
:10D36000182F8823A9F00E9428CF182F8823C1F0F6
:10D3700020E030E0A9016DE0CE01F5DE882321F048
:10D3800086E18C8310E004C00E94F3408111F8CF45
:10D39000CE0124DF812FDF91CF911F910F9108954E
:10D3A00087E18C83F5CF86E0ECCF1F93CF93DF939B
:10D3B000EC01CCDE20E030E0A9016CE0CE01D3DE50
:10D3C00011E0882319F010E083E08C83CE0106DFA2
:10D3D000812FDF91CF911F9108951F93CF93DF93FA
:10D3E000EC018F81833039F089E0440F551F661FAF
:10D3F000771F8A95D1F79A01AB0162E1CE01B3DEC6
:10D4000011E0882319F010E085E08C83CE01E6DE80
:10D41000812FDF91CF911F9108958F929F92AF92AC
:10D42000BF92EF92FF920F931F93CF93DF938C01E4
:10D43000EB017A010E943ECE4B015C012CE2820E90
:10D4400021E0921EA11CB11C0E94F340F8018683CA
:10D450008F3F69F40E943ECE681979098A099B09B9
:10D4600097FDF2CF81E1F8018483C0E021C08E3FB7
:10D4700069F5F1E0EF1AF1088FEF8EBDFE012FEF95
:10D480000DB407FEFDCF8EB581932EBDCF018C1B51
:10D490009D0B8E159F05A0F30DB407FEFDCF8EB535
:10D4A000CE0DDF1D88830E94F3400E94F340C1E04F
:10D4B000C80194DE8C2FDF91CF911F910F91FF90C7
:10D4C000EF90BF90AF909F908F9008958FE0CBCF5B
:10D4D0000F931F93CF93DF93EC018B0137DE40E076
:10D4E00052E0B801CE0199DFDF91CF911F910F91EA
:10D4F00008950F931F93CF93DF93EC0189018F81E0
:10D50000833039F089E0440F551F661F771F8A95D5
:10D51000D1F79A01AB0161E1CE0125DE882351F0FC
:10D5200084E08C83CE015ADE80E0DF91CF911F91A1
:10D530000F91089540E052E0B801CE016EDFF5CFC3
:10D54000B0E0A0E0E6EAFAE60C94E1EEEC01162F7A
:10D550001F821C824B830E943ECE6B017C0120ED1A
:10D56000C20E27E0D21EE11CF11CA89561E08B8160
:10D570000E9459CD8B810E9407B3249A2C9A279A36
:10D580002698259A81E00E94FA4085E08D830E94CA
:10D59000FA400AE08FEF0E94EE400150D9F7A895BB
:10D5A00020E030E0A90160E0CE01DDDD8E83813036
:10D5B00079F00E943ECE6C197D098E099F0997FD76
:10D5C000EFCF81E08C83CE0109DE1A8280E065C056
:10D5D000A8952AEA31E040E050E068E0CE01C3DDE2
:10D5E000853031F581E08F83A8958F81812C912C36
:10D5F0005401823029F4812C912CA12C80E4B82E86
:10D6000020E030E0A90167E3CE01ADDDA501940182
:10D6100069E2CE01A8DD8E838823F1F00E943ECE20
:10D620006C197D098E099F0997FDEACF8AE0CACF60
:10D6300004E00E94F3408E830150D9F78A3A11F436
:10D6400082E0D1CF0E943ECE6C197D098E099F09E0
:10D6500097FDBFCF82E0B6CF8F818230B9F420E052
:10D6600030E0A9016AE3CE017EDD882311F088E075
:10D67000A9CF0E94F340807C803C11F483E08F832B
:10D680000E94F3400E94F3400E94F340CE01A6DDC9
:10D6900081E08A83173030F41D83CDB7DEB7ECE02C
:10D6A0000C94FDEE88E18C8391CF0F931F93CF9361
:10D6B000DF93EC018B0120E030E0A90169E053DD4C
:10D6C000882351F080E18C83CE0188DD80E0DF91FA
:10D6D000CF911F910F91089540E150E0B801CE0124
:10D6E0009CDEF5CFCF93C82FCB010E945E3488E932
:10D6F0009DE10E945E3489E89DE1CC2311F08EE823
:10D700009DE10E945E348AE00E943D34CF910895ED
:10D710000C944ACE4091790521E042276CE070E0FC
:10D720000C94DBB24091790521E0422764E070E07F
:10D730000C94DBB24091790521E0422761E070E072
:10D740000C94DBB24091790521E0422761E070E062
:10D750000C94DBB24091790521E0422768E070E04B
:10D760000C94DBB24091790521E042276CE070E037
:10D770000C94DBB241E061E070E00C94DBB24091CC
:10D78000790521E042270C94DBB26CE070E00C9448
:10D79000E8CD61E070E00C94E8CD61E070E00C94BD
:10D7A000E8CD6CE070E00C94E8CD64E070E00C949F
:10D7B000E8CD9091980481E089270C941E2A61E0BD
:10D7C0008CE297E00C94AA2A20E030E0A901BC0189
:10D7D00087E791E00C94F5C380E090E0A0E8B0E426
:10D7E00080937F0190938001A0938101B093820187
:10D7F00088E492E0E9DF80E090E0A0EFB1E480937C
:10D80000770190937801A0937901B0937A01809386
:10D810007B0190937C01A0937D01B0937E01E09108
:10D82000D505EE0FFF0BE85DFD4F808191818330C0
:10D83000910539F184309105C9F1029761F480E0D6
:10D8400090E0A3E4B3E48093770190937801A093F0
:10D850007901B0937A0180E392E0B6DF10927F0104
:10D8600010928001109281011092820188E492E06E
:10D87000ABDF8091D5058F5F8430ECF48093D505C4
:10D88000089580E090E0A3E4B3E48093770190935F
:10D890007801A0937901B0937A0180937B019093F2
:10D8A0007C01A0937D01B0937E01D5CF80E090E014
:10D8B000A3E4B3E4F2CF1092D5050895A4E0B0E05C
:10D8C000E4E6FCE60C94EBEE84EF91E0A0E0B0E03F
:10D8D00089839A83AB83BC83BE016F5F7F4F88E7E8
:10D8E0000E9405332496E2E00C9407EFB0E0A0E03C
:10D8F000ECE7FCE60C94EBEE20E24F8158856E815C
:10D900008D810E940CC9E2E00C9407EF80912C07F6
:10D9100090912D070C947FCE68ED78E982E00C940D
:10D920001ACB6CED78E981E00C941ACB60EE78E9C3
:10D9300080E00C941ACB64EE78E983E00C941ACB67
:10D94000109246070C94BFD44FE350E06DEC7BE19E
:10D950008AEE96E00C94C7F18091371390913813BA
:10D96000891B8F7011F40C94FE2B81E00895809137
:10D970006C01882341F06091CD057091CE0541E0A6
:10D9800081E00C94ACC808950F931F93CF93DF935D
:10D99000FC012381222331F080E0DF91CF911F91A0
:10D9A0000F9108958B01EC01FB018789803139F5D6
:10D9B00082E08B831D8A1E8A1F8A188E808D918D2E
:10D9C000B0E0A0E025E0880F991FAA1FBB1F2A9591
:10D9D000D1F7898B9A8BAB8BBC8B1A8F098F81E027
:10D9E0008983188619861A861B861C821D821E82D0
:10D9F0001F82188A1C861D861E861F86CECF803207
:10DA000059F683E08B83428D538D648D758D4D8BDC
:10DA10005E8B6F8B788F9E012F5E3F4FC8010E94F7
:10DA20001DD68111DACFB8CFCF93DF93EC010E94DE
:10DA300086D61B82DF91CF910895CF93DF93EC01BF
:10DA4000462F41706C857D858E859F850E942FD3E2
:10DA5000882351F0888920E2829FC00111248A58CE
:10DA60009F4EDF91CF91089590E080E0FACFCF9361
:10DA7000DF93EB01FC012381211104C080E0DF91E1
:10DA8000CF9108952250223028F48FE288831982A2
:10DA900081E0F5CF60E0D1DF009781F3DC0160E049
:10DAA00080E09EE22D91203299F0883031F49E0181
:10DAB000260F311DF90190836F5F9E01260F311DE6
:10DAC000AD0141505109FA014081F90140836F5F76
:10DAD0008F5F8B3039F7FE01E60FF11D1082D8CF32
:10DAE000ACE0B0E0E6E7FDE60C94DCEE5C01DC01C6
:10DAF00059968D909C90F40181859285A385B4857B
:10DB00009C01AD012F5F3F4F4F4F5F4F29873A87F1
:10DB10004B875C87D50114964D905D906D907C90FD
:10DB20001797411451046104710409F459C0BFEFFF
:10DB30004B1A5B0A6B0A7B0A312C730162011D824E
:10DB40001E821F821886F40181859285A385B48583
:10DB50002D813E814F815885281739074A075B0779
:10DB600008F056C089859A85AB85BC858C159D05C6
:10DB7000AE05BF0550F482E0C82ED12CE12CF12C6B
:10DB800092E0492E512C612C712C9E012F5F3F4F4A
:10DB9000B701A601C4010E94A1D58823C9F18981DA
:10DBA0009A81AB81BC81892B8A2B8B2B01F12601B9
:10DBB00037019FEF491A590A690A790A2D813E8176
:10DBC0004F8158852F5F3F4F4F4F5F4F2D833E83CF
:10DBD0004F8358873FEFC31AD30AE30AF30AB3CF40
:10DBE000408051806280738033243394A6CFC41464
:10DBF000D504E604F70411F70FEF1FEF2FEF3FE016
:10DC0000B701A601C4010E9427D5782E811106C054
:10DC1000712C872D2C96E1E10C94F8EEF5014481EE
:10DC2000558166817781411551056105710539F08E
:10DC300097018601C4010E9427D5882349F3D501A5
:10DC40001496CD92DD92ED92FC921797332051F00D
:10DC5000D701C6010196A11DB11DF40180839183F6
:10DC6000A283B383F50185899689A789B08D892B15
:10DC70008A2B8B2B71F6C58AD68AE78AF08E818132
:10DC800080688183C6CF40E050E0BA010C94CFD6C3
:10DC90004F925F926F927F92AF92BF92CF92DF923C
:10DCA000EF92FF920F931F93CF93DF931F92CDB705
:10DCB000DEB78C017B015A01C22EDB0159968D9192
:10DCC0009C91F801928F818FCB01DDDF712CF701E0
:10DCD00080859185A285B38541895289638974893C
:10DCE00084179507A607B70708F052C055E0B69508
:10DCF000A795979587955A95D1F7F82FFF70DF2E46
:10DD0000D70113968C91823010F480E0DAC041E0A4
:10DD100050E0BE016F5F7F4FC7010E94CAD70197D5
:10DD2000A1F7F70180859185A285B3854F96A11D46
:10DD3000B11D80879187A287B387F0E2DF9EB00193
:10DD400011246A587F4E61157105F9F2DB018C913F
:10DD5000882341F0853E09F04BC0772029F07724D5
:10DD60007394B5CF71100EC0809176129091771296
:10DD7000A0917812B0917912F80184879587A687CF
:10DD8000B787D08ADB018C918111E9CF7724739416
:10DD90008C2D8274823409F0B8CF772009F4A1C0A9
:10DDA000F801D08861E0C80148DE009709F4ADCFE2
:10DDB00020E2DC011D922A95E9F72BE0F501DC0158
:10DDC00001900D922A95E1F721E238E2FC01318BB6
:10DDD000208B40E058E057874687338B228B318F6A
:10DDE000208F578B468B0E94E6D2811109C08DCFC0
:10DDF0004BE050E0C5010E9477F1892B09F067CF15
:10DE0000F0E2DF9ED00111249D012A583F4EF90116
:10DE10008385817121F08C2D827109F000C1F80198
:10DE2000818D928D40917612509177126091781287
:10DE3000709179124487558766877787D08AFD016C
:10DE4000EA58FF4E44885588712C612C32015524C4
:10DE50004424D80155964D925D926D927C925897CC
:10DE6000428D538D70E060E0442955296629772959
:10DE700055964D935D936D937C935897D9011B965E
:10DE80002C91287109F0BDC0848D958DA68DB78D1C
:10DE9000F801818B928BA38BB48B81E083838C2DD3
:10DEA0008F70F80181831482158216821782108682
:10DEB00011861286138681E0C4FE03C0C8010E9449
:10DEC00054D70F90DF91CF911F910F91FF90EF905A
:10DED000DF90CF90BF90AF907F906F905F904F900A
:10DEE0000895D70113968C911397823009F40DCFC2
:10DEF00051968D919D910D90BC91A02D803E9F4F8C
:10DF0000AF41B10508F001CFC701EADD882309F46C
:10DF1000FCCE0E94E6D2882309F4F7CED7015996A9
:10DF2000ED91FC915A9714964D905D906D907C9078
:10DF30001797B2E04B1A510861087108858504C033
:10DF4000440C551C661C771C8A95D2F786859785EC
:10DF5000A089B189480E591E6A1E7B1E81E08093FC
:10DF60007A124092761250927712609278127092E2
:10DF70007912E6E7F0E180E092E0DF019C011D927A
:10DF800021503040E1F7DD24D394D7015996ED912B
:10DF9000FC918481D816C0F480917B1290917C1200
:10DFA000DC01ED91FC910288F389E02D26E730E158
:10DFB000B301A2014D0D511D611D711D09958823ED
:10DFC00009F4A3CED394E1CF258580E092E0A0E0D0
:10DFD000B0E004C0880F991FAA1FBB1F2A95D2F773
:10DFE000F7014189528963897489840F951FA61F9F
:10DFF000B71F818B928BA38BB48B86E790E1D12CDA
:10E00000D7CE203161F498012F5E3F4F0E941DD67C
:10E01000882329F084E0D80113968C9340CFD8014F
:10E0200013961C9272CEFC0123812111FDCC089520
:10E03000A1E4B0E0EEE1F0E70C94DBEE4C015B0113
:10E040007A01222E19821C821C8E1F8E6115710589
:10E0500069F410E0CE014C96E6DFCE010196E3DFD5
:10E06000812FCF5BDF4FE2E10C94F7EEFC0183815F
:10E070008111EFCFFA0180818F3251F18B01CE01F6
:10E0800001966C012C0180E2382E360122963FAEBB
:10E09000229721963FAE21973FAE3EAE3DAE3CAEBD
:10E0A0003BAE3AAE39AE38AE3FAA970190E047E0BA
:10E0B000D9018D91882309F446C08F3209F443C0F9
:10E0C0008E3201F54A3029F298E04AE09D01F0CF06
:10E0D000FB0183818250823098F0618D728DCE0178
:10E0E0004C9652DC882309F4B4CF8E01045E1F4F96
:10E0F000C7017C010196F70120812F32D1F3BFCFF8
:10E100008B01F6CFE9E2FAE22491222321F0319645
:10E110008213FACF9ECF491708F49BCF813208F4BF
:10E1200098CF8F3709F495CF3FE9380F3A3108F48B
:10E1300020EEE7E3F0E0EC0FFD1FE90FF11D820F89
:10E1400080839F5FC3CF8FA9803209F482CF79018A
:10E15000F90180812F5F3F4F8F32C9F38823C1F0CF
:10E1600021E0AE01495C5F4FB801C60191DD882313
:10E1700009F46FCF0A151B0511F0C80155DCCE015B
:10E180004C964C145D0409F0C30186016C017ECFEE
:10E19000222DAE01495C5F4FB801C40179DD182F13
:10E1A00059CF8F929F92AF92BF92CF92DF92EF9210
:10E1B000FF920F931F93CF93C82F0BE812E1F80142
:10E1C00060857185072E000C880B990B0E94FBE778
:10E1D0006B017C01F80184809580A680B78080E285
:10E1E0000E943D3484E50E943D348AE30E943D3420
:10E1F00042E0C501B4010E9426B382E29AE20E9485
:10E200005E3442E0C701B6010E9426B362E070E0CE
:10E2100080E090E00E94B5CD87E1C802F0011124B2
:10E22000E557FD4E628570E085E29AE20E94683F04
:10E23000CF911F910F91FF90EF90DF90CF90BF9003
:10E24000AF909F908F9008950F930FB70F93009109
:10E250006E000B7F00936E0078940F930BB70F93B3
:10E260000CB70F921F922F933F934F935F936F932F
:10E270007F938F939F93AF93BF93EF93FF9311245B
:10E280000E94C4ABFF91EF91BF91AF919F918F918D
:10E290007F916F915F914F913F912F911F900F90C0
:10E2A0000CBF0F910BBF0F910460F89400936E00A8
:10E2B0000F910FBF0F911895CF93DF9310928705A1
:10E2C000CBE8D2E1198618860E944ACE1A865D985C
:10E2D000DF91CF910895EF92FF920F931F93CF9309
:10E2E000C82F7B018A0180912B078330E0F00E94C8
:10E2F000F83DC7010E945E3488EA99E20E945E34CC
:10E30000C7FD0EC086EA99E20E945E346C2FCC0FE6
:10E31000770B880B990B0E94DCB08AE00E943D3499
:10E320008AE00E943D34C8DFA89580917006811173
:10E330000DC081E08093700682E080932B07BCDFE4
:10E3400040E063EA79E2C8010E941A40CF911F9130
:10E350000F91FF90EF900895CF93DF93A895809150
:10E360008D1290918E120E9454B260938F1270930E
:10E3700090128093911290939212C0918D12D0912D
:10E380008E128091650190916601C817D90734F407
:10E3900044EE59E261EF79E280E09DDF80919312D3
:10E3A00090919412181619066CF480916301909163
:10E3B00064018C179D0734F443E05AE260E17AE28D
:10E3C00080E089DFDF91CF9108958F929F92AF9285
:10E3D000BF92CF92DF92EF92FF92CF93DF9300D064
:10E3E00000D0CDB7DEB780912B07811110C0A89562
:10E3F0000F900F900F900F90DF91CF91FF90EF90C3
:10E40000DF90CF90BF90AF909F908F9008958091B4
:10E4100071068111EDCF81E08093710680918805AE
:10E42000811103C010927106E3CF96DF1092880528
:10E430000E943ECE6B017C010E94F7B04B015C0153
:10E440006091690170916A01072E000C880B990B8D
:10E450000E94FBE79B01AC01C501B4010E94B2F030
:10E4600018160CF469C06091931270919412072EE3
:10E47000000C880B990B0E94FBE769837A838B83DE
:10E480009C83CE0101960E9489CE80908F1290903D
:10E490009012A0909112B0909212609167017091C9
:10E4A0006801072E000C880B990B0E94FBE79B016B
:10E4B000AC01C501B4010E94B2F01816CCF4609111
:10E4C000690170916A01072E000C880B990B0E945C
:10E4D000FBE79B01AC01C501B4010E94F5E787FF92
:10E4E00007C00E9400B10E94F5EF7595679501C0C5
:10E4F00060E0609395128091871290918812A091AC
:10E500008912B0918A120097A105B10509F48ACF4A
:10E51000C81AD90AEA0AFB0AF7FC84CF0E94F7B0AE
:10E520000E94F5EF209185123091861262177307D1
:10E5300054F00E944ACE76CF44EE59E261EF79E280
:10E5400080E0C9DE90CF46EC59E265ED79E280E0EB
:10E55000C2DE68CFCF92DF92EF92FF92CF93DF932C
:10E56000EC01C880D980EA80FB8089E999E20E94A9
:10E570005E34C701B6010E946826CC80DD80EE8043
:10E58000FF8087E290E30E945E34C701B6010E94DB
:10E590006826C884D984EA84FB8483E290E30E94DD
:10E5A0005E34C701B6010E9468268AE00E943D34AD
:10E5B000DF91CF91FF90EF90DF90CF900895BC0155
:10E5C00020915106309152064091510650915206C9
:10E5D0002417350731F481E02617370709F080E06A
:10E5E00008959A01F1CF0F930FB70F9300916E002A
:10E5F0000F930B7F00936E0000916F000D7F0093CF
:10E600006F000F930BB70F930CB70F921F922F93BE
:10E610003F934F935F936F937F938F939F93AF93AA
:10E62000BF93EF93FF931124E1D4FF91EF91BF913A
:10E63000AF919F918F917F916F915F914F913F919A
:10E640002F911F900F900CBF0F910BBF0F91026085
:10E65000F89400936F000F9100936E000F910FBF1D
:10E660000F91189500C000C08091E50680FF1FC083
:10E67000459A8FEF80930A068091E50681FF1AC0C4
:10E68000479A8FEF80930B068091E50682FF15C0B5
:10E690002A988FEF80930C068091E50683FF10C0C7
:10E6A00028988FEF80930D0600C000C0089545980C
:10E6B00081E0E0CF479881E0E5CF2A9A81E0EACF78
:10E6C000289A81E0EFCF80917A05982F977F9093D9
:10E6D0007A05982F937081E011F080E008955E9A9A
:10E6E00008955E9880917A05886080937A050895F0
:10E6F000E82FF0E021E030E0082E02C0220F331FA7
:10E700000A94E2F72095309590917A0592239093A0
:10E710007A05EC5DFD4F2081922321E019F020E085
:10E72000822F0895813079F038F08230C9F7159A38
:10E73000909158079B7F04C05E9A909158079E7FE6
:10E7400090935807EDCF5E9A909158079D7FF8CF30
:10E7500080E0CEDF81E0CCDF82E0CADFB4CF813061
:10E7600079F070F0823071F021E030E001C0220FCA
:10E770008A95EAF780917A05822B80937A0508952D
:10E780005E98F2CF1598F0CFB0E0A0E0EAECF3E7A6
:10E790000C94E3EECAE4DDE000E717E08AE5A82E7A
:10E7A0008DE0B82EC12CD12C7601C394699179915A
:10E7B000899199910E94F9E7288939894A895B8969
:10E7C0000E945AE80E94FAEFF801619371938193D5
:10E7D00091938F01C616D706E806F90610F46B016F
:10E7E0007C01AC16BD0611F76FEF7FEFCB01A701DF
:10E7F00096010E9423EE2093800730938107409377
:10E80000820750938307CDB7DEB7EAE00C94FFEEA2
:10E810000F931F93CF93DF930EE51DE0C9E8D7E078
:10E82000F80121913191419151918F0160E070E0A7
:10E8300080E89FE30E948DEF699379938993999380
:10E84000F7E0C939DF0761F70E9418C49DDFDF9147
:10E85000CF911F910F910895DBCFDACFD9CFD8CFC9
:10E860009091371380913813981306C08091920DC0
:10E870009091930D892B21F080E00E940B41F0CF05
:10E8800008959091371380913813981307C08091A1
:10E89000920D9091930D892B09F45ACF80E00E943C
:10E8A0000B41EFCFCF92DF92EF92FF92CF93DF93A6
:10E8B00020919804222319F1EC0108960E94CF2799
:10E8C0006B017C0120E030E0A9010E94F5E720E027
:10E8D00030E0A901882349F0CE010E944728A70112
:10E8E00096010E945AE89B01AC01688579858A856A
:10E8F0009B850E9412EF688779878A879B87DF91C3
:10E90000CF91FF90EF90DF90CF900895CF92DF925C
:10E91000EF92FF92CF93DF9320919804222319F175
:10E92000EC0108960E94CF276B017C0120E030E0CB
:10E93000A9010E94F5E720E030E0A901882349F011
:10E94000CE010E944728A70196010E945AE89B0128
:10E95000AC01688579858A859B850E9413EF68875D
:10E9600079878A879B87DF91CF91FF90EF90DF9027
:10E97000CF900895AEE1B0E0E0ECF4E70C94DDEE6A
:10E980009E8F8D8F5B018A01FC01EA5BFF4F208126
:10E99000318142815381298B3A8B4B8B5C8BCA012D
:10E9A000B9010E94F9E76B017C01D5012D913D91E0
:10E9B0004D915C910E945AE80E9477EF2B013C0137
:10E9C000F8012081318142815381C701B6010E9443
:10E9D0005AE80E9477EF4B015C01C301B2010E942B
:10E9E000FAEF6D8B7E8B8F8B988F68377105810561
:10E9F000910540F428E730E040E050E02D8B3E8B5D
:10EA00004F8B588FC501B4010E94FAEF698F7A8F3E
:10EA10008B8F9C8F683771058105910540F488E7DD
:10EA200090E0A0E0B0E0898F9A8FAB8FBC8FED8D26
:10EA3000FE8DEE5AFF4F208131814281538129871B
:10EA40003A874B875C87CA01B9010E94FBE72B011B
:10EA50003C016D897E898F89988D0E94F9E76D83CD
:10EA60007E838F83988720E030E0A901C301B20143
:10EA70000E94F5E7882309F4BBC1A7019601C701ED
:10EA8000B6010E945AE84B015C012D813E814F8105
:10EA90005885CA01B9010E945AE89B01AC01C50121
:10EAA000B4010E9412EF4B015C01A3019201C3016A
:10EAB000B2010E9413EF9B01AC01C501B4010E9499
:10EAC0008DEF0E9477EF0E94FAEF69837A838B8340
:10EAD0009C8369857A858B859C85909580957095BA
:10EAE00061957F4F8F4F9F4F0E94FBE74B015C0169
:10EAF000698D7A8D8B8D9C8D0E94F9E769877A8765
:10EB00008B879C8720E030E0A901C501B4010E94F9
:10EB1000F5E7882309F470C129853A854B855C8522
:10EB2000CA01B9010E945AE86D877E878F87988B4A
:10EB3000A7019601C701B6010E945AE89B01AC01EA
:10EB40006D857E858F8598890E9412EF6B017C010F
:10EB5000A5019401C501B4010E9413EF9B01AC0112
:10EB6000C701B6010E948DEF0E9426F0AD8DBE8DCB
:10EB700095962D913D914D915C9198972D873E876B
:10EB80004F87588B69017A0129813A814B815C81D9
:10EB9000C21AD30AE40AF50A0E94FAEFC61AD70A83
:10EBA000E80AF90AF7FE8CC02D813E814F81588515
:10EBB000CA01B9010E945AE86B017C0120E030E0F3
:10EBC000A901C301B2010E94F5E7882309F418C125
:10EBD0006D857E858F8598890E94F9E79B01AC0140
:10EBE0000E9413EFA30192010E945AE84B015C01BD
:10EBF00029853A854B855C85CA01B9010E945AE88E
:10EC00009B01AC01C501B4010E9413EFA70196015D
:10EC10000E9412EF4B015C0120E030E040E850E43C
:10EC2000C301B2010E945AE89B01AC01C501B401C5
:10EC30000E948DEF0E9477EF4B015C0120E030E0F5
:10EC4000A9010E94B2F087FF03C0812C912C5401CE
:10EC5000C501B4010E94FAEF69837A838B839C8398
:10EC60002D853E854F855889261737074807590750
:10EC700020F429833A834B835C8369817A818B8179
:10EC80009C810E94F9E74B015C01A3019201C30141
:10EC9000B2010E9413EF9B01AC01C501B4010E94B7
:10ECA0005AE8A70196010E9413EF0E94F1F00E941A
:10ECB000FAEF698B7A8B8B8B9C8BC12CD12C7601D4
:10ECC00069897A898B899C892D893E894F89588DDC
:10ECD000621B730B840B950B0E94F9E7A301920151
:10ECE0000E948DEF20E034E244EF59E40E945AE89C
:10ECF0000E94FAEF4B015C0169897A898B899C89B2
:10ED0000298D3A8D4B8D5C8D621B730B840B950B9B
:10ED10000E94F9E7A30192010E948DEF20E034E206
:10ED200044EF59E40E945AE80E94FAEF6D837E8313
:10ED30008F839887C501B4010E94D8632B013C01E1
:10ED40006D817E818F8198850E94D86329813A8167
:10ED50004B815C81AD8DBE8D99962D933D934D93E6
:10ED60005C939C9789019A010C0D1D1D2E1D3F1D62
:10ED7000FD0105A716A727A730ABE65BFF4F2D893E
:10ED80003E894F89588D2083318342835383D596A2
:10ED90008D929D92AD92BC92D8972D813E814F81EC
:10EDA0005885D9962D933D934D935C93DC973D9771
:10EDB000408251826282738234966083718382833F
:10EDC000938329893A894B895C89D1962D933D9308
:10EDD0004D935C93D4973D96298D3A8D4B8D5C8DE8
:10EDE00020833183428353836E96E0E10C94F9EEE5
:10EDF00060E070E0CB0165CE60E070E0CB01B4CEA6
:10EE000060E070E0CB0116CF90916F0081E091FD42
:10EE100002C080E0089590916F009D7F90936F00F5
:10EE20000895EFE6F0E08081826080830895CF93BB
:10EE3000C82FEADF94E0C99F90011124F901EC5A30
:10EE4000F94F205A394FD9014D915D916D917C91C7
:10EE5000408351836283738391E0909353068111C1
:10EE6000E0DFCF910895CF93DF938091E406811185
:10EE700005C08091E606882309F44EC08091E5051F
:10EE8000329B4DC081608093E5058091E505339B01
:10EE900048C082608093E5058091E505349B43C0BE
:10EEA00084608093E505C0914406C0FF0FC0809147
:10EEB000E50680FF0BC08091E50580FF07C08091CB
:10EEC0002A07816080932A0780E0B1DFC1FF0FC06D
:10EED0008091E50681FF0BC08091E50581FF07C0A9
:10EEE00080912A07826080932A0781E0A0DFC2FF19
:10EEF00013C08091E50682FF0FC08091E60688234B
:10EF000059F08091E50582FF07C080912A0784604F
:10EF100080932A0782E08BDFDF91CF9108958E7F67
:10EF2000B2CF8D7FB7CF8B7FBCCF6EDF10928407BF
:10EF3000109285071092860710928707811171CF72
:10EF400008950F931F938091371390913813891B65
:10EF50008F7009F449C090913413992361F0833084
:10EF600040F48FEF890F29F08093341390E080E014
:10EF700038C010923413809138132BE5829FC00162
:10EF800011248756984FFC01208120FDEFCF40913E
:10EF90008407509185076091860770918707E95A29
:10EFA000FF4F0081118122813381401B510B620B85
:10EFB000730B409384075093850760938607709383
:10EFC0008707209138132F5F2F70209335133091CE
:10EFD000381320913613321304C020913513209337
:10EFE00036131F910F910895A0DFC0CFA3E1B0E0C9
:10EFF000ECEFF7E70C94DBEE8FEF9FEF9093890037
:10F00000809388002AE02983312C212C78948091E8
:10F010004D0690914E06A0914F06B0915006892B57
:10F020008A2B8B2B09F0C2C1809153068823D1F023
:10F03000809151069091520610925306892B91F0BF
:10F040001092520610925106109244069091371376
:10F0500080913813981731F0809138138F5F8F703B
:10F06000809338138091510690915206892B09F4B0
:10F070009DC14091490650914A0660914B0670919E
:10F080004C068091450690914606A0914706B091A6
:10F09000480600913B0610E030E020E0841B950B11
:10F0A000A60BB70B081719072A073B0710F4D9015D
:10F0B000C8018A8B840F951FA61FB71F809349062E
:10F0C00090934A06A0934B06B0934C06E1E0C090A3
:10F0D0001206D0901306E0901406F0901506809169
:10F0E000220690912306A0912406B0912506C80E11
:10F0F000D91EEA1EFB1EC0922206D0922306E09281
:10F100002406F0922506F7FC33C040910A06042E2F
:10F11000000C550B660B770B809160069091610691
:10F12000A0916206B0916306840F951FA61FB71FBA
:10F130008093600690936106A0936206B093630685
:10F1400080910E0690910F06A0911006B0911106C5
:10F15000B701A601481B590B6A0B7B0BDB01CA01E7
:10F160008093220690932306A0932406B09325064D
:10F170000091160610911706209118063091190675
:10F180008091260690912706A0912806B091290625
:10F19000080F191F2A1F3B1F0093260610932706EE
:10F1A000209328063093290637FD33C040910B0683
:10F1B000042E000C550B660B770B80916406909122
:10F1C0006506A0916606B0916706840F951FA61F7D
:10F1D000B71F8093640690936506A0936606B0936C
:10F1E000670680910E0690910F06A0911006B091CF
:10F1F000110628013901481A590A6A0A7B0AD30103
:10F20000C2018093260690932706A0932806B09308
:10F21000290640911A0650911B0660911C067091B8
:10F220001D0680912A0690912B06A0912C06B09184
:10F230002D06480F591F6A1F7B1F40932A065093C3
:10F240002B0660932C0670932D0677FD33C08090BB
:10F250000C06082C000C9908AA08BB0880916806C7
:10F2600090916906A0916A06B0916B06880D991D70
:10F27000AA1DBB1D8093680690936906A0936A0639
:10F28000B0936B0680910E0690910F06A091100628
:10F29000B09111063A014B01681A790A8A0A9B0A51
:10F2A000D401C30180932A0690932B06A0932C06C9
:10F2B000B0932D0680901E0690901F06A090200609
:10F2C000B090210680912E0690912F06A0913006D5
:10F2D000B0913106880D991DAA1DBB1D80932E0685
:10F2E00090932F06A0933006B0933106B7FD33C03C
:10F2F00040900D06042C000C550866087708809095
:10F300006C0690906D06A0906E06B0906F06840C0F
:10F31000951CA61CB71C80926C0690926D06A0925C
:10F320006E06B0926F0680900E0690900F06A09029
:10F330001006B09011062C013D01481859086A08C2
:10F340007B085301420180922E0690922F06A092D4
:10F350003006B0923106E11104C0E0918400F091D2
:10F360008500F7FE5F9A37FF469A77FF2B9AB7FF23
:10F37000299AE0918400F0918500E0918400F09159
:10F380008500F7FE5F9837FF469877FF2B98B7FF09
:10F3900029985A88552021F0809184009091850009
:10F3A0002A8921502A8BE0E0211191CE80914D06CF
:10F3B00090914E06A0914F06B0915006892B8A2B52
:10F3C0008B2B09F004C740905106509052065B8A7F
:10F3D0004A8A4114510409F456C780914906909114
:10F3E0004A06A0914B06B0914C06409145065091BB
:10F3F0004606609147067091480684179507A60750
:10F40000B70708F49DC080915B01882309F44FC0C1
:10F41000F20185899689A789B08D892B8A2B8B2B40
:10F4200081F4818D928DA38DB48D892B8A2B8B2BAA
:10F4300041F4858D968DA78DB0A1892B8A2B8B2BBE
:10F44000B1F1AA89BB8991966D917D918D919C9125
:10F45000949780907F0590908005A0908105B09052
:10F460008205AB5BBF4F2C9123FF07C09095809521
:10F47000709561957F4F8F4F9F4F0E94FBE72091C2
:10F4800095073091960740919707509198070E94F1
:10F490005AE89B01AC01C501B4010E9412EF6093D0
:10F4A0007F0570938005809381059093820510926B
:10F4B0005206109251061092440690913713809193
:10F4C0003813981709F4DFC6809138138F5F8F7057
:10F4D00080933813A0EDCA2EA7E0DA2EE12CF12C90
:10F4E0008091510690915206892B09F068C629DD5A
:10F4F0009093520680935106892B09F460C6409080
:10F500005106509052065B8A4A8AD2018C9183FF41
:10F5100008C5C20145960E94776310925206109268
:10F520005106109244069091371380913813981722
:10F53000F1F2809138138F5F8F7080933813D7CF9B
:10F5400040914006509141066091420670914306F9
:10F55000481759076A077B0708F40FC240913C0619
:10F5600050913D0660913E0670913F06EA89FB8905
:10F5700085A996A9A7A9B0AD481759076A077B07BF
:10F5800008F0D0C1411551056105710509F066C04B
:10F590008090830590908405A0908505B0908605A5
:10F5A00089E799E2A1E0FC0105911591259134913B
:10F5B000081519052A053B0558F4B694A7949794A5
:10F5C0008794AA0F0496E5E9F9E2E817F90759F7D5
:10F5D000A0933B06F0E28F169104A104B10428F435
:10F5E000E0E28E2E912CA12CB12C20E2821A9108FF
:10F5F000A108B108811438E09306A104B10408F40D
:10F600009AC1A4E09A9EC001112487589A4DFC012A
:10F61000329625913491B82DEE27B39F8001B29F89
:10F62000010D1E1F06940E1F1E1F112430E020E046
:10F63000FC01C590D490F12CE12CC01AD10AE20A49
:10F64000F30A4C0D5D1D6E1D7F1D40933C065093CB
:10F650003D0660933E0670933F0642CF00E01A815C
:10F66000942F852E862FBC81AD81FE81EF81388558
:10F6700029854B80E0917B05E99FA12DFF273091E3
:10F680007C05399FA00DF11D10907D05199EF00D90
:10F69000E89DA00DF11D389DF00DE89FF00D4A2E5C
:10F6A000BF2F4A9EE12D332722274F9EE00D311DAB
:10F6B000201FBA9FE00D311D201FBF9F300D211D5F
:10F6C000432EB22F4A9E112D332722274F9E100D15
:10F6D000311D201FBA9F100D311D201FBF9F300DFF
:10F6E000211D432EB22FEE27909183058090840533
:10F6F000809185050090A402002A09F483C030910E
:10F70000A002349DE119900B800A800B2091A10288
:10F71000249DE0199109800A800B1091A202149D8A
:10F7200090198108800B3B9FE0199109800A800B9A
:10F730002B9F90198108800B1B9F801881094A9E7E
:10F74000112D332722274F9E100D311D201FBA9FE8
:10F75000100D311D201FBF9F300D211D432EB22FD4
:10F7600030919C02349DE10D901F801E801F2091DE
:10F770009D02249DE00D911D801E801F10919E0210
:10F78000149D900D811C801F3B9FE00D911D801EDC
:10F79000801F2B9F900D811C801F1B9F800C811D43
:10F7A0004A9E112D332722274F9E100D311D201FF9
:10F7B000BA9F100D311D201FBF9F300D211D432EFC
:10F7C000B22F30919802349DE119900B800A800B82
:10F7D00020919902249DE0199109800A800B1091D3
:10F7E0009A02149D90198108800B3B9FE0199109A2
:10F7F000800A800B2B9F90198108800B1B9F80181B
:10F80000810982C03091A002349DE10D901F801EBD
:10F81000801F2091A102249DE00D911D801E801F5C
:10F820001091A202149D900D811C801F3B9FE00D42
:10F83000911D801E801F2B9F900D811C801F1B9F80
:10F84000800C811D4A9E112D332722274F9E100DBB
:10F85000311D201FBA9F100D311D201FBF9F300D7D
:10F86000211D432EB22F30919C02349DE119900B43
:10F87000800A800B20919D02249DE0199109800A45
:10F88000800B10919E02149D90198108800B3B9F64
:10F89000E0199109800A800B2B9F90198108800B39
:10F8A0001B9F801881094A9E112D332722274F9EC6
:10F8B000100D311D201FBA9F100D311D201FBF9F3D
:10F8C000300D211D432EB22F30919802349DE10D51
:10F8D000901F801E801F20919902249DE00D911D94
:10F8E000801E801F10919A02149D900D811C801F14
:10F8F0003B9FE00D911D801E801F2B9F900D811C52
:10F90000801F1B9F800C811D11244B821A83BC8396
:10F91000AD83FE83EF8338872987982C892EB12CFD
:10F92000A82E3ECEAA89BB89D1968D909D90AD9090
:10F93000BC90D49735CED501C401B695A7959795BF
:10F9400087958C7F87589E4DFC01C590D490FC0113
:10F95000329625913491E82DE7708E2EE29FC001FA
:10F96000E39F900D112433E0969587953A95E1F742
:10F97000C81AD90AF12CE12C64CE40913706509177
:10F9800038066091390670913A06481759076A0798
:10F990007B0708F030C28090320690903306A0902A
:10F9A0003406B090350680913606EA89FB898111CC
:10F9B0007CC0EF5BFF4FE080F18002811381EA8918
:10F9C000FB89E25BFF4F2081318142815381AA890B
:10F9D000BB89D1966D917D918D919C91D4970E9418
:10F9E0008063B1E0B0933606EA89FB8941A952A948
:10F9F00063A974A989E799E2A1E0FC010591159139
:10FA000025913491041715072607370758F4769582
:10FA1000679557954795AA0F0496E5E9F9E2E81727
:10FA2000F90759F7A0933B0640325105610571056E
:10FA300020F440E250E060E070E04052510961097A
:10FA400071094115F8E05F076105710508F4B3C15C
:10FA500024E0529FC001112487589A4DFC01329630
:10FA600025913491AA27439FF001429FE10DFA1F8F
:10FA70000694EA1FFA1F1124AF0170E060E0FC0158
:10FA8000C590D490F12CE12CC41AD50AE60AF70AE5
:10FA90008C0C9D1CAE1CBF1C8092320690923306CB
:10FAA000A0923406B09235061BCD81AD92ADA3ADC8
:10FAB000B4AD88169906AA06BB0608F072C1811477
:10FAC0009104A104B10449F4409183055091840547
:10FAD00060918505709186058DCFA0E0FA85982DFF
:10FAE000492D8A2DEB857C856D85BE855F8538899E
:10FAF000298950917B05599F612DBB2730917C0549
:10FB0000399F600DB11D10907D05199EB00D549F59
:10FB1000600DB11D349FB00D589FB00DE62F7B2FA7
:10FB2000E69F512D33272227EB9F500D311D2A1FB1
:10FB3000769F500D311D2A1F7B9F300D211DE32F15
:10FB4000722FE69FF12D33272227EB9FF00D311DF9
:10FB50002A1F769FF00D311D2A1F7B9F300D211D1E
:10FB6000E32F722F55279091830540918405809152
:10FB700085050090A4020A2A09F483C03091A002EE
:10FB80003E9F51199A0B4A0B8A0B2091A1022E9F7E
:10FB9000501991094A0B8A0BF091A202FE9F90190D
:10FBA00041098A0B379F501991094A0B8A0B279FED
:10FBB000901941098A0BF79F40198109E69FF12DA1
:10FBC00033272227EB9FF00D311D2A1F769FF00D62
:10FBD000311D2A1F7B9F300D211DE32F722F309185
:10FBE0009C023E9F510D9A1F4A1F8A1F20919D0221
:10FBF0002E9F500D911D4A1F8A1FF0919E02FE9F5D
:10FC0000900D411D8A1F379F500D911D4A1F8A1F5D
:10FC1000279F900D411D8A1FF79F400D811DE69F74
:10FC2000F12D33272227EB9FF00D311D2A1F769FE0
:10FC3000F00D311D2A1F7B9F300D211DE32F722FE8
:10FC4000309198023E9F51199A0B4A0B8A0B2091D2
:10FC500099022E9F501991094A0B8A0BF0919A0232
:10FC6000FE9F901941098A0B379F501991094A0B41
:10FC70008A0B279F901941098A0BF79F4019810928
:10FC800082C03091A0023E9F510D9A1F4A1F8A1FC9
:10FC90002091A1022E9F500D911D4A1F8A1FF091A5
:10FCA000A202FE9F900D411D8A1F379F500D911D8E
:10FCB0004A1F8A1F279F900D411D8A1FF79F400DE5
:10FCC000811DE69FF12D33272227EB9FF00D311D7B
:10FCD0002A1F769FF00D311D2A1F7B9F300D211D9D
:10FCE000E32F722F30919C023E9F51199A0B4A0BC1
:10FCF0008A0B20919D022E9F501991094A0B8A0B65
:10FD0000F0919E02FE9F901941098A0B379F50196E
:10FD100091094A0B8A0B279F901941098A0BF79F7B
:10FD200040198109E69FF12D33272227EB9FF00D23
:10FD3000311D2A1F769FF00D311D2A1F7B9F300D2C
:10FD4000211DE32F722F309198023E9F510D9A1F73
:10FD50004A1F8A1F209199022E9F500D911D4A1F04
:10FD60008A1FF0919A02FE9F900D411D8A1F379FB6
:10FD7000500D911D4A1F8A1F279F900D411D8A1FFC
:10FD8000F79F400D811D1124FA87EB877C876D87D3
:10FD9000BE875F87388B298B542F492F70E0682FDF
:10FDA00029CE2A893B89225B3F4FD9014D915D9134
:10FDB0006D917C911FCEDB01CA01B695A7959795F1
:10FDC00087958C7F87589E4DFC01C590D490FC018F
:10FDD0003296259134914770429FC001439F900D08
:10FDE0001124A3E096958795AA95E1F7C81AD90A38
:10FDF000F12CE12C4DCE80915C0190915D01A091A0
:10FE00005E01B0915F01B7FF61C0EA89FB89EA5BDF
:10FE1000FF4FC080D180E280F38089E799E221E042
:10FE2000FC0145915591659174914C155D056E05E8
:10FE30007F0558F4F694E794D794C794220F04965C
:10FE400045E959E24817590759F720933B0650E214
:10FE5000C516D104E104F10428F470E2C72ED12CB8
:10FE6000E12CF12C60E2C61AD108E108F108C114B6
:10FE700078E0D706E104F10408F431C0A4E0DA9E8A
:10FE8000C001112487589A4DFC0132962591349176
:10FE9000BC2D6627B39FA001B29F410D561F06944B
:10FEA000461F561F112470E060E0FC01859194917B
:10FEB000B0E0A0E0841B950BA60BB70B80935C0110
:10FEC00090935D01A0935E01B0935F01C0905C01CF
:10FED000D0905D01E0905E01F0905F0101CBD70111
:10FEE000C601B695A795979587958C7F87589E4DA7
:10FEF000FC0125913491FC01329645915491EC2DF1
:10FF0000E770E49FC001E59F900D112463E0969592
:10FF100087956A95E1F7281B390BC901B0E0A0E08D
:10FF2000CDCFEA89FB8985889688A788B08C81E047
:10FF300081149104A104B10409F480E0AA89BB8969
:10FF40005996CD90DD90ED90FC905C97C114D10452
:10FF5000E104F10409F08260EA89FB89458D568D40
:10FF6000678D70A1411551056105710509F0846027
:10FF70008093440610923206109233061092340693
:10FF80001092350610923C0610923D0610923E06E5
:10FF900010923F06EA89FB8985A196A1A7A1B0A589
:10FFA0008093450690934606A0934706B093480673
:10FFB000442455243201481A590A6A0A7B0A40929D
:10FFC00022065092230660922406709225064092E3
:10FFD00026065092270660922806709229064092C3
:10FFE0002A0650922B0660922C0670922D0641A094
:10FFF00052A063A074A0440C551C661C771C880C8E
:020000021000EC
:10000000991CAA1CBB1C8092120690921306A09207
:100010001406B0921506CC0CDD1CEE1CFF1CC09221
:100020001606D0921706E0921806F0921906440FB1
:10003000551F661F771F40931A0650931B06609347
:100040001C0670931D0640921E0650921F06609279
:10005000200670922106880F991FAA1FBB1F80934C
:100060000E0690930F06A0931006B09311061092FF
:10007000490610924A0610924B0610924C0681A532
:1000800092A5A3A5B4A58093400690934106A093A2
:100090004206B093430685A596A5A7A5B0A980936F
:1000A000370690933806A0933906B0933A06EB5B77
:1000B000FF4F80819091E506891721F08093E50636
:1000C0000E9432730E94337744244A94542C3201A4
:1000D00040925C0150925D0160925E0170925F01FE
:1000E000EA89FB89FD96E080F18002811381AA896B
:1000F000BB89D1962D913D914D915C91D4976D0125
:10010000BAE4CB0ED11CF6016081718182819381AA
:100110000E94806310923606D6014D915D916D91DB
:100120007C9189E799E2A1E0FC0105911591259167
:100130003491041715072607370758F47695679505
:1001400057954795AA0F0496E5E9F9E2E817F907EC
:1001500059F7A0933B06403251056105710520F423
:1001600040E250E060E070E04052510961097109DD
:100170004115F8E05F076105710508F462C024E0ED
:10018000529FC001112487589A4DFC013296259147
:100190003491AA27439FF001429FE10DFA1F069474
:1001A000EA1FFA1F1124AF0170E060E0FC01C59066
:1001B000D490F12CE12CC41AD50AE60AF70AC092B1
:1001C0004D06D0924E06E0924F06F0925006809176
:1001D0004D0690914E06A0914F06B0915006AC018D
:1001E000BD01009731E0A307B10520F04FEF5FEFAD
:1001F00060E070E0841B950BA60BB70B80934D0657
:1002000090934E06A0934F06B0935006F8948091B9
:100210008400909185004096A981A150A983AA23CA
:1002200081F1240E351E2816390610F40C94067838
:10023000309289002092880078946396E2E10C94D1
:10024000F7EEDB01CA01B695A795979587958C7F48
:1002500087589E4DFC01C590D490FC0132962591A3
:1002600034914770429FC001439F900D112433E0A9
:10027000969587953A95E1F7C81AD90AF12CE12CA1
:100280009ECF1C01D5CF80EDC82E87E0D82EE12C63
:10029000F12C2DC9CF93DF938091371390913813B0
:1002A000891B80958F7019F40E940B41F5CF8091C6
:1002B00037138F5F8F70A09137139BE5A99FD001F3
:1002C0001124FD01E756F84FEF0119929A95E9F7CD
:1002D00098E09083A255B84F90E1E9E3F3E10190F3
:1002E0000D929A95E1F720913713909138132913C5
:1002F00003C094E690933413809337130E941177D0
:10030000DF91CF910895FC01208131814281538199
:1003100060916A0D70916B0D80916C0D90916D0DD7
:100320000E945AE80E94B7F06093451370934613F9
:10033000809347139093481390913713809138130B
:10034000981709F0A7CF0E9430740E94047740915B
:100350004513509146136091471370914813409391
:100360006C0650936D0660936E0670936F06811154
:100370000C94117708954F925F926F927F928F92B3
:100380009F92AF92BF92CF92DF92EF92FF92CF9364
:10039000DF93EC0120916A0D30916B0D40916C0D53
:1003A00050916D0D6C857D858E859F850E945AE8E4
:1003B0000E94B7F06B017C012091660D3091670DB2
:1003C0004091680D5091690D688579858A859B8576
:1003D0000E945AE80E94B7F04B015C012091620D27
:1003E0003091630D4091640D5091650D6C817D815C
:1003F0008E819F810E945AE80E94B7F02B013C0138
:1004000020915E0D30915F0D4091600D5091610D16
:10041000688179818A819B810E945AE80E94B7F0A5
:100420006093391370933A1380933B1390933C136A
:1004300040923D1350923E1360923F1370924013CE
:100440008092411390924213A0924313B0924413AE
:10045000C0924513D0924613E0924713F09248138E
:100460009091371380913813981781F013DFDF9143
:10047000CF91FF90EF90DF90CF90BF90AF909F9083
:100480008F907F906F905F904F9008950E9430748E
:100490000E940477C82F89E393E10E947763CC23FD
:1004A00031F30E941177E3CFCF92DF92EF92FF9268
:1004B000CF93DF93C82F0E94047794E0C99FE00197
:1004C0001124FE01E05AF94FC080D180E280F38010
:1004D00081110E941177C757D84FC701B6010E94FA
:1004E000FBE7288139814A815B810E945AE8DF91CC
:1004F000CF91FF90EF90DF90CF9008958F929F92D1
:10050000AF92BF92CF92DF92EF92FF921F93CF9361
:10051000DF93CDB7DEB760970FB6F894DEBF0FBE9E
:10052000CDBF182F80E0C0DF4B015C018092E60553
:100530009092E705A092E805B092E90581E0B4DF6A
:100540006B017C01C092EA05D092EB05E092EC05CC
:10055000F092ED0582E0A8DF6093EE057093EF0561
:100560008093F0059093F1051D861E861F86188ADC
:1005700089829A82AB82BC82CD82DE82EF82F8864B
:1005800069877A878B879C8783E08EDF6D877E877C
:100590008F87988BCE0101960E9452741E3FD9F42A
:1005A00080E1FE013196A7E7B1E001900D928A95B6
:1005B000E1F760960FB6F894DEBF0FBECDBFDF91B6
:1005C000CF911F91FF90EF90DF90CF90BF90AF90B1
:1005D0009F908F90089584E0189FF0011124DF010F
:1005E000A958BE4F81E090E08C0F9D1FE80FF91FC6
:1005F00040815181628173814D935D936D937C93B2
:100600001397D7CFCF92DF92EF92FF92CF93DF93E2
:10061000C82F0E94047794E0C99FE0011124FE01D5
:10062000EC5AF94FC080D180E280F38081110E94A2
:100630001177C757D84FC701B6010E94FBE7288141
:1006400039814A815B810E945AE8DF91CF91FF9006
:10065000EF90DF90CF900895A1E0B0E0E2E3F3E8FF
:100660000C94EBEE898360E0CE0101960E94D26487
:1006700061E0CE0101960E94D26462E0CE01019653
:100680000E94D26489812196E2E00C9407EFA2E1F6
:10069000B0E0EDE4F3E80C94E7EEDEDF8823C1F18F
:1006A000EDB6FEB647E952E082FF02C04EE852E0E6
:1006B00027E932E081FF02C020E932E080FD25C059
:1006C00087E992E05F934F933F932F939F938F938C
:1006D0008AE09EE19F938F938E010F5F1F4F1F93C0
:1006E0000F930E948EE70E94FC3DC8010E944F3488
:1006F000C8010E9481C20FB6F894DEBF0FBECDBF05
:1007000081E06296E6E00C9403EF82E992E0DACFB2
:1007100080E0F7CFA0E2B0E0E0E9F3E80C94DBEE94
:1007200080913B01882309F4BEC08091F805082F11
:1007300010E080FF3CC0C0903D01D0903E01E090B1
:100740003F01F0904001209188043091890440914C
:100750008A0450918B04C701B6010E94B2F01816AA
:1007600044F4C0928804D0928904E0928A04F09202
:100770008B04C0904901D0904A01E0904B01F09069
:100780004C01209188043091890440918A04509151
:100790008B04C701B6010E94F5E787FF08C0C0922D
:1007A0008804D0928904E0928A04F0928B0401FFBD
:1007B0003CC0C0904101D0904201E0904301F090D4
:1007C000440120918C0430918D0440918E0450910D
:1007D0008F04C701B6010E94B2F0181644F4C0920B
:1007E0008C04D0928D04E0928E04F0928F04C0901D
:1007F0004D01D0904E01E0904F01F09050012091BA
:100800008C0430918D0440918E0450918F04C70167
:10081000B6010E94F5E787FF08C0C0928C04D09211
:100820008D04E0928E04F0928F0402FF3CC0C090D1
:100830004501D0904601E0904701F0904801209199
:100840009004309191044091920450919304C70117
:10085000B6010E94B2F0181644F4C0929004D092EF
:100860009104E0929204F0929304C0905101D090D0
:100870005201E0905301F090540120919004309186
:1008800091044091920450919304C701B6010E94D3
:10089000F5E787FF08C0C0929004D0929104E092DF
:1008A0009204F09293048091490D83FD61C02091E0
:1008B00083013091840140918501509186016091BE
:1008C00094047091950480919604909197040E94ED
:1008D000F5E7882309F44CC00E94D4B3182F88236D
:1008E00031F00E94FC3D8FEE9DE10E945E3420912C
:1008F000830130918401409185015091860160917E
:1009000094047091950480919604909197040E94AC
:1009100012EF9F7720917101309172014091730124
:10092000509174010E945AE820E030E046E154E41E
:100930000E94B2F01816D4F40E94FC3D80ED9DE1B7
:100940000E945E348091940490919504A091960445
:10095000B09197048093830190938401A0938501C3
:10096000B093860184E994E0CEDC02C01111EACF95
:100970002AE037ED43E25CE3609135017091360186
:1009800080913701909138010E945AE86B017C01F7
:100990006091390170913A01072E000C880B990B78
:1009A0000E94FBE79B01AC01C701B6010E945AE817
:1009B000698B7A8B8B8B9C8B80919804882309F1AF
:1009C0008090990490909A04A0909B04B0909C040D
:1009D000C0909004D0909104E0909204F090930421
:1009E00020E030E0A901C501B4010E94F5E78823A9
:1009F000F9F0A7019601C501B4010E94B2F01816E2
:100A0000BCF020E030E0A901BE016F5E7F4F88E8B6
:100A100094E00E94F5C380E1E8E8F4E0A7E7B1E0E4
:100A200001900D928A95E1F7A096E2E10C94F7EE21
:100A300020917701309178014091790150917A01AC
:100A4000609188047091890480918A0490918B044C
:100A50000E9412EF4B015C0120917B0130917C01DF
:100A600040917D0150917E0160918C0470918D04C4
:100A700080918E0490918F040E9412EF6D8B7E8B7B
:100A80008F8B988F20917F0130918001409181015F
:100A900050918201C701B6010E9412EF6D8F7E8FC7
:100AA0008F8F98A32091830130918401409185011B
:100AB0005091860160919404709195048091960400
:100AC000909197040E9412EF698F7A8F8B8F9C8F81
:100AD00020E030E0A901C501B4010E94F5E78111D1
:100AE0000CC020E030E0A9016D897E898F89988D46
:100AF0000E94F5E7882309F484CFA5019401C5017C
:100B0000B4010E945AE86B017C012D893E894F890E
:100B1000588DCA01B9010E945AE89B01AC01C70176
:100B2000B6010E9413EF6B017C012D8D3E8D4F8D20
:100B300058A1CA01B9010E945AE89B01AC01C70142
:100B4000B6010E9413EF6B017C01298D3A8D4B8D0C
:100B50005C8DCA01B9010E945AE89B01AC01C70132
:100B6000B6010E9413EF6B017C010E94F1F02B0192
:100B70003C012CEC3CEB4CE85BE2C701B6010E9467
:100B8000F5E787FF06C0498C5A8C6B8C7C8CE89407
:100B900077F82DEB37E346E855E3C301B2010E9435
:100BA000F5E787FD38CF2DEC3CEC4CE45EE3C30168
:100BB000B2010E945AE80E94FAEF1B01672B19F458
:100BC00022242394312CB10190E080E00E94F9E7C7
:100BD0009B01AC0160E070E080E89FE30E948DEF34
:100BE0006B017C01AC019B01C301B2010E945AE878
:100BF0002B013C01A7019601C501B4010E945AE8EE
:100C00004B015C01A70196016D897E898F89988DC2
:100C10000E945AE86D8B7E8B8F8B988FA70196016F
:100C20006D8D7E8D8F8D98A10E945AE86D8F7E8F7D
:100C30008F8F98A3A7019601698D7A8D8B8D9C8DDE
:100C40000E945AE8698F7A8F8B8F9C8F80E1E7E74B
:100C5000F1E08E010F5F1F4FD80101900D928A9530
:100C6000E1F70E943ECE6B017C0128ECC20ED11C44
:100C7000E11CF11C81E0281A310809F454C00E94DB
:100C80003ECE9B01AC012C193D094E095F0957FD71
:100C90004DC06B017C0128ECC20ED11CE11CF11C83
:100CA00080E00E940B41A501940169817A818B81CA
:100CB0009C810E9413EF69837A838B839C832D89A7
:100CC0003E894F89588D6D817E818F8198850E94E4
:100CD00013EF6D837E838F8398872D8D3E8D4F8D8F
:100CE00058A169857A858B859C850E9413EF698759
:100CF0007A878B879C87298D3A8D4B8D5C8D6D858E
:100D00007E858F8598890E9413EF6D877E878F87F8
:100D1000988BA3019201BE016F5E7F4FC8010E94B4
:100D2000F5C38111A7CFA30192016ECE0E94E57198
:100D3000BACF8091F4059091F505A091F605B09198
:100D4000F7058093350190933601A0933701B09356
:100D500038018091F2059091F30590933A018093C8
:100D6000390108958091350190913601A0913701A4
:100D7000B09138018093F4059093F505A093F605A2
:100D8000B093F7058091390190913A019093F30562
:100D90008093F20584E690E090933A0180933901C4
:100DA0000895ACE0B0E0E7EDF6E80C94DDEE2B0141
:100DB0003C0129873A874B875C8747015801D60158
:100DC000CD90DD90ED90FC9020E030E0A901C701CE
:100DD000B6010E94F5E7811171C080916D0190917B
:100DE0006E01A0916F01B091700189839A83AB83EA
:100DF000BC8320E030E0A901C701B6010E94F5E7FD
:100E0000811106C0C12CD12C80E8E82E80E4F82E98
:100E1000CD82DE82EF82F886A501940160917F0188
:100E20007091800180918101909182010E94F5E78B
:100E300087FF0CC080927F0190928001A092810177
:100E4000B0928201CE0105960E94E46B4092770138
:100E5000509278016092790170927A0189859A8521
:100E6000AB85BC8580937B0190937C01A0937D0131
:100E7000B0937E01CE0101960E94E46BA50194011E
:100E800060917F0170918001809181019091820138
:100E90000E94B2F0181664F480927F019092800153
:100EA000A0928101B0928201CE0105960E94E46B6E
:100EB0000E9430742C96E0E10C94F9EED701C60143
:100EC00094CFCF92DF92EF92FF920F931F936B011B
:100ED000FC01E080F18002811381E7E7F1E02481E9
:100EE000358146815781608171818281938159DF8B
:100EF0001F910F91FF90EF90DF90CF9008950C9489
:100F000018C40F931F93CF93DF93EC018B010E94C2
:100F1000D33F882331F081E0DF91CF911F910F9172
:100F20000895B801CE01CDDF80912A07C82FC47083
:100F300082FD0AC010922A0782E0E0DAE0DF81E059
:100F4000CC2351F380E0E8CF0E94923F882391F3B5
:100F5000E2CFCF930E940477C82F809138138093FB
:100F60003713809336138093351384E680933413BC
:100F70000E94957780ED93E09093930D8093920D6E
:100F8000C1110E94117781E0809353060E94307452
:100F90008EEFB4DAB4DFCF910895ACE0B0E0E3EDCA
:100FA000F7E80C94EBEE0E9493B30E9404779CE068
:100FB000E0E6F6E0DE01119601900D929A95E1F7D8
:100FC00081110E941177CE0101960E94AA722C967F
:100FD000E2E00C9407EFB0E0A0E0E1EFF7E80C945A
:100FE000DDEE40907701509078016090790170902B
:100FF0007A0180907B0190907C01A0907D01B0905F
:101000007E01C0907F01D0908001E0908101F0903E
:1010100082010E94C4736091550170915601072EA0
:10102000000C880B990B0E94FBE72AE037ED43E2A6
:101030005CE30E945AE8609371017093720180939F
:101040007301909374010DE311E0D0E0C0E0CE0194
:10105000835D9E4D0E94C627F80161937193819331
:1010600091938F01CE018F5D9E4D0E94C627F8019E
:1010700060877187828793872496CC30D10539F7B2
:1010800060E086E096E00E94AA2A0E94772B0E94E8
:101090000874A301920160917701709178018091A9
:1010A000790190917A010E94F5E781111BC0A50199
:1010B000940160917B0170917C0180917D01909100
:1010C0007E010E94F5E781110DC020917F013091D2
:1010D00080014091810150918201C701B6010E94B7
:1010E000F5E781115ADFCDB7DEB7E0E10C94F9EEF8
:1010F000A4E0B0E0EEE7F8E80C94EBEE84EF91E0CA
:10110000A0E0B0E089839A83AB83BC83BE016F5FAC
:101110007F4F8CE30E94053386EB9DE10E945E3495
:1011200086B160EB7DE182FB882780F90E94726BBB
:1011300086B16AEA7DE183FB882780F90E94726BA1
:1011400086B164EA7DE1829581700E94726B80B104
:101150006BE97DE182FB882780F90E94726B3499EC
:1011600007C00E9439332496E2E00C9407EF06C0D2
:101170000E9422332496E2E00C9407EF8091E4066B
:10118000811103C08091E60681110C943377089594
:10119000ACE0B0E0EEECF8E80C94EBEEAAE4BDE0D5
:1011A00090E080E0FC01E759FE4D45915591659135
:1011B00074914D935D936D937D93FC01E75AFE4DC1
:1011C000459155916591749150964D935D936D93B2
:1011D0007C935397FC01E75BFE4D459155916591DA
:1011E000749190964D935D936D937C939397049631
:1011F00080319105B9F680E29EE4A0E0B0E08093F2
:101200005A0D90935B0DA0935C0DB0935D0D80E043
:1012100090E0AAEFB3E480937E0D90937F0DA093AE
:10122000800DB093810D8093820D9093830DA093D8
:10123000840DB093850D8093860D9093870DA093B8
:10124000880DB093890D10928A0D10928B0D10921B
:101250008C0D10928D0D10928E0D10928F0D10929C
:10126000900D1092910D8AE097EDA3EABDE3809373
:101270006C0790936D07A0936E07B0936F07109261
:101280005B010E941E1A80E090E0A0EEB0E4809323
:10129000570190935801A0935901B0935A0180E0EF
:1012A00090E0A0E2B1E48093060690930706A09335
:1012B0000806B09309060E94602A8CE0E3EBF1E097
:1012C000DE01119601900D928A95E1F789819A814C
:1012D000AB81BC818093261390932713A09328138E
:1012E000B09329138D819E81AF81B88580932A1395
:1012F00090932B13A0932C13B0932D1389859A856B
:10130000AB85BC8580932E1390932F13A09330133D
:10131000B09331138EEB90E090937205809371053A
:10132000109274051092730586EE90E09093760506
:101330008093750510927805109277058FE892ECEE
:10134000ADE8B1E48093961290939712A09398120F
:10135000B09399128CE998EFA5E4BEE380939A12BA
:1013600090939B12A0939C12B0939D1281E49CEBEE
:10137000ABECB3E480939E1290939F12A093A012C3
:10138000B093A1121092E4061092E306F7DE23DE7A
:101390002C96E2E00C9407EFFBCEA4E0B0E0E3ED86
:1013A000F9E80C94DCEE9091E606981709F455C024
:1013B000382E80E090E0A0E2B1E489839A83AB8389
:1013C000BC83C0902E13D0902F13E0903013F09078
:1013D000311320E030E0A901C701B6010E94F5E712
:1013E00087FF0CC0A701960160E070E080E291E405
:1013F0000E9412EF69837A838B839C83CE010196CE
:101400000E94A9C4409077015090780160907901C2
:1014100070907A0180907B0190907C01A0907D017A
:10142000B0907E013320F1F00E94D33F19821A82DE
:101430001B821C82E0907F01F0908001009181016D
:1014400010918201CE0101966C01A5019401C301A6
:10145000B201A7DC3092E60691DE80E02496E1E15D
:101460000C94F8EE0E94923FE1CFB0E0A0E0EBE3F5
:10147000FAE80C94DDEEC82FE82EF12CF701E352C8
:10148000F14DD491823071F481E087DF811105C084
:101490000E94D33F882309F4E2C0CDB7DEB7E0E174
:1014A0000C94F9EE6D2FDD0F770B880B990B0E94D2
:1014B000FBE72B013C01C701880F991F880F991F7B
:1014C000875A914E0E94C6274B015C01A3019201ED
:1014D000C501B4010E945AE84B015C016701CC0CC4
:1014E000DD1CCC0CDD1CC601835B914E0E94C6271F
:1014F000A30192010E945AE820E030E040EC5FE353
:101500000E945AE8AB01BC0100E010E098018C2F6A
:101510000E94FFC7C23009F0CCC00E94923F20E079
:1015200030E0A901C501B4010E94F5E7882329F143
:1015300000E010E020E830E4B501A40170588C2FE1
:101540000E94FFC7C23009F467C0A5019401C5011C
:10155000B4010E9413EF4B015C01C23009F062C07C
:1015600000E010E020E030E4B501A4018C2F0E94DF
:10157000FFC7C23011F40E94923F81E090E00C2E30
:1015800001C0880F0A94EAF790915807982B90931E
:1015900058079091F805892B8093F805C6018F5B59
:1015A000914E0E94C627F601E958FE4F6083718371
:1015B00082839383C230D1F420912E1330912F1364
:1015C000409130135091311360917F0170918001EF
:1015D00080918101909182010E9412EF60937F01BE
:1015E00070938001809381019093820188DCF601E1
:1015F000E857FB4FD601A958BE4F8D919D910D9094
:10160000BC91A02D80839183A283B383C23009F063
:1016100044CF0E94CC2741CF0E94D33F882309F4B6
:1016200094CF3BCFF701E25CF14E6491611107C0AA
:101630000E94FC3D8CE19EE10E945E346AE070E015
:1016400090E080E00E94F9E79B01AC0161E070E06E
:1016500088E492E40E948DEF8B019C0185CF81E6A6
:101660009EE10E94C62720E030E0A9010E94F5E734
:10167000882309F417CF6D2FDD0F770B880B990B9B
:101680000E94FBE72B013C0181E69EE10E94C627F8
:101690004B015C0120E030E040EA50E40E94B2F0EF
:1016A00087FF14CF812C912C90EAA92E90E4B92EBB
:1016B0000DCF20E030E0A901C501B4010E94F5E79B
:1016C000882309F45ACF00E010E0980135CF8091CB
:1016D0002A07882319F010922A07089540E070E045
:1016E00060E08BE79DE10E941A401F920F920FB6B7
:1016F0000F9211240BB60F922F933F934F935F934A
:101700006F937F938F939F93AF93BF93EF93FF93C9
:101710000E943377FF91EF91BF91AF919F918F918D
:101720007F916F915F914F913F912F910F900BBEE1
:101730000F900FBE0F901F9018950F931F938091DD
:101740006807813019F50E943ECE0091DD051091A9
:10175000DE052091DF053091E005601B710B820BE7
:10176000930B28EE33E040E050E00E9423EE6091BE
:10177000D9057091DA058091DB059091DC05620F47
:10178000731F841F951F1F910F9108956091E105AC
:101790007091E2058091E3059091E405D6CF109217
:1017A00068071092DD051092DE051092DF05109299
:1017B000E0051092E1051092E2051092E305109207
:1017C000E4051092D9051092DA051092DB0510920B
:1017D000DC050895809168078130E1F08230C1F422
:1017E000ACDF6093D9057093DA058093DB059093A5
:1017F000DC0581E0809368070E943ECE6093DD05A2
:101800007093DE058093DF059093E00581E00895F5
:10181000C6DFEFCF80E008950E94F7C40E94112C2C
:10182000882351F08091A11482FD06C08BED98E1D0
:101830009093E9068093E806CDCF809168078130C8
:1018400079F482E0809368070E943ECE6093E105C0
:101850007093E2058093E3059093E40581E0089599
:1018600080E00895809168078150823070F4109272
:1018700068070E943ECE6093E1057093E205809375
:10188000E3059093E40581E0089580E008959C01CC
:1018900097FF26C0EE27FF27E81BF90B2D398FEFA6
:1018A00038070CF05DC08DE280938304CF0164E6BD
:1018B00070E00E94ADEECB012AE030E0B9010E9459
:1018C000ADEE805D80938404CF01B9010E94ADEE3E
:1018D000CB01B9010E94ADEE805D809385042AC0E2
:1018E000283E83E03807B4F1C90168EE73E00E9436
:1018F000ADEECB01EAE0F0E0BF010E94ADEE805D0D
:1019000080938304C90164E670E00E94ADEECB01D0
:10191000BF010E94ADEE805D80938404C901BF01C8
:101920000E94ADEECB01BF010E94ADEE805D8093C1
:101930008504F901CF016AE070E00E94ADEE805DA0
:101940008093860483E894E008958DE237FDC5CF47
:1019500080E2C3CFF90180E2243631050CF0A4CF38
:1019600080E28093830480938404EA30F1056CF371
:101970008DE237FF80E280938404CF016AE070E05B
:101980000E94ADEE605D60938504D4CF9C0197FD0D
:101990002DC080E2243631055CF0C90164E670E0B8
:1019A0000E94ADEECB016AE070E00E94ADEE805D7A
:1019B0008093840480E22A3031055CF0EAE0F0E0B4
:1019C000C901BF010E94ADEECB01BF010E94ADEE87
:1019D000805D80938504C9016AE070E00E94ADEEED
:1019E000805D8093860484E894E008953195219584
:1019F00031098DE2DDCFCF92DF92EF92FF92FC01B1
:101A0000C080D180E280F38020E030E0A901C701EE
:101A1000B6010E94F5E787FD26C06DEB77E386E00F
:101A200095E3A70196010E9413EF6B017C0120E072
:101A300030E0A9010E94F5E720E030E040E05FE3FC
:101A400087FF04C020E030E040E05FEBC701B60153
:101A50000E9413EF0E94F5EFCB0198DFFF90EF900B
:101A6000DF90CF9008956DEB77E386E095EBD9CFCB
:101A7000A4E0B0E0EEE3FDE80C94EBEE0E94FBE79F
:101A800069837A838B839C83CE010196B4DF24968D
:101A9000E2E00C9407EFFC01608171818281938107
:101AA0000E94F5EFCB0172CFA4E0B0E0EAE5FDE8DB
:101AB0000C94EBEE0E94FBE769837A838B839C8313
:101AC000CE010196E8DF2496E2E00C9407EF8F92B6
:101AD0009F92AF92BF92EF92FF920F931F93CF937B
:101AE000DF93EC018B01E42EF22E8091491390914B
:101AF0004A138C179D07C9F129EAC431D20709F0AE
:101B00003FC08F519C4271F40E943ECE6E517B4F7C
:101B10008F4F9F4F6093C9057093CA058093CB0583
:101B20009093CC05D0934A13C093491330E020E042
:101B300000934B0710934C0720934D0730934E07AB
:101B4000E0924607F0924707CF51DC4221F4109211
:101B50007F041092C80582E080936C0181E080933D
:101B6000480710927E041092D405DF91CF911F9107
:101B70000F91FF90EF90BF90AF909F908F9008953E
:101B80002CE2CF31D20771F68451994AD9F40E94E0
:101B90003ECE8090C9059090CA05A090CB05B0902C
:101BA000CC05681979098A099B0997FF0BC08091B8
:101BB00058078770873031F40E94AC6CCCECDDE9BB
:101BC0008111B0CFCFE1DCE2ADCF20E040E070E0AA
:101BD00060E08BE99CE67BCF0E94D4B3882339F088
:101BE00020E040E070E060E08EEE9CE970CFEDCF49
:101BF00021E020937F04FC0180819181A281B38147
:101C00008093310190933201A0933301B09334015A
